******************************************************************************
                  TI ARM Linker PC v18.1.3                     
******************************************************************************
>> Linked Thu Nov  8 15:07:37 2018

OUTPUT FILE NAME:   <pdmstream_CC1350STK_TI.out>
ENTRY POINT SYMBOL: "ResetISR"  address: 00006835


MEMORY CONFIGURATION

         name            origin    length      used     unused   attr    fill
----------------------  --------  ---------  --------  --------  ----  --------
  FLASH                 00000000   00020000  000073bc  00018c44  R  X
  GPRAM                 11000000   00002000  00000000  00002000  RW X
  SRAM                  20000000   00005000  00003cb1  0000134f  RW X


SEGMENT ALLOCATION MAP

run origin  load origin   length   init length attrs members
----------  ----------- ---------- ----------- ----- -------
00000000    00000000    00000728   00000728    r--
  00000000    00000000    0000003c   0000003c    r-- .resetVecs
  0000003c    0000003c    0000044c   0000044c    r-- .const
  00000488    00000488    000002a0   000002a0    r-- .cinit
00001000    00001000    00006c48   00006c48    r-x
  00001000    00001000    0000003c   0000003c    r-- .const:ti_sysbios_knl_Task_Object__PARAMS__C
  0000103c    0000103c    00000034   00000034    r-- .const:ti_sysbios_knl_Mailbox_Object__PARAMS__C
  00001070    00001070    00000030   00000030    r-- .const:ti_sysbios_family_arm_m3_Hwi_Object__PARAMS__C
  000010a0    000010a0    0000002c   0000002c    r-- .const:ti_sysbios_hal_Hwi_Object__PARAMS__C
  000010cc    000010cc    00000028   00000028    r-- .const:ti_sysbios_heaps_HeapMem_Module__FXNS__C
  000010f4    000010f4    00000028   00000028    r-- .const:ti_sysbios_knl_Swi_Object__PARAMS__C
  0000111c    0000111c    00000024   00000024    r-- .const:ti_sysbios_gates_GateHwi_Module__FXNS__C
  00001140    00001140    00000024   00000024    r-- .const:ti_sysbios_gates_GateMutex_Module__FXNS__C
  00001164    00001164    00000024   00000024    r-- .const:ti_sysbios_heaps_HeapMem_Object__PARAMS__C
  00001188    00001188    00000024   00000024    r-- .const:ti_sysbios_knl_Clock_Object__PARAMS__C
  000011ac    000011ac    00000024   00000024    r-- .const:ti_sysbios_knl_Semaphore_Object__PARAMS__C
  000011d0    000011d0    00000020   00000020    r-- .const:ti_sysbios_family_arm_m3_Hwi_Object__DESC__C
  000011f0    000011f0    00000020   00000020    r-- .const:ti_sysbios_gates_GateHwi_Object__DESC__C
  00001210    00001210    00000020   00000020    r-- .const:ti_sysbios_gates_GateMutex_Object__DESC__C
  00001230    00001230    00000020   00000020    r-- .const:ti_sysbios_hal_Hwi_Object__DESC__C
  00001250    00001250    00000020   00000020    r-- .const:ti_sysbios_heaps_HeapMem_Object__DESC__C
  00001270    00001270    00000020   00000020    r-- .const:ti_sysbios_knl_Clock_Object__DESC__C
  00001290    00001290    00000020   00000020    r-- .const:ti_sysbios_knl_Mailbox_Object__DESC__C
  000012b0    000012b0    00000020   00000020    r-- .const:ti_sysbios_knl_Queue_Object__DESC__C
  000012d0    000012d0    00000020   00000020    r-- .const:ti_sysbios_knl_Semaphore_Object__DESC__C
  000012f0    000012f0    00000020   00000020    r-- .const:ti_sysbios_knl_Swi_Object__DESC__C
  00001310    00001310    00000020   00000020    r-- .const:ti_sysbios_knl_Task_Object__DESC__C
  00001330    00001330    00000018   00000018    r-- .const:ti_sysbios_gates_GateHwi_Object__PARAMS__C
  00001348    00001348    00000018   00000018    r-- .const:ti_sysbios_gates_GateMutex_Object__PARAMS__C
  00001360    00001360    00000018   00000018    r-- .const:ti_sysbios_knl_Queue_Object__PARAMS__C
  00001378    00001378    00000008   00000008    r-- .const:ti_sysbios_knl_Idle_funcList__C
  00001384    00001384    00000004   00000004    r-- .const:ti_sysbios_family_arm_cc26xx_Timer_startupNeeded__C
  00001388    00001388    00000004   00000004    r-- .const:ti_sysbios_family_arm_m3_Hwi_E_alreadyDefined__C
  0000138c    0000138c    00000004   00000004    r-- .const:ti_sysbios_family_arm_m3_Hwi_E_hwiLimitExceeded__C
  00001390    00001390    00000004   00000004    r-- .const:ti_sysbios_family_arm_m3_Hwi_NUM_INTERRUPTS__C
  00001394    00001394    00000004   00000004    r-- .const:ti_sysbios_family_arm_m3_Hwi_Object__count__C
  00001398    00001398    00000004   00000004    r-- .const:ti_sysbios_family_arm_m3_Hwi_Object__table__C
  0000139c    0000139c    00000004   00000004    r-- .const:ti_sysbios_family_arm_m3_Hwi_ccr__C
  000013a0    000013a0    00000004   00000004    r-- .const:ti_sysbios_family_arm_m3_Hwi_excHandlerFunc__C
  000013a4    000013a4    00000004   00000004    r-- .const:ti_sysbios_family_arm_m3_Hwi_nullIsrFunc__C
  000013a8    000013a8    00000004   00000004    r-- .const:ti_sysbios_family_arm_m3_Hwi_numSparseInterrupts__C
  000013ac    000013ac    00000004   00000004    r-- .const:ti_sysbios_family_arm_m3_Hwi_priGroup__C
  000013b0    000013b0    00000004   00000004    r-- .const:ti_sysbios_family_arm_m3_TaskSupport_stackAlignment__C
  000013b4    000013b4    00000004   00000004    r-- .const:ti_sysbios_heaps_HeapMem_E_memory__C
  000013b8    000013b8    00000004   00000004    r-- .const:ti_sysbios_heaps_HeapMem_Module__gateObj__C
  000013bc    000013bc    00000004   00000004    r-- .const:ti_sysbios_heaps_HeapMem_Object__count__C
  000013c0    000013c0    00000004   00000004    r-- .const:ti_sysbios_heaps_HeapMem_Object__table__C
  000013c4    000013c4    00000004   00000004    r-- .const:ti_sysbios_heaps_HeapMem_reqAlign__C
  000013c8    000013c8    00000004   00000004    r-- .const:ti_sysbios_knl_Clock_serviceMargin__C
  000013cc    000013cc    00000004   00000004    r-- .const:ti_sysbios_knl_Mailbox_Object__count__C
  000013d0    000013d0    00000004   00000004    r-- .const:ti_sysbios_knl_Mailbox_Object__table__C
  000013d4    000013d4    00000004   00000004    r-- .const:ti_sysbios_knl_Mailbox_maxTypeAlign__C
  000013d8    000013d8    00000004   00000004    r-- .const:ti_sysbios_knl_Queue_Object__count__C
  000013dc    000013dc    00000004   00000004    r-- .const:ti_sysbios_knl_Queue_Object__table__C
  000013e0    000013e0    00000004   00000004    r-- .const:ti_sysbios_knl_Swi_Object__count__C
  000013e4    000013e4    00000004   00000004    r-- .const:ti_sysbios_knl_Swi_Object__table__C
  000013e8    000013e8    00000004   00000004    r-- .const:ti_sysbios_knl_Swi_numPriorities__C
  000013ec    000013ec    00000004   00000004    r-- .const:ti_sysbios_knl_Task_Object__count__C
  000013f0    000013f0    00000004   00000004    r-- .const:ti_sysbios_knl_Task_Object__table__C
  000013f4    000013f4    00000004   00000004    r-- .const:ti_sysbios_knl_Task_allBlockedFunc__C
  000013f8    000013f8    00000004   00000004    r-- .const:ti_sysbios_knl_Task_defaultStackHeap__C
  000013fc    000013fc    00000004   00000004    r-- .const:ti_sysbios_knl_Task_defaultStackSize__C
  00001400    00001400    00000004   00000004    r-- .const:ti_sysbios_knl_Task_numConstructedTasks__C
  00001406    00001406    00000002   00000002    r-- .const:ti_sysbios_family_arm_cc26xx_Timer_Module__id__C
  00001408    00001408    00000002   00000002    r-- .const:ti_sysbios_family_arm_cc26xx_TimestampProvider_useClockTimer__C
  0000140a    0000140a    00000002   00000002    r-- .const:ti_sysbios_family_arm_m3_Hwi_Module__id__C
  0000140c    0000140c    00000002   00000002    r-- .const:ti_sysbios_gates_GateHwi_Module__id__C
  0000140e    0000140e    00000002   00000002    r-- .const:ti_sysbios_gates_GateMutex_Module__id__C
  00001410    00001410    00000002   00000002    r-- .const:ti_sysbios_heaps_HeapMem_Module__id__C
  00001412    00001412    00000002   00000002    r-- .const:ti_sysbios_knl_Task_initStackFlag__C
  00001414    00001414    00000001   00000001    r-- .const:ti_sysbios_knl_Clock_tickMode__C
  00001418    00001418    00000008   00000008    r-- .const:xdc_runtime_Startup_firstFxns__C
  00001420    00001420    00000008   00000008    r-- .const:xdc_runtime_Startup_lastFxns__C
  00001428    00001428    00000004   00000004    r-- .const:xdc_runtime_Assert_E_assertFailed__C
  0000142c    0000142c    00000004   00000004    r-- .const:xdc_runtime_Error_E_memory__C
  00001430    00001430    00000004   00000004    r-- .const:xdc_runtime_Error_policyFxn__C
  00001434    00001434    00000004   00000004    r-- .const:xdc_runtime_IGateProvider_Interface__BASE__C
  00001438    00001438    00000004   00000004    r-- .const:xdc_runtime_IHeap_Interface__BASE__C
  0000143c    0000143c    00000004   00000004    r-- .const:xdc_runtime_IModule_Interface__BASE__C
  00001440    00001440    00000004   00000004    r-- .const:xdc_runtime_Main_Module__diagsEnabled__C
  00001444    00001444    00000004   00000004    r-- .const:xdc_runtime_Main_Module__diagsIncluded__C
  00001448    00001448    00000004   00000004    r-- .const:xdc_runtime_Main_Module__diagsMask__C
  0000144c    0000144c    00000004   00000004    r-- .const:xdc_runtime_Memory_defaultHeapInstance__C
  00001450    00001450    00000004   00000004    r-- .const:xdc_runtime_Startup_execImpl__C
  00001454    00001454    00000004   00000004    r-- .const:xdc_runtime_Startup_maxPasses__C
  00001458    00001458    00000004   00000004    r-- .const:xdc_runtime_Startup_sfxnRts__C
  0000145c    0000145c    00000004   00000004    r-- .const:xdc_runtime_Startup_sfxnTab__C
  00001460    00001460    00000004   00000004    r-- .const:xdc_runtime_Startup_startModsFxn__C
  00001464    00001464    00000004   00000004    r-- .const:xdc_runtime_SysCallback_abortFxn__C
  00001468    00001468    00000004   00000004    r-- .const:xdc_runtime_SysCallback_exitFxn__C
  0000146c    0000146c    00000004   00000004    r-- .const:xdc_runtime_System_abortFxn__C
  00001470    00001470    00000004   00000004    r-- .const:xdc_runtime_System_exitFxn__C
  00001474    00001474    00000004   00000004    r-- .const:xdc_runtime_System_maxAtexitHandlers__C
  00001478    00001478    00000004   00000004    r-- .const:xdc_runtime_Text_charTab__C
  0000147c    0000147c    00000004   00000004    r-- .const:xdc_runtime_Text_nameEmpty__C
  00001480    00001480    00000004   00000004    r-- .const:xdc_runtime_Text_nameStatic__C
  00001484    00001484    00000004   00000004    r-- .const:xdc_runtime_Text_nameUnknown__C
  00001488    00001488    00000002   00000002    r-- .const:xdc_runtime_Main_Module__id__C
  0000148a    0000148a    00000002   00000002    r-- .const:xdc_runtime_Memory_Module__id__C
  0000148c    0000148c    00000002   00000002    r-- .const:xdc_runtime_Text_charCnt__C
  0000148e    0000148e    00000002   00000002    r-- .const:xdc_runtime_Text_isLoaded__C
  00001490    00001490    00000001   00000001    r-- .const:xdc_runtime_Error_policy__C
  00001494    00001494    00000004   00000004    r-- .const:ti_sysbios_rom_ROM_AONRTCChannelEnable
  00001498    00001498    00000004   00000004    r-- .const:ti_sysbios_rom_ROM_AONRTCCompareValueSet
  0000149c    0000149c    00000004   00000004    r-- .const:ti_sysbios_rom_ROM_AONRTCCurrentCompareValueGet
  000014a0    000014a0    00000004   00000004    r-- .const:ti_sysbios_rom_ROM_AONRTCEventClear
  000014a4    000014a4    00000004   00000004    r-- .const:ti_sysbios_rom_ROM_ti_sysbios_family_arm_cc26xx_Timer_getCount64__E
  000014a8    000014a8    00000004   00000004    r-- .const:ti_sysbios_rom_ROM_ti_sysbios_family_arm_cc26xx_Timer_getCurrentTick__E
  000014ac    000014ac    00000004   00000004    r-- .const:ti_sysbios_rom_ROM_ti_sysbios_family_arm_cc26xx_Timer_getMaxTicks__E
  000014b0    000014b0    00000004   00000004    r-- .const:ti_sysbios_rom_ROM_ti_sysbios_family_arm_cc26xx_Timer_initDevice__I
  000014b4    000014b4    00000004   00000004    r-- .const:ti_sysbios_rom_ROM_ti_sysbios_family_arm_cc26xx_Timer_setNextTick__E
  000014b8    000014b8    00000004   00000004    r-- .const:ti_sysbios_rom_ROM_ti_sysbios_family_arm_cc26xx_Timer_setThreshold__I
  000014bc    000014bc    00000004   00000004    r-- .const:ti_sysbios_rom_ROM_ti_sysbios_family_arm_cc26xx_Timer_start__E
  000014c0    000014c0    00000004   00000004    r-- .const:ti_sysbios_rom_ROM_ti_sysbios_family_arm_cc26xx_TimestampProvider_get32__E
  000014c4    000014c4    00000004   00000004    r-- .const:ti_sysbios_rom_ROM_xdc_runtime_Startup_getState__I
  000014c8    000014c8    00000004   00000004    r-- .const:ti_sysbios_rom_ROM_xdc_runtime_System_SupportProxy_abort__E
  000014cc    000014cc    00000004   00000004    r-- .const:ti_sysbios_rom_ROM_xdc_runtime_System_SupportProxy_exit__E
  000014d0    000014d0    00000004   00000004    r-- .const:ti_sysbios_gates_GateMutex_Instance_State_sem__O
  000014d4    000014d4    00000004   00000004    r-- .const:ti_sysbios_knl_Clock_Module_State_clockQ__O
  000014d8    000014d8    00000004   00000004    r-- .const:ti_sysbios_knl_Mailbox_Instance_State_dataQue__O
  000014dc    000014dc    00000004   00000004    r-- .const:ti_sysbios_knl_Mailbox_Instance_State_dataSem__O
  000014e0    000014e0    00000004   00000004    r-- .const:ti_sysbios_knl_Mailbox_Instance_State_freeQue__O
  000014e4    000014e4    00000004   00000004    r-- .const:ti_sysbios_knl_Mailbox_Instance_State_freeSem__O
  000014e8    000014e8    00000004   00000004    r-- .const:ti_sysbios_knl_Semaphore_Instance_State_pendQ__O
  000014ec    000014ec    00000004   00000004    r-- .const:ti_sysbios_knl_Task_Module_State_inactiveQ__O
  000014f0    000014f0    00006758   00006758    r-x .text
0001ffa8    0001ffa8    00000058   00000058    r--
  0001ffa8    0001ffa8    00000058   00000058    r-- .ccfg
20000100    20000100    000038ee   00000000    rw-
  20000100    20000100    00000044   00000000    rw- .data:ti_sysbios_knl_Task_Module__state__V
  20000144    20000144    00000034   00000000    rw- .data:ti_sysbios_family_arm_m3_Hwi_Module__state__V
  20000178    20000178    0000002c   00000000    rw- .data:ti_sysbios_knl_Clock_Module__state__V
  200001a4    200001a4    00000024   00000000    rw- .data:ti_sysbios_BIOS_Module__state__V
  200001c8    200001c8    0000001c   00000000    rw- .data:ti_sysbios_knl_Swi_Module__state__V
  200001e4    200001e4    00000008   00000000    rw- .data:ti_sysbios_family_arm_cc26xx_Timer_Module__state__V
  200001ec    200001ec    00000004   00000000    rw- .data:ti_sysbios_family_arm_cc26xx_TimestampProvider_Module__state__V
  200001f0    200001f0    00000008   00000000    rw- .data:xdc_runtime_Startup_Module__state__V
  200001f8    200001f8    00000008   00000000    rw- .data:xdc_runtime_System_Module__state__V
  20000200    20000200    00000004   00000000    rw- .data:xdc_runtime_Memory_Module__state__V
  20000208    20000208    00003377   00000000    rw- .bss
  20003580    20003580    0000046e   00000000    rw- .data
20004d00    20004d00    00000300   00000000    rw-
  20004d00    20004d00    00000300   00000000    rw- .stack


SECTION ALLOCATION MAP

 output                                  attributes/
section   page    origin      length       input sections
--------  ----  ----------  ----------   ----------------
.const     0    0000003c    0000044c     
                  0000003c    000000b2     drivers_cc13xxware.aem3 : Codec1.oem3 (.const:Codec1_stepsizeLut)
                  000000ee    00000002     pdmstream_pem3.oem3 (.const:xdc_runtime_SysMin_flushAtExit__C)
                  000000f0    0000006c     drivers_cc13xxware.aem3 : PDMCC26XX.oem3 (.const:PDMCC26XX_aBqCoeffs)
                  0000015c    00000064     CC1350STK.obj (.const:BoardGpioInitTable)
                  000001c0    0000004c     drivers_cc13xxware.aem3 : PowerCC26XX.oem3 (.const:resourceDB)
                  0000020c    00000048     pdmstream_pem3.oem3 (.const:.string)
                  00000254    00000040     drivers_cc13xxware.aem3 : UARTCC26XX.oem3 (.const)
                  00000294    00000028                             : UARTCC26XX.oem3 (.const:UARTCC26XX_fxnTable)
                  000002bc    00000028     pdmstream_pem3.oem3 (.const:xdc_runtime_Startup_sfxnTab__A)
                  000002e4    00000024     drivers_cc13xxware.aem3 : PDMCC26XX.oem3 (.const:$P$T0$1)
                  00000308    00000024                             : UART.oem3 (.const:UART_defaultParams)
                  0000032c    00000020     pdmstream_pem3.oem3 (.const:ti_sysbios_knl_Event_Object__DESC__C)
                  0000034c    00000020     CC1350STK.obj (.const:uartCC26XXHWAttrs)
                  0000036c    0000001c     display.aem3 : DisplayUart.oem3 (.const)
                  00000388    00000018     CC1350STK.obj (.const:Display_config)
                  000003a0    00000018     CC1350STK.obj (.const:UART_config)
                  000003b8    00000018     pdmstream_pem3.oem3 (.const:ti_sysbios_knl_Event_Object__PARAMS__C)
                  000003d0    00000014     CC1350STK.obj (.const:displayUartHWAttrs)
                  000003e4    00000014     pdmstream_pem3.oem3 (.const:xdc_runtime_Startup_sfxnRts__A)
                  000003f8    00000010     drivers_cc13xxware.aem3 : Codec1.oem3 (.const:.string)
                  00000408    00000010     CC1350STK.obj (.const:PDMCC26XX_I2S_config)
                  00000418    00000010     CC1350STK.obj (.const:PowerCC26XX_config)
                  00000428    0000000c     CC1350STK.obj (.const:pdmC26XXI2SHWAttrs)
                  00000434    0000000c     pdmstream_pem3.oem3 (.const:xdc_runtime_Startup_firstFxns__A)
                  00000440    0000000a     drivers_cc13xxware.aem3 : PDMCC26XX.oem3 (.const)
                  0000044a    00000002     pdmstream_pem3.oem3 (.const:xdc_runtime_Text_registryModsLastId__C)
                  0000044c    00000008     CC1350STK.obj (.const:PDMCC26XX_config)
                  00000454    00000008     CC1350STK.obj (.const:PINCC26XX_hwAttrs)
                  0000045c    00000008     CC1350STK.obj (.const:pdmCC26XXHWAttrs)
                  00000464    00000004     pdmstream_pem3.oem3 (.const:ti_sysbios_knl_Clock_tickPeriod__C)
                  00000468    00000004     pdmstream_pem3.oem3 (.const:ti_sysbios_knl_Clock_triggerClock__C)
                  0000046c    00000004     pdmstream_pem3.oem3 (.const:ti_sysbios_knl_Event_Instance_State_pendQ__O)
                  00000470    00000004     pdmstream_pem3.oem3 (.const:ti_sysbios_knl_Idle_funcList__A)
                  00000474    00000004     pdmstream_pem3.oem3 (.const:xdc_runtime_SysMin_bufSize__C)
                  00000478    00000004     pdmstream_pem3.oem3 (.const:xdc_runtime_SysMin_outputFunc__C)
                  0000047c    00000004     pdmstream_pem3.oem3 (.const:xdc_runtime_System_extendFxn__C)
                  00000480    00000004     pdmstream_pem3.oem3 (.const:xdc_runtime_Text_visitRopeFxn__C)
                  00000484    00000002     pdmstream_pem3.oem3 (.const:xdc_runtime_Text_unnamedModsLastId__C)
                  00000486    00000001     display.aem3 : Display.oem3 (.const)
                  00000487    00000001     pdmstream_pem3.oem3 (.const:xdc_runtime_Text_charTab__A)

.text      0    000014f0    00006758     
                  000014f0    0000090c     pdm_cc13xxware.aem3 : pdm2pcm_ccs.oem3 (.text:pdm2pcm16k)
                  00001dfc    0000033c     rom_sysbios.aem3 : rom_sysbios.obj (.text:xdc_runtime_System_doPrint__I)
                  00002138    000002d8     drivers_cc13xxware.aem3 : PDMCC26XX.oem3 (.text:PDMCC26XX_taskFxn)
                  00002410    00000288     pdmstream.obj (.text:SA_processPDMData)
                  00002698    00000270     pdmstream.obj (.text:taskFxn)
                  00002908    00000240     pdmstream.obj (.text:main)
                  00002b48    00000228     driverlib.lib : sys_ctrl.obj (.text:NOROM_SysCtrlSetRechargeBeforePowerDown)
                  00002d70    00000228     drivers_cc13xxware.aem3 : PowerCC26XX.oem3 (.text:Power_sleep)
                  00002f98    000001ec                             : PowerCC26XX_calibrateRCOSC.oem3 (.text:calibrateRcoscHf1)
                  00003184    000001c4                             : PINCC26XX.oem3 (.text:PIN_init)
                  00003348    000001c0                             : PDMCC26XX_util.oem3 (.text:PDMCC26XX_I2S_open)
                  00003508    000001a0                             : PowerCC26XX_calibrateRCOSC.oem3 (.text:PowerCC26XX_doCalibrate)
                  000036a8    000001a0                             : UARTCC26XX.oem3 (.text:UARTCC26XX_open)
                  00003848    00000144                             : PDMCC26XX.oem3 (.text:PDMCC26XX_open)
                  0000398c    00000130     driverlib.lib : setup_rom.obj (.text:NOROM_SetupAfterColdResetWakeupFromShutDownCfg3)
                  00003abc    0000012c     drivers_cc13xxware.aem3 : PowerCC26XX.oem3 (.text:Power_init)
                  00003be8    0000011c                             : UARTCC26XX.oem3 (.text:UARTCC26XX_read)
                  00003d04    00000110                             : UARTCC26XX.oem3 (.text:UARTCC26XX_hwiIntFxn)
                  00003e14    00000104                             : PDMCC26XX_util.oem3 (.text:PDMCC26XX_I2S_startStream)
                  00003f18    000000fc                             : UARTCC26XX.oem3 (.text:UARTCC26XX_write)
                  00004014    000000f8     pdmstream_pem3.oem3 (.text:xdc_runtime_System_printfExtend__I)
                  0000410c    000000f0     driverlib.lib : setup_rom.obj (.text:NOROM_SetupAfterColdResetWakeupFromShutDownCfg2)
                  000041fc    000000e8     rom_sysbios.aem3 : rom_sysbios.obj (.text:ti_sysbios_knl_Event_pend__E)
                  000042e4    000000e0     drivers_cc13xxware.aem3 : PINCC26XX.oem3 (.text:PINCC26XX_setIoCfg)
                  000043c4    000000d8     driverlib.lib : i2s.obj (.text:NOROM_I2SChannelConfigure)
                  0000449c    000000d8     pdmstream.obj (.text:SA_envelopeDetector)
                  00004574    000000d4     power_cc13xx_tirtos.aem3 : PowerCC26XX_tirtos.oem3 (.text:PowerCC26XX_standbyPolicy)
                  00004648    000000d4     drivers_cc13xxware.aem3 : PowerCC26XX.oem3 (.text:Power_releaseDependency)
                  0000471c    000000d0                             : PowerCC26XX.oem3 (.text:Power_setDependency)
                  000047ec    000000ca                             : PDMCC26XX_util.oem3 (.text:PDMCC26XX_I2S_initIO)
                  000048b6    00000002     display.aem3 : DisplayUart.oem3 (.text:DisplayUart_clear)
                  000048b8    000000c8     drivers_cc13xxware.aem3 : UARTCC26XX.oem3 (.text:UARTCC26XX_initHw)
                  00004980    000000c4                             : PDMCC26XX_util.oem3 (.text:PDMCC26XX_I2S_hwiFxn)
                  00004a44    000000c0     driverlib.lib : setup.obj (.text:TrimAfterColdResetWakeupFromShutDown)
                  00004b04    000000b0     drivers_cc13xxware.aem3 : PDMCC26XX.oem3 (.text:PDMCC26XX_startStream)
                  00004bb4    000000ac                             : Codec1.oem3 (.text:Codec1_encodeSingle)
                  00004c60    000000a8     driverlib.lib : setup.obj (.text:NOROM_SetupTrimDevice)
                  00004d08    000000a4                   : setup_rom.obj (.text:NOROM_SetupAfterColdResetWakeupFromShutDownCfg1)
                  00004dac    000000a0     auto_init.aem3 : auto_init.oem3 (.text)
                  00004e4c    0000009e     rom_sysbios.aem3 : rom_sysbios.obj (.text:xdc_runtime_Text_putSite__E)
                  00004eea    00000002     display.aem3 : DisplayUart.oem3 (.text:DisplayUart_clearLines)
                  00004eec    0000009c     drivers_cc13xxware.aem3 : PDMCC26XX_util.oem3 (.text:PDMCC26XX_I2S_initHw)
                  00004f88    0000009c     rtsv7M3_T_le_eabi.lib : memcpy_t2.asm.obj (.text)
                  00005024    00000098     rom_sysbios.aem3 : rom_sysbios.obj (.text:ti_sysbios_knl_Clock_workFuncDynamic__E)
                  000050bc    00000096     rtsv7M3_T_le_eabi.lib : ull_div_t2.asm.obj (.text)
                  00005152    00000002                           : _lock.c.obj (.text:_nop)
                  00005154    00000094     drivers_cc13xxware.aem3 : PINCC26XX.oem3 (.text:PIN_open)
                  000051e8    00000094                             : UARTCC26XX.oem3 (.text:writeFinishedDoCallback)
                  0000527c    00000094     rom_sysbios.aem3 : rom_sysbios.obj (.text:xdc_runtime_Text_putMod__E)
                  00005310    00000090     drivers_cc13xxware.aem3 : PowerCC26XX.oem3 (.text:switchXOSCHFclockFunc)
                  000053a0    0000008c                             : UARTCC26XX.oem3 (.text:UARTCC26XX_initIO)
                  0000542c    0000008c                             : UARTCC26XX.oem3 (.text:UARTCC26XX_writeCancel)
                  000054b8    0000008c                             : PowerCC26XX.oem3 (.text:disableLFClockQualifiers)
                  00005544    00000088                             : PowerCC26XX_calibrateRCOSC.oem3 (.text:calibrateRcoscHf2)
                  000055cc    00000084                             : PDMCC26XX_util.oem3 (.text:PDMCC26XX_I2S_stopStream)
                  00005650    00000080     pdmstream.obj (.text:SA_PDMCC26XX_callbackFxn)
                  000056d0    0000007c     drivers_cc13xxware.aem3 : PDMCC26XX_util.oem3 (.text:PDMCC26XX_I2S_close)
                  0000574c    0000007a     rtsv7M3_T_le_eabi.lib : memset_t2.asm.obj (.text)
                  000057c6    00000002     drivers_cc13xxware.aem3 : PowerCC26XX.oem3 (.text:emptyClockFunc)
                  000057c8    00000078                             : Codec1.oem3 (.text:Codec1_encodeBuff)
                  00005840    00000078                             : UARTCC26XX.oem3 (.text:UARTCC26XX_close)
                  000058b8    00000074     driverlib.lib : setup_rom.obj (.text:NOROM_SetupSetVddrLevel)
                  0000592c    00000074     drivers_cc13xxware.aem3 : PowerCC26XX_calibrateRCOSC.oem3 (.text:PowerCC26XX_auxISR)
                  000059a0    00000074     rom_sysbios.aem3 : rom_sysbios.obj (.text:ti_sysbios_family_arm_cc26xx_Timer_start__E)
                  00005a14    00000074     drivers_cc13xxware.aem3 : UARTCC26XX.oem3 (.text:writeTxFifoFlush)
                  00005a88    00000070     driverlib.lib : chipinfo.obj (.text:NOROM_ChipInfo_GetHwRevision)
                  00005af8    00000070     rom_sysbios.aem3 : rom_sysbios.obj (.text:ti_sysbios_knl_Event_post__E)
                  00005b68    0000006d                      : rom_sysbios.obj (.text:xdc_runtime_System_formatNum__I)
                  00005bd5    00000001     --HOLE-- [fill = 0]
                  00005bd6    00000002     rtsv7M3_T_le_eabi.lib : div0.asm.obj (.text)
                  00005bd8    0000006c     driverlib.lib : setup_rom.obj (.text:NOROM_SetupGetTrimForAmpcompCtrl)
                  00005c44    0000006c     drivers_cc13xxware.aem3 : PowerCC26XX.oem3 (.text:PowerCC26XX_calibrate)
                  00005cb0    0000006c                             : UARTCC26XX.oem3 (.text:UARTCC26XX_readCancel)
                  00005d1c    00000068     driverlib.lib : setup_rom.obj (.text:NOROM_SetupGetTrimForAnabypassValue1)
                  00005d84    00000068                   : sys_ctrl.obj (.text:NOROM_SysCtrl_DCDC_VoltageConditionalControl)
                  00005dec    00000068     rtsv7M3_T_le_eabi.lib : copy_decompress_lzss.c.obj (.text:decompress:lzss:__TI_decompress_lzss)
                  00005e54    00000064     driverlib.lib : osc.obj (.text:NOROM_OSCHF_AttemptToSwitchToXosc)
                  00005eb8    00000064     drivers_cc13xxware.aem3 : PDMCC26XX.oem3 (.text:PDMCC26XX_init)
                  00005f1c    00000064                             : UARTCC26XX.oem3 (.text:UARTCC26XX_control)
                  00005f80    00000060     driverlib.lib : osc.obj (.text:NOROM_OSCClockSourceSet)
                  00005fe0    00000060     drivers_cc13xxware.aem3 : PowerCC26XX_calibrateRCOSC.oem3 (.text:PowerCC26XX_RCOSC_clockFunc)
                  00006040    00000060                             : PowerCC26XX_calibrateRCOSC.oem3 (.text:updateSubSecInc)
                  000060a0    0000005c     driverlib.lib : sys_ctrl.obj (.text:NOROM_SysCtrlAdjustRechargeAfterPowerDown)
                  000060fc    0000005c     drivers_cc13xxware.aem3 : PINCC26XX.oem3 (.text:PIN_remove)
                  00006158    0000005c     pdmstream_pem3.oem3 (.text:xdc_runtime_Startup_getState__I)
                  000061b4    0000005b     rom_sysbios.aem3 : rom_sysbios.obj (.text:xdc_runtime_Text_putLab__E)
                  0000620f    00000001     --HOLE-- [fill = 0]
                  00006210    00000058     display.aem3 : DisplayUart.oem3 (.text:DisplayUart_put5)
                  00006268    00000058     rtsv7M3_T_le_eabi.lib : hostwrite.c.obj (.text:HOSTwrite)
                  000062c0    00000058     drivers_cc13xxware.aem3 : PDMCC26XX.oem3 (.text:PDMCC26XX_rollbackDriverInitialisation)
                  00006318    00000058                             : PowerCC26XX_calibrateRCOSC.oem3 (.text:PowerCC26XX_initiateCalibration)
                  00006370    00000058     pdmstream.obj (.text:buttonCallbackFxn)
                  000063c8    00000054     drivers_cc13xxware.aem3 : PDMCC26XX.oem3 (.text:PDMCC26XX_stopStream)
                  0000641c    00000054                             : PowerCC26XX.oem3 (.text:configureXOSCHF)
                  00006470    00000050     driverlib.lib : setup_rom.obj (.text:NOROM_SetupSetCacheModeAccordingToCcfgSetting)
                  000064c0    00000050     drivers_cc13xxware.aem3 : PDMCC26XX_util.oem3 (.text:PDMCC26XX_I2S_requestBuffer)
                  00006510    0000004c     display.aem3 : DisplayUart.oem3 (.text:DisplayUart_open)
                  0000655c    0000004c     drivers_cc13xxware.aem3 : PDMCC26XX.oem3 (.text:PDMCC26XX_setPcmBufferReady)
                  000065a8    0000004c     rtsv7M3_T_le_eabi.lib : cpy_tbl.c.obj (.text:copy_in)
                  000065f4    0000004c     drivers_cc13xxware.aem3 : UARTCC26XX.oem3 (.text:startTxFifoEmptyClk)
                  00006640    00000048     display.aem3 : Display.oem3 (.text:Display_doOpen)
                  00006688    00000048     driverlib.lib : chipinfo.obj (.text:NOROM_ChipInfo_GetChipFamily)
                  000066d0    00000048     drivers_cc13xxware.aem3 : PINCC26XX.oem3 (.text:PIN_setOutputEnable)
                  00006718    00000048                             : PINCC26XX.oem3 (.text:PIN_swi)
                  00006760    00000048                             : PowerCC26XX.oem3 (.text:notify)
                  000067a8    00000046                             : RingBuf.oem3 (.text:RingBuf_put)
                  000067ee    00000002     rom_sysbios.aem3 : rom_sysbios.obj (.text:ti_sysbios_BIOS_linkedWithIncorrectBootLibrary__E)
                  000067f0    00000044     drivers_cc13xxware.aem3 : PDMCC26XX.oem3 (.text:PDMCC26XX_requestBuffer)
                  00006834    00000044     boot.aem3 : boot.oem3 (.text)
                  00006878    00000044     rom_sysbios.aem3 : rom_sysbios.obj (.text:xdc_runtime_SysMin_flush__E)
                  000068bc    00000044                      : rom_sysbios.obj (.text:xdc_runtime_Text_xprintf__I)
                  00006900    00000040     drivers_cc13xxware.aem3 : RingBuf.oem3 (.text:RingBuf_get)
                  00006940    00000040     rtsv7M3_T_le_eabi.lib : u_divt2.asm.obj (.text)
                  00006980    0000003c     driverlib.lib : osc.obj (.text:NOROM_OSC_HPOSCRelativeFrequencyOffsetGet)
                  000069bc    0000003c     drivers_cc13xxware.aem3 : PINCC26XX.oem3 (.text:PIN_setOutputValue)
                  000069f8    0000003c                             : UARTCC26XX.oem3 (.text:UARTCC26XX_swiIntFxn)
                  00006a34    00000038                             : PDMCC26XX.oem3 (.text:PDMCC26XX_initIO)
                  00006a6c    00000038                             : PINCC26XX.oem3 (.text:PIN_setInterrupt)
                  00006aa4    00000038     pdmstream.obj (.text:SA_audioMalloc)
                  00006adc    00000038     rtsv7M3_T_le_eabi.lib : trgmsg.c.obj (.text:__TI_writemsg)
                  00006b14    00000038     drivers_cc13xxware.aem3 : UARTCC26XX.oem3 (.text:readData)
                  00006b4c    00000038     rom_sysbios.aem3 : rom_sysbios.obj (.text:ti_sysbios_family_arm_cc26xx_Timer_getCurrentTick__E)
                  00006b84    00000038     drivers_cc13xxware.aem3 : UARTCC26XX.oem3 (.text:writeData)
                  00006bbc    00000038     rom_sysbios.aem3 : rom_sysbios.obj (.text:xdc_runtime_SysMin_putch__E)
                  00006bf4    00000034     driverlib.lib : osc.obj (.text:NOROM_OSCHF_SwitchToRcOscTurnOffXosc)
                  00006c28    00000034     drivers_cc13xxware.aem3 : PINCC26XX.oem3 (.text:PIN_setConfig)
                  00006c5c    00000034     rtsv7M3_T_le_eabi.lib : trgmsg.c.obj (.text:__TI_readmsg)
                  00006c90    00000034     drivers_cc13xxware.aem3 : UARTCC26XX.oem3 (.text:readData2RingBuf)
                  00006cc4    00000034     rom_sysbios.aem3 : rom_sysbios.obj (.text:ti_sysbios_family_arm_cc26xx_Timer_initDevice__I)
                  00006cf8    00000032     drivers_cc13xxware.aem3 : PDMCC26XX.oem3 (.text:PDMCC26XX_getNewPcmBuffer)
                  00006d2a    00000032     rom_sysbios.aem3 : rom_sysbios.obj (.text:ti_sysbios_family_arm_cc26xx_Timer_setNextTick__E)
                  00006d5c    00000030     driverlib.lib : i2s.obj (.text:NOROM_I2SSampleStampConfigure)
                  00006d8c    00000030                   : prcm.obj (.text:NOROM_PRCMAudioClockConfigSetOverride)
                  00006dbc    00000030                   : setup_rom.obj (.text:NOROM_SetupSetAonRtcSubSecInc)
                  00006dec    00000030     drivers_cc13xxware.aem3 : PDMCC26XX_util.oem3 (.text:PDMCC26XX_I2S_cleanUpQueues)
                  00006e1c    00000030                             : PowerCC26XX.oem3 (.text:Power_releaseConstraint)
                  00006e4c    00000030                             : PowerCC26XX.oem3 (.text:Power_setConstraint)
                  00006e7c    00000030                             : UART.oem3 (.text:UART_open)
                  00006eac    00000030     pdmstream_pem3.oem3 (.text:ti_sysbios_BIOS_atExitFunc__I)
                  00006edc    00000030     pdmstream_pem3.oem3 (.text:ti_sysbios_BIOS_startFunc__I)
                  00006f0c    00000030     rom_sysbios.aem3 : rom_sysbios.obj (.text:ti_sysbios_family_arm_cc26xx_Timer_setThreshold__I)
                  00006f3c    00000030                      : rom_sysbios.obj (.text:xdc_runtime_SysMin_abort__E)
                  00006f6c    0000002f                      : rom_sysbios.obj (.text:xdc_runtime_Text_printVisFxn__I)
                  00006f9b    00000001     --HOLE-- [fill = 0]
                  00006f9c    0000002c     driverlib.lib : ddi.obj (.text:NOROM_DDI32RegWrite)
                  00006fc8    0000002c                   : osc.obj (.text:NOROM_OSCClockSourceGet)
                  00006ff4    0000002c                   : setup_rom.obj (.text:NOROM_SetupGetTrimForRadcExtCfg)
                  00007020    0000002c     drivers_cc13xxware.aem3 : PINCC26XX.oem3 (.text:PINCC26XX_setMux)
                  0000704c    0000002c     rom_sysbios.aem3 : rom_sysbios.obj (.text:ti_sysbios_knl_Clock_getTicksUntilInterrupt__E)
                  00007078    0000002c     pdmstream_pem3.oem3 (.text:ti_sysbios_knl_Event_construct)
                  000070a4    0000002c     rom_sysbios.aem3 : rom_sysbios.obj (.text:ti_sysbios_knl_Event_pendTimeout__I)
                  000070d0    0000002a                      : rom_sysbios.obj (.text:xdc_runtime_System_putchar__I)
                  000070fa    00000002     pdmstream_pem3.oem3 (.text:ti_sysbios_BIOS_nullFunc__I)
                  000070fc    00000028     driverlib.lib : aon_batmon.obj (.text:NOROM_AONBatMonTemperatureGetDegC)
                  00007124    00000028                   : i2s.obj (.text:NOROM_I2SEnable)
                  0000714c    00000028     drivers_cc13xxware.aem3 : PowerCC26XX.oem3 (.text:Power_registerNotify)
                  00007174    00000028     driverlib.lib : adi.obj (.text:SafeHapiVoid)
                  0000719c    00000026     display.aem3 : Display.oem3 (.text:Display_doPut5)
                  000071c2    00000026     drivers_cc13xxware.aem3 : List.oem3 (.text:List_put)
                  000071e8    00000024                             : PINCC26XX.oem3 (.text:PINCC26XX_getPinCount)
                  0000720c    00000024     pdmstream.obj (.text:SA_audioFree)
                  00007230    00000024     drivers_cc13xxware.aem3 : PowerCC26XX_calibrateRCOSC.oem3 (.text:getTdcSemaphore)
                  00007254    00000024     pdmstream_pem3.oem3 (.text:ti_sysbios_BIOS_registerRTSLock__I)
                  00007278    00000024     pdmstream_pem3.oem3 (.text:ti_sysbios_BIOS_removeRTSLock__I)
                  0000729c    00000024     rom_sysbios.aem3 : rom_sysbios.obj (.text:ti_sysbios_family_arm_cc26xx_Timer_getMaxTicks__E)
                  000072c0    00000024                      : rom_sysbios.obj (.text:xdc_runtime_System_vprintf__E)
                  000072e4    00000022     pdmstream_pem3.oem3 (.text:xdc_runtime_SysMin_output__I)
                  00007306    00000002     rom_sysbios.aem3 : rom_sysbios.obj (.text:ti_sysbios_knl_Clock_triggerFunc__I)
                  00007308    00000020     driverlib.lib : i2s.obj (.text:NOROM_I2SAudioFormatConfigure)
                  00007328    00000020                   : setup_rom.obj (.text:NOROM_SetupGetTrimForXoscHfCtl)
                  00007348    00000020     drivers_cc13xxware.aem3 : PowerCC26XX.oem3 (.text:Power_unregisterNotify)
                  00007368    00000020     pdmstream_pem3.oem3 (.text:ti_sysbios_BIOS_rtsLock__I)
                  00007388    00000020     rom_sysbios.aem3 : rom_sysbios.obj (.text:ti_sysbios_family_arm_cc26xx_Timer_dynamicStub__E)
                  000073a8    00000020                      : rom_sysbios.obj (.text:ti_sysbios_knl_Clock_stop__E)
                  000073c8    00000020                      : rom_sysbios.obj (.text:ti_sysbios_knl_Event_checkEvents__I)
                  000073e8    00000020                      : rom_sysbios.obj (.text:xdc_runtime_Registry_findById__E)
                  00007408    00000020                      : rom_sysbios.obj (.text:xdc_runtime_SysMin_Module_startup__E)
                  00007428    0000001e     drivers_cc13xxware.aem3 : PINCC26XX.oem3 (.text:PIN_close)
                  00007446    0000001e                             : PowerCC26XX.oem3 (.text:Power_getTransitionLatency)
                  00007464    0000001c     driverlib.lib : setup_rom.obj (.text:NOROM_SetupGetTrimForAmpcompTh2)
                  00007480    0000001c                   : setup_rom.obj (.text:NOROM_SetupGetTrimForRcOscLfRtuneCtuneTrim)
                  0000749c    0000001c     drivers_cc13xxware.aem3 : PINCC26XX.oem3 (.text:PINCC26XX_setIoCfgMux)
                  000074b8    0000001c                             : PINCC26XX.oem3 (.text:PIN_hwi)
                  000074d4    0000001c     rom_sysbios.aem3 : rom_sysbios.obj (.text:ti_sysbios_family_arm_m3_Hwi_clearInterrupt__E)
                  000074f0    0000001c                      : rom_sysbios.obj (.text:xdc_runtime_SysMin_exit__E)
                  0000750c    0000001a     drivers_cc13xxware.aem3 : List.oem3 (.text:List_remove)
                  00007526    0000001a     rom_sysbios.aem3 : rom_sysbios_config.obj (.text:xdc_runtime_System_printf__E)
                  00007540    0000001a                      : rom_sysbios_config.obj (.text:xdc_runtime_System_snprintf__E)
                  0000755a    00000018     display.aem3 : DisplayUart.oem3 (.text:DisplayUart_close)
                  00007572    00000002     pdmstream_pem3.oem3 (.text:ti_sysbios_rom_cortexm_cc13xx_CC13xx_badRomRevision__E)
                  00007574    00000018     driverlib.lib : aon_rtc.obj (.text:NOROM_AONRTCCurrentCompareValueGet)
                  0000758c    00000018                   : chipinfo.obj (.text:NOROM_ChipInfo_GetPackageType)
                  000075a4    00000018                   : i2s.obj (.text:NOROM_I2SBufferConfig)
                  000075bc    00000018                   : osc.obj (.text:NOROM_OSCHF_TurnOnXosc)
                  000075d4    00000018                   : setup_rom.obj (.text:NOROM_SetupGetTrimForAdcShModeEn)
                  000075ec    00000018                   : setup_rom.obj (.text:NOROM_SetupGetTrimForAdcShVbufEn)
                  00007604    00000018                   : setup_rom.obj (.text:NOROM_SetupGetTrimForAmpcompTh1)
                  0000761c    00000018                   : setup_rom.obj (.text:NOROM_SetupGetTrimForDblrLoopFilterResetVoltage)
                  00007634    00000018                   : setup_rom.obj (.text:NOROM_SetupGetTrimForRcOscLfIBiasTrim)
                  0000764c    00000018                   : setup_rom.obj (.text:NOROM_SetupGetTrimForXoscLfRegulatorAndCmirrwrRatio)
                  00007664    00000018     drivers_cc13xxware.aem3 : PDMCC26XX_util.oem3 (.text:PDMCC26XX_I2S_init)
                  0000767c    00000018                             : PDMCC26XX.oem3 (.text:PDMCC26XX_i2sCallbackFxn)
                  00007694    00000018                             : PowerCC26XX.oem3 (.text:Power_idleFunc)
                  000076ac    00000018                             : UARTCC26XX.oem3 (.text:UARTCC26XX_init)
                  000076c4    00000018                             : UART.oem3 (.text:UART_Params_init)
                  000076dc    00000018     rtsv7M3_T_le_eabi.lib : args_main.c.obj (.text:_args_main)
                  000076f4    00000018     drivers_cc13xxware.aem3 : PowerCC26XX.oem3 (.text:configureRFCoreClocks)
                  0000770c    00000018     rtsv7M3_T_le_eabi.lib : ll_mul_t2.asm.obj (.text)
                  00007724    00000018     pdmstream_pem3.oem3 (.text:ti_sysbios_BIOS_rtsUnlock__I)
                  0000773c    00000018     rom_sysbios.aem3 : rom_sysbios.obj (.text:ti_sysbios_knl_Swi_or__E)
                  00007754    00000018     pdmstream_pem3.oem3 (.text:ti_sysbios_rom_cortexm_cc13xx_CC13xx_checkRevision__E)
                  0000776c    00000016     driverlib.lib : chipinfo.obj (.text:NOROM_ThisCodeIsBuiltForCC13xxHwRev20AndLater_HaltIfViolated)
                  00007782    00000016     pdmstream_pem3.oem3 (.text:ti_sysbios_BIOS_exitFunc__I)
                  00007798    00000016     pdmstream.obj (.text:ti_sysbios_knl_Semaphore_Params_init)
                  000077ae    00000016     pdmstream.obj (.text:ti_sysbios_knl_Task_Params_init)
                  000077c4    00000014     driverlib.lib : aon_rtc.obj (.text:NOROM_AONRTCCurrent64BitValueGet)
                  000077d8    00000014                   : i2s.obj (.text:NOROM_I2SPointerSet)
                  000077ec    00000014     drivers_cc13xxware.aem3 : PDMCC26XX_util.oem3 (.text:PDMCC26XX_I2S_releaseBuffer)
                  00007800    00000014                             : PINCC26XX.oem3 (.text:PINCC26XX_getInputValue)
                  00007814    00000014     rtsv7M3_T_le_eabi.lib : strlen.c.obj (.text:strlen)
                  00007828    00000014     pdmstream_pem3.oem3 (.text:ti_sysbios_knl_Clock_doTick__I)
                  0000783c    00000014     rom_sysbios.aem3 : rom_sysbios.obj (.text:ti_sysbios_knl_Event_Instance_init__E)
                  00007850    00000012     drivers_cc13xxware.aem3 : RingBuf.oem3 (.text:RingBuf_construct)
                  00007862    00000012     pdmstream_pem3.oem3 (.text:xdc_runtime_Startup_exec__I)
                  00007874    00000010     driverlib.lib : setup_rom.obj (.text:NOROM_SetupGetTrimForXoscHfFastStart)
                  00007884    00000010                   : setup_rom.obj (.text:NOROM_SetupGetTrimForXoscHfIbiastherm)
                  00007894    00000010     drivers_cc13xxware.aem3 : PDMCC26XX.oem3 (.text:PDMCC26XX_close)
                  000078a4    00000010                             : UARTCC26XX.oem3 (.text:uartPostNotify)
                  000078b4    00000010     rom_sysbios.aem3 : rom_sysbios.obj (.text:xdc_runtime_SysMin_ready__E)
                  000078c4    00000010                      : rom_sysbios.obj (.text:xdc_runtime_System_vsnprintf__E)
                  000078d4    0000000e     driverlib.lib : vims.obj (.text:NOROM_VIMSModeGet)
                  000078e2    0000000e     rtsv7M3_T_le_eabi.lib : copy_decompress_none.c.obj (.text:decompress:none:__TI_decompress_none)
                  000078f0    0000000e     rom_sysbios.aem3 : rom_sysbios.obj (.text:ti_sysbios_family_arm_cc26xx_TimestampProvider_get32__E)
                  000078fe    0000000c     display.aem3 : Display.oem3 (.text:Display_doClear)
                  0000790a    0000000c     driverlib.lib : cpu.obj (.text:NOROM_CPUcpsid)
                  00007916    0000000c                   : cpu.obj (.text:NOROM_CPUcpsie)
                  00007922    0000000c     drivers_cc13xxware.aem3 : PINCC26XX.oem3 (.text:PIN_registerIntCb)
                  0000792e    00000002     rom_sysbios.aem3 : rom_sysbios.obj (.text:xdc_runtime_SysCallback_defaultAbort)
                  00007930    0000000c     drivers_cc13xxware.aem3 : PowerCC26XX.oem3 (.text:Power_getConstraintMask)
                  0000793c    0000000c                             : PowerCC26XX.oem3 (.text:Power_getDependencyCount)
                  00007948    0000000c     rtsv7M3_T_le_eabi.lib : _lock.c.obj (.text:_register_lock)
                  00007954    0000000c                           : _lock.c.obj (.text:_register_unlock)
                  00007960    0000000c                           : copy_zero_init.c.obj (.text:decompress:ZI:__TI_zero_init)
                  0000796c    0000000c     pdmstream_pem3.oem3 (.text:ti_sysbios_knl_Event_Params__init__S)
                  00007978    0000000c     pdmstream.obj (.text:ti_sysbios_knl_Semaphore_handle)
                  00007984    0000000c     rom_sysbios.aem3 : rom_sysbios.obj (.text:ti_sysbios_knl_Swi_getTrigger__E)
                  00007990    0000000c     pdmstream_pem3.oem3 (.text:xdc_runtime_Startup_reset__I)
                  0000799c    0000000c     rom_sysbios.aem3 : rom_sysbios.obj (.text:xdc_runtime_Startup_rtsDone__E)
                  000079a8    0000000a     drivers_cc13xxware.aem3 : List.oem3 (.text:List_empty)
                  000079b2    0000000a                             : UART.oem3 (.text:UART_close)
                  000079bc    0000000a                             : UART.oem3 (.text:UART_write)
                  000079c6    00000008                             : PDMCC26XX_util.oem3 (.text:PDMCC26XX_I2S_callback)
                  000079ce    00000008                             : UARTCC26XX.oem3 (.text:readSemCallback)
                  000079d6    00000008                             : UARTCC26XX.oem3 (.text:writeSemCallback)
                  000079de    00000008     pdmstream_pem3.oem3 (.text:xdc_runtime_Text_visitRope__I)
                  000079e6    00000006     display.aem3 : DisplayUart.oem3 (.text:DisplayUart_control)
                  000079ec    00000006                  : DisplayUart.oem3 (.text:DisplayUart_getType)
                  000079f2    00000006                  : Display.oem3 (.text:Display_doParamsInit)
                  000079f8    00000006     drivers_cc13xxware.aem3 : UARTCC26XX.oem3 (.text:UARTCC26XX_readPolling)
                  000079fe    00000006                             : UARTCC26XX.oem3 (.text:UARTCC26XX_writePolling)
                  00007a04    00000004     tirtosport.aem3 : HwiP_tirtos.oem3 (.text:HwiP_disable)
                  00007a08    00000004     drivers_cc13xxware.aem3 : List.oem3 (.text:List_head)
                  00007a0c    00000004                             : List.oem3 (.text:List_next)
                  00007a10    00000004                             : PowerCC26XX.oem3 (.text:nopResourceHandler)
                  00007a14    00000004     rom_sysbios.aem3 : rom_sysbios.obj (.text:ti_sysbios_family_arm_cc26xx_Timer_getCount64__E)
                  00007a18    00000004                      : rom_sysbios.obj (.text:ti_sysbios_knl_Semaphore_getCount__E)
                  00007a1c    00000004                      : rom_sysbios.obj (.text:xdc_runtime_System_printf_va__F)
                  00007a20    00000004                      : rom_sysbios.obj (.text:xdc_runtime_System_snprintf_va__F)
                  00007a24    00000002                      : rom_sysbios.obj (.text:xdc_runtime_SysCallback_defaultExit)
                  00007a26    00000002     --HOLE-- [fill = 0]
                  00007a28    00000008     (.tramp.xdc_runtime_Core_assignParams__I.1)
                  00007a30    00000008     (.tramp.xdc_runtime_Startup_startMods__I.1)
                  00007a38    00000008     (.tramp.ti_sysbios_knl_Clock_logTick__E.1)
                  00007a40    00000008     (.tramp.ti_sysbios_BIOS_RtsGateProxy_leave__E.1)
                  00007a48    00000008     (.tramp.ti_sysbios_BIOS_RtsGateProxy_enter__E.1)
                  00007a50    00000008     (.tramp.xdc_runtime_Memory_free__E.1)
                  00007a58    00000008     (.tramp.xdc_runtime_Core_constructObject__I.1)
                  00007a60    00000008     (.tramp.ti_sysbios_knl_Task_startup__E.1)
                  00007a68    00000008     (.tramp.ti_sysbios_knl_Swi_startup__E.1)
                  00007a70    00000008     (.tramp.ti_sysbios_hal_Hwi_startup__E.1)
                  00007a78    00000008     (.tramp.ti_sysbios_family_arm_cc26xx_Timer_startup__E.1)
                  00007a80    00000008     (.tramp.xdc_runtime_System_atexit__E.1)
                  00007a88    00000008     (.tramp.ti_sysbios_BIOS_setThreadType__E.1)
                  00007a90    00000008     (.tramp.xdc_runtime_Memory_alloc__E.1)
                  00007a98    00000008     (.tramp.xdc_runtime_Error_init__E.1)
                  00007aa0    00000008     (.tramp.xdc_runtime_Gate_leaveSystem__E.1)
                  00007aa8    00000008     (.tramp.xdc_runtime_Gate_enterSystem__E.1)
                  00007ab0    00000008     (.tramp.xdc_runtime_System_exit__E.1)
                  00007ab8    00000008     (.tramp.ti_sysbios_knl_Task_Params__init__S.1)
                  00007ac0    00000008     (.tramp.ti_sysbios_knl_Task_unblockI__E.1)
                  00007ac8    00000008     (.tramp.ti_sysbios_knl_Queue_remove__E.1)
                  00007ad0    00000008     (.tramp.ti_sysbios_knl_Queue_head__E.1)
                  00007ad8    00000008     (.tramp.ti_sysbios_knl_Clock_destruct.1)
                  00007ae0    00000008     (.tramp.ti_sysbios_knl_Swi_destruct.1)
                  00007ae8    00000008     (.tramp.ti_sysbios_knl_Semaphore_destruct.1)
                  00007af0    00000008     (.tramp.ti_sysbios_family_arm_m3_Hwi_destruct.1)
                  00007af8    00000008     (.tramp.ti_sysbios_family_arm_m3_Hwi_disableInterrupt__E.1)
                  00007b00    00000008     (.tramp.ti_sysbios_knl_Clock_scheduleNextTick__E.1)
                  00007b08    00000008     (.tramp.ti_sysbios_knl_Clock_walkQueueDynamic__E.1)
                  00007b10    00000008     (.tramp.ti_sysbios_knl_Clock_TimerProxy_getCurrentTick__E.1)
                  00007b18    00000008     (.tramp.ti_sysbios_knl_Semaphore_post__E.1)
                  00007b20    00000008     (.tramp.ti_sysbios_knl_Queue_get__E.1)
                  00007b28    00000008     (.tramp.ti_sysbios_knl_Queue_put__E.1)
                  00007b30    00000008     (.tramp.ti_sysbios_BIOS_getCpuFreq__E.1)
                  00007b38    00000008     (.tramp.ti_sysbios_knl_Clock_removeI__E.1)
                  00007b40    00000008     (.tramp.ti_sysbios_knl_Clock_startI__E.1)
                  00007b48    00000008     (.tramp.ti_sysbios_knl_Task_blockI__E.1)
                  00007b50    00000008     (.tramp.ti_sysbios_knl_Task_self__E.1)
                  00007b58    00000008     (.tramp.ti_sysbios_knl_Clock_addI__E.1)
                  00007b60    00000008     (.tramp.ti_sysbios_family_arm_m3_Hwi_enableInterrupt__E.1)
                  00007b68    00000008     (.tramp.ti_sysbios_knl_Swi_post__E.1)
                  00007b70    00000008     (.tramp.ti_sysbios_knl_Clock_setTimeout__E.1)
                  00007b78    00000008     (.tramp.ti_sysbios_knl_Clock_construct.1)
                  00007b80    00000008     (.tramp.ti_sysbios_knl_Clock_Params__init__S.1)
                  00007b88    00000008     (.tramp.ti_sysbios_knl_Clock_start__E.1)
                  00007b90    00000008     (.tramp.xdc_runtime_System_abortSpin__E.1)
                  00007b98    00000008     (.tramp.ti_sysbios_knl_Queue_enqueue__E.1)
                  00007ba0    00000008     (.tramp.ti_sysbios_knl_Queue_construct.1)
                  00007ba8    00000008     (.tramp.ti_sysbios_family_arm_m3_Hwi_restoreFxn__E.1)
                  00007bb0    00000008     (.tramp.ti_sysbios_family_arm_m3_Hwi_disableFxn__E.1)
                  00007bb8    00000008     (.tramp.ti_sysbios_knl_Swi_construct.1)
                  00007bc0    00000008     (.tramp.ti_sysbios_knl_Swi_Params__init__S.1)
                  00007bc8    00000008     (.tramp.ti_sysbios_family_arm_m3_Hwi_construct.1)
                  00007bd0    00000008     (.tramp.ti_sysbios_family_arm_m3_Hwi_Params__init__S.1)
                  00007bd8    00000008     (.tramp.ti_sysbios_knl_Semaphore_Params__init__S.1)
                  00007be0    00000008     (.tramp.ti_sysbios_knl_Task_restore__E.1)
                  00007be8    00000008     (.tramp.ti_sysbios_knl_Swi_restore__E.1)
                  00007bf0    00000008     (.tramp.ti_sysbios_knl_Swi_disable__E.1)
                  00007bf8    00000008     (.tramp.ti_sysbios_knl_Task_disable__E.1)
                  00007c00    00000008     (.tramp.ti_sysbios_BIOS_start__E.1)
                  00007c08    00000008     (.tramp.ti_sysbios_knl_Semaphore_construct.1)
                  00007c10    00000008     (.tramp.ti_sysbios_knl_Task_construct.1)
                  00007c18    00000008     (.tramp.xdc_runtime_System_abort__E.1)
                  00007c20    00000008     (.tramp.ti_sysbios_knl_Task_sleep__E.1)
                  00007c28    00000008     (.tramp.ti_sysbios_knl_Semaphore_pend__E.1)
                  00007c30    00000008     (.tramp.ti_sysbios_knl_Queue_destruct.1)
                  00007c38    00000008     (.tramp.ti_sysbios_knl_Queue_empty__E.1)
                  00007c40    00000008     (.tramp.ti_sysbios_knl_Queue_dequeue__E.1)

.binit     0    00000000    00000000     

.cinit     0    00000488    000002a0     
                  00000488    00000165     (.cinit..data.load) [load image, compression = lzss]
                  000005ed    00000028     (.cinit..data:ti_sysbios_family_arm_m3_Hwi_Module__state__V.load) [load image, compression = lzss]
                  00000615    00000021     (.cinit..data:ti_sysbios_knl_Task_Module__state__V.load) [load image, compression = lzss]
                  00000636    0000001f     (.cinit..data:ti_sysbios_BIOS_Module__state__V.load) [load image, compression = lzss]
                  00000655    0000001d     (.cinit..data:ti_sysbios_knl_Clock_Module__state__V.load) [load image, compression = lzss]
                  00000672    00000010     (.cinit..data:ti_sysbios_knl_Swi_Module__state__V.load) [load image, compression = lzss]
                  00000682    00000002     --HOLE-- [fill = 0]
                  00000684    0000000c     (__TI_handler_table)
                  00000690    0000000b     (.cinit..data:ti_sysbios_family_arm_cc26xx_Timer_Module__state__V.load) [load image, compression = lzss]
                  0000069b    0000000b     (.cinit..data:xdc_runtime_System_Module__state__V.load) [load image, compression = lzss]
                  000006a6    00000002     --HOLE-- [fill = 0]
                  000006a8    00000008     (.cinit..bss.load) [load image, compression = zero_init]
                  000006b0    00000008     (.cinit..data:xdc_runtime_Memory_Module__state__V.load) [load image, compression = lzss]
                  000006b8    00000007     (.cinit..data:ti_sysbios_family_arm_cc26xx_TimestampProvider_Module__state__V.load) [load image, compression = lzss]
                  000006bf    00000007     (.cinit..data:xdc_runtime_Startup_Module__state__V.load) [load image, compression = lzss]
                  000006c6    00000002     --HOLE-- [fill = 0]
                  000006c8    00000060     (__TI_cinit_table)

.init_array 
*          0    00000000    00000000     UNINITIALIZED

.ccfg      0    0001ffa8    00000058     
                  0001ffa8    00000058     ccfg.obj (.ccfg:retain)

.const:ti_sysbios_knl_Task_Object__PARAMS__C 
*          0    00001000    0000003c     
                  00001000    0000003c     pdmstream_pem3.oem3 (.const:ti_sysbios_knl_Task_Object__PARAMS__C)

.const:ti_sysbios_knl_Mailbox_Object__PARAMS__C 
*          0    0000103c    00000034     
                  0000103c    00000034     pdmstream_pem3.oem3 (.const:ti_sysbios_knl_Mailbox_Object__PARAMS__C)

.const:ti_sysbios_family_arm_m3_Hwi_Object__PARAMS__C 
*          0    00001070    00000030     
                  00001070    00000030     pdmstream_pem3.oem3 (.const:ti_sysbios_family_arm_m3_Hwi_Object__PARAMS__C)

.const:ti_sysbios_hal_Hwi_Object__PARAMS__C 
*          0    000010a0    0000002c     
                  000010a0    0000002c     pdmstream_pem3.oem3 (.const:ti_sysbios_hal_Hwi_Object__PARAMS__C)

.const:ti_sysbios_heaps_HeapMem_Module__FXNS__C 
*          0    000010cc    00000028     
                  000010cc    00000028     pdmstream_pem3.oem3 (.const:ti_sysbios_heaps_HeapMem_Module__FXNS__C)

.const:ti_sysbios_knl_Swi_Object__PARAMS__C 
*          0    000010f4    00000028     
                  000010f4    00000028     pdmstream_pem3.oem3 (.const:ti_sysbios_knl_Swi_Object__PARAMS__C)

.const:ti_sysbios_gates_GateHwi_Module__FXNS__C 
*          0    0000111c    00000024     
                  0000111c    00000024     pdmstream_pem3.oem3 (.const:ti_sysbios_gates_GateHwi_Module__FXNS__C)

.const:ti_sysbios_gates_GateMutex_Module__FXNS__C 
*          0    00001140    00000024     
                  00001140    00000024     pdmstream_pem3.oem3 (.const:ti_sysbios_gates_GateMutex_Module__FXNS__C)

.const:ti_sysbios_heaps_HeapMem_Object__PARAMS__C 
*          0    00001164    00000024     
                  00001164    00000024     pdmstream_pem3.oem3 (.const:ti_sysbios_heaps_HeapMem_Object__PARAMS__C)

.const:ti_sysbios_knl_Clock_Object__PARAMS__C 
*          0    00001188    00000024     
                  00001188    00000024     pdmstream_pem3.oem3 (.const:ti_sysbios_knl_Clock_Object__PARAMS__C)

.const:ti_sysbios_knl_Semaphore_Object__PARAMS__C 
*          0    000011ac    00000024     
                  000011ac    00000024     pdmstream_pem3.oem3 (.const:ti_sysbios_knl_Semaphore_Object__PARAMS__C)

.const:ti_sysbios_family_arm_m3_Hwi_Object__DESC__C 
*          0    000011d0    00000020     
                  000011d0    00000020     pdmstream_pem3.oem3 (.const:ti_sysbios_family_arm_m3_Hwi_Object__DESC__C)

.const:ti_sysbios_gates_GateHwi_Object__DESC__C 
*          0    000011f0    00000020     
                  000011f0    00000020     pdmstream_pem3.oem3 (.const:ti_sysbios_gates_GateHwi_Object__DESC__C)

.const:ti_sysbios_gates_GateMutex_Object__DESC__C 
*          0    00001210    00000020     
                  00001210    00000020     pdmstream_pem3.oem3 (.const:ti_sysbios_gates_GateMutex_Object__DESC__C)

.const:ti_sysbios_hal_Hwi_Object__DESC__C 
*          0    00001230    00000020     
                  00001230    00000020     pdmstream_pem3.oem3 (.const:ti_sysbios_hal_Hwi_Object__DESC__C)

.const:ti_sysbios_heaps_HeapMem_Object__DESC__C 
*          0    00001250    00000020     
                  00001250    00000020     pdmstream_pem3.oem3 (.const:ti_sysbios_heaps_HeapMem_Object__DESC__C)

.const:ti_sysbios_knl_Clock_Object__DESC__C 
*          0    00001270    00000020     
                  00001270    00000020     pdmstream_pem3.oem3 (.const:ti_sysbios_knl_Clock_Object__DESC__C)

.const:ti_sysbios_knl_Mailbox_Object__DESC__C 
*          0    00001290    00000020     
                  00001290    00000020     pdmstream_pem3.oem3 (.const:ti_sysbios_knl_Mailbox_Object__DESC__C)

.const:ti_sysbios_knl_Queue_Object__DESC__C 
*          0    000012b0    00000020     
                  000012b0    00000020     pdmstream_pem3.oem3 (.const:ti_sysbios_knl_Queue_Object__DESC__C)

.const:ti_sysbios_knl_Semaphore_Object__DESC__C 
*          0    000012d0    00000020     
                  000012d0    00000020     pdmstream_pem3.oem3 (.const:ti_sysbios_knl_Semaphore_Object__DESC__C)

.const:ti_sysbios_knl_Swi_Object__DESC__C 
*          0    000012f0    00000020     
                  000012f0    00000020     pdmstream_pem3.oem3 (.const:ti_sysbios_knl_Swi_Object__DESC__C)

.const:ti_sysbios_knl_Task_Object__DESC__C 
*          0    00001310    00000020     
                  00001310    00000020     pdmstream_pem3.oem3 (.const:ti_sysbios_knl_Task_Object__DESC__C)

.const:ti_sysbios_gates_GateHwi_Object__PARAMS__C 
*          0    00001330    00000018     
                  00001330    00000018     pdmstream_pem3.oem3 (.const:ti_sysbios_gates_GateHwi_Object__PARAMS__C)

.const:ti_sysbios_gates_GateMutex_Object__PARAMS__C 
*          0    00001348    00000018     
                  00001348    00000018     pdmstream_pem3.oem3 (.const:ti_sysbios_gates_GateMutex_Object__PARAMS__C)

.const:ti_sysbios_knl_Queue_Object__PARAMS__C 
*          0    00001360    00000018     
                  00001360    00000018     pdmstream_pem3.oem3 (.const:ti_sysbios_knl_Queue_Object__PARAMS__C)

.const:ti_sysbios_knl_Idle_funcList__C 
*          0    00001378    00000008     
                  00001378    00000008     pdmstream_pem3.oem3 (.const:ti_sysbios_knl_Idle_funcList__C)

.const:ti_sysbios_family_arm_cc26xx_Timer_startupNeeded__C 
*          0    00001384    00000004     
                  00001384    00000004     pdmstream_pem3.oem3 (.const:ti_sysbios_family_arm_cc26xx_Timer_startupNeeded__C)

.const:ti_sysbios_family_arm_m3_Hwi_E_alreadyDefined__C 
*          0    00001388    00000004     
                  00001388    00000004     pdmstream_pem3.oem3 (.const:ti_sysbios_family_arm_m3_Hwi_E_alreadyDefined__C)

.const:ti_sysbios_family_arm_m3_Hwi_E_hwiLimitExceeded__C 
*          0    0000138c    00000004     
                  0000138c    00000004     pdmstream_pem3.oem3 (.const:ti_sysbios_family_arm_m3_Hwi_E_hwiLimitExceeded__C)

.const:ti_sysbios_family_arm_m3_Hwi_NUM_INTERRUPTS__C 
*          0    00001390    00000004     
                  00001390    00000004     pdmstream_pem3.oem3 (.const:ti_sysbios_family_arm_m3_Hwi_NUM_INTERRUPTS__C)

.const:ti_sysbios_family_arm_m3_Hwi_Object__count__C 
*          0    00001394    00000004     
                  00001394    00000004     pdmstream_pem3.oem3 (.const:ti_sysbios_family_arm_m3_Hwi_Object__count__C)

.const:ti_sysbios_family_arm_m3_Hwi_Object__table__C 
*          0    00001398    00000004     
                  00001398    00000004     pdmstream_pem3.oem3 (.const:ti_sysbios_family_arm_m3_Hwi_Object__table__C)

.const:ti_sysbios_family_arm_m3_Hwi_ccr__C 
*          0    0000139c    00000004     
                  0000139c    00000004     pdmstream_pem3.oem3 (.const:ti_sysbios_family_arm_m3_Hwi_ccr__C)

.const:ti_sysbios_family_arm_m3_Hwi_excHandlerFunc__C 
*          0    000013a0    00000004     
                  000013a0    00000004     pdmstream_pem3.oem3 (.const:ti_sysbios_family_arm_m3_Hwi_excHandlerFunc__C)

.const:ti_sysbios_family_arm_m3_Hwi_nullIsrFunc__C 
*          0    000013a4    00000004     
                  000013a4    00000004     pdmstream_pem3.oem3 (.const:ti_sysbios_family_arm_m3_Hwi_nullIsrFunc__C)

.const:ti_sysbios_family_arm_m3_Hwi_numSparseInterrupts__C 
*          0    000013a8    00000004     
                  000013a8    00000004     pdmstream_pem3.oem3 (.const:ti_sysbios_family_arm_m3_Hwi_numSparseInterrupts__C)

.const:ti_sysbios_family_arm_m3_Hwi_priGroup__C 
*          0    000013ac    00000004     
                  000013ac    00000004     pdmstream_pem3.oem3 (.const:ti_sysbios_family_arm_m3_Hwi_priGroup__C)

.const:ti_sysbios_family_arm_m3_TaskSupport_stackAlignment__C 
*          0    000013b0    00000004     
                  000013b0    00000004     pdmstream_pem3.oem3 (.const:ti_sysbios_family_arm_m3_TaskSupport_stackAlignment__C)

.const:ti_sysbios_heaps_HeapMem_E_memory__C 
*          0    000013b4    00000004     
                  000013b4    00000004     pdmstream_pem3.oem3 (.const:ti_sysbios_heaps_HeapMem_E_memory__C)

.const:ti_sysbios_heaps_HeapMem_Module__gateObj__C 
*          0    000013b8    00000004     
                  000013b8    00000004     pdmstream_pem3.oem3 (.const:ti_sysbios_heaps_HeapMem_Module__gateObj__C)

.const:ti_sysbios_heaps_HeapMem_Object__count__C 
*          0    000013bc    00000004     
                  000013bc    00000004     pdmstream_pem3.oem3 (.const:ti_sysbios_heaps_HeapMem_Object__count__C)

.const:ti_sysbios_heaps_HeapMem_Object__table__C 
*          0    000013c0    00000004     
                  000013c0    00000004     pdmstream_pem3.oem3 (.const:ti_sysbios_heaps_HeapMem_Object__table__C)

.const:ti_sysbios_heaps_HeapMem_reqAlign__C 
*          0    000013c4    00000004     
                  000013c4    00000004     pdmstream_pem3.oem3 (.const:ti_sysbios_heaps_HeapMem_reqAlign__C)

.const:ti_sysbios_knl_Clock_serviceMargin__C 
*          0    000013c8    00000004     
                  000013c8    00000004     pdmstream_pem3.oem3 (.const:ti_sysbios_knl_Clock_serviceMargin__C)

.const:ti_sysbios_knl_Mailbox_Object__count__C 
*          0    000013cc    00000004     
                  000013cc    00000004     pdmstream_pem3.oem3 (.const:ti_sysbios_knl_Mailbox_Object__count__C)

.const:ti_sysbios_knl_Mailbox_Object__table__C 
*          0    000013d0    00000004     
                  000013d0    00000004     pdmstream_pem3.oem3 (.const:ti_sysbios_knl_Mailbox_Object__table__C)

.const:ti_sysbios_knl_Mailbox_maxTypeAlign__C 
*          0    000013d4    00000004     
                  000013d4    00000004     pdmstream_pem3.oem3 (.const:ti_sysbios_knl_Mailbox_maxTypeAlign__C)

.const:ti_sysbios_knl_Queue_Object__count__C 
*          0    000013d8    00000004     
                  000013d8    00000004     pdmstream_pem3.oem3 (.const:ti_sysbios_knl_Queue_Object__count__C)

.const:ti_sysbios_knl_Queue_Object__table__C 
*          0    000013dc    00000004     
                  000013dc    00000004     pdmstream_pem3.oem3 (.const:ti_sysbios_knl_Queue_Object__table__C)

.const:ti_sysbios_knl_Swi_Object__count__C 
*          0    000013e0    00000004     
                  000013e0    00000004     pdmstream_pem3.oem3 (.const:ti_sysbios_knl_Swi_Object__count__C)

.const:ti_sysbios_knl_Swi_Object__table__C 
*          0    000013e4    00000004     
                  000013e4    00000004     pdmstream_pem3.oem3 (.const:ti_sysbios_knl_Swi_Object__table__C)

.const:ti_sysbios_knl_Swi_numPriorities__C 
*          0    000013e8    00000004     
                  000013e8    00000004     pdmstream_pem3.oem3 (.const:ti_sysbios_knl_Swi_numPriorities__C)

.const:ti_sysbios_knl_Task_Object__count__C 
*          0    000013ec    00000004     
                  000013ec    00000004     pdmstream_pem3.oem3 (.const:ti_sysbios_knl_Task_Object__count__C)

.const:ti_sysbios_knl_Task_Object__table__C 
*          0    000013f0    00000004     
                  000013f0    00000004     pdmstream_pem3.oem3 (.const:ti_sysbios_knl_Task_Object__table__C)

.const:ti_sysbios_knl_Task_allBlockedFunc__C 
*          0    000013f4    00000004     
                  000013f4    00000004     pdmstream_pem3.oem3 (.const:ti_sysbios_knl_Task_allBlockedFunc__C)

.const:ti_sysbios_knl_Task_defaultStackHeap__C 
*          0    000013f8    00000004     
                  000013f8    00000004     pdmstream_pem3.oem3 (.const:ti_sysbios_knl_Task_defaultStackHeap__C)

.const:ti_sysbios_knl_Task_defaultStackSize__C 
*          0    000013fc    00000004     
                  000013fc    00000004     pdmstream_pem3.oem3 (.const:ti_sysbios_knl_Task_defaultStackSize__C)

.const:ti_sysbios_knl_Task_numConstructedTasks__C 
*          0    00001400    00000004     
                  00001400    00000004     pdmstream_pem3.oem3 (.const:ti_sysbios_knl_Task_numConstructedTasks__C)

.const:ti_sysbios_family_arm_cc26xx_Timer_Module__id__C 
*          0    00001406    00000002     
                  00001406    00000002     pdmstream_pem3.oem3 (.const:ti_sysbios_family_arm_cc26xx_Timer_Module__id__C)

.const:ti_sysbios_family_arm_cc26xx_TimestampProvider_useClockTimer__C 
*          0    00001408    00000002     
                  00001408    00000002     pdmstream_pem3.oem3 (.const:ti_sysbios_family_arm_cc26xx_TimestampProvider_useClockTimer__C)

.const:ti_sysbios_family_arm_m3_Hwi_Module__id__C 
*          0    0000140a    00000002     
                  0000140a    00000002     pdmstream_pem3.oem3 (.const:ti_sysbios_family_arm_m3_Hwi_Module__id__C)

.const:ti_sysbios_gates_GateHwi_Module__id__C 
*          0    0000140c    00000002     
                  0000140c    00000002     pdmstream_pem3.oem3 (.const:ti_sysbios_gates_GateHwi_Module__id__C)

.const:ti_sysbios_gates_GateMutex_Module__id__C 
*          0    0000140e    00000002     
                  0000140e    00000002     pdmstream_pem3.oem3 (.const:ti_sysbios_gates_GateMutex_Module__id__C)

.const:ti_sysbios_heaps_HeapMem_Module__id__C 
*          0    00001410    00000002     
                  00001410    00000002     pdmstream_pem3.oem3 (.const:ti_sysbios_heaps_HeapMem_Module__id__C)

.const:ti_sysbios_knl_Task_initStackFlag__C 
*          0    00001412    00000002     
                  00001412    00000002     pdmstream_pem3.oem3 (.const:ti_sysbios_knl_Task_initStackFlag__C)

.const:ti_sysbios_knl_Clock_tickMode__C 
*          0    00001414    00000001     
                  00001414    00000001     pdmstream_pem3.oem3 (.const:ti_sysbios_knl_Clock_tickMode__C)

.const:xdc_runtime_Startup_firstFxns__C 
*          0    00001418    00000008     
                  00001418    00000008     pdmstream_pem3.oem3 (.const:xdc_runtime_Startup_firstFxns__C)

.const:xdc_runtime_Startup_lastFxns__C 
*          0    00001420    00000008     
                  00001420    00000008     pdmstream_pem3.oem3 (.const:xdc_runtime_Startup_lastFxns__C)

.const:xdc_runtime_Assert_E_assertFailed__C 
*          0    00001428    00000004     
                  00001428    00000004     pdmstream_pem3.oem3 (.const:xdc_runtime_Assert_E_assertFailed__C)

.const:xdc_runtime_Error_E_memory__C 
*          0    0000142c    00000004     
                  0000142c    00000004     pdmstream_pem3.oem3 (.const:xdc_runtime_Error_E_memory__C)

.const:xdc_runtime_Error_policyFxn__C 
*          0    00001430    00000004     
                  00001430    00000004     pdmstream_pem3.oem3 (.const:xdc_runtime_Error_policyFxn__C)

.const:xdc_runtime_IGateProvider_Interface__BASE__C 
*          0    00001434    00000004     
                  00001434    00000004     pdmstream_pem3.oem3 (.const:xdc_runtime_IGateProvider_Interface__BASE__C)

.const:xdc_runtime_IHeap_Interface__BASE__C 
*          0    00001438    00000004     
                  00001438    00000004     pdmstream_pem3.oem3 (.const:xdc_runtime_IHeap_Interface__BASE__C)

.const:xdc_runtime_IModule_Interface__BASE__C 
*          0    0000143c    00000004     
                  0000143c    00000004     pdmstream_pem3.oem3 (.const:xdc_runtime_IModule_Interface__BASE__C)

.const:xdc_runtime_Main_Module__diagsEnabled__C 
*          0    00001440    00000004     
                  00001440    00000004     pdmstream_pem3.oem3 (.const:xdc_runtime_Main_Module__diagsEnabled__C)

.const:xdc_runtime_Main_Module__diagsIncluded__C 
*          0    00001444    00000004     
                  00001444    00000004     pdmstream_pem3.oem3 (.const:xdc_runtime_Main_Module__diagsIncluded__C)

.const:xdc_runtime_Main_Module__diagsMask__C 
*          0    00001448    00000004     
                  00001448    00000004     pdmstream_pem3.oem3 (.const:xdc_runtime_Main_Module__diagsMask__C)

.const:xdc_runtime_Memory_defaultHeapInstance__C 
*          0    0000144c    00000004     
                  0000144c    00000004     pdmstream_pem3.oem3 (.const:xdc_runtime_Memory_defaultHeapInstance__C)

.const:xdc_runtime_Startup_execImpl__C 
*          0    00001450    00000004     
                  00001450    00000004     pdmstream_pem3.oem3 (.const:xdc_runtime_Startup_execImpl__C)

.const:xdc_runtime_Startup_maxPasses__C 
*          0    00001454    00000004     
                  00001454    00000004     pdmstream_pem3.oem3 (.const:xdc_runtime_Startup_maxPasses__C)

.const:xdc_runtime_Startup_sfxnRts__C 
*          0    00001458    00000004     
                  00001458    00000004     pdmstream_pem3.oem3 (.const:xdc_runtime_Startup_sfxnRts__C)

.const:xdc_runtime_Startup_sfxnTab__C 
*          0    0000145c    00000004     
                  0000145c    00000004     pdmstream_pem3.oem3 (.const:xdc_runtime_Startup_sfxnTab__C)

.const:xdc_runtime_Startup_startModsFxn__C 
*          0    00001460    00000004     
                  00001460    00000004     pdmstream_pem3.oem3 (.const:xdc_runtime_Startup_startModsFxn__C)

.const:xdc_runtime_SysCallback_abortFxn__C 
*          0    00001464    00000004     
                  00001464    00000004     pdmstream_pem3.oem3 (.const:xdc_runtime_SysCallback_abortFxn__C)

.const:xdc_runtime_SysCallback_exitFxn__C 
*          0    00001468    00000004     
                  00001468    00000004     pdmstream_pem3.oem3 (.const:xdc_runtime_SysCallback_exitFxn__C)

.const:xdc_runtime_System_abortFxn__C 
*          0    0000146c    00000004     
                  0000146c    00000004     pdmstream_pem3.oem3 (.const:xdc_runtime_System_abortFxn__C)

.const:xdc_runtime_System_exitFxn__C 
*          0    00001470    00000004     
                  00001470    00000004     pdmstream_pem3.oem3 (.const:xdc_runtime_System_exitFxn__C)

.const:xdc_runtime_System_maxAtexitHandlers__C 
*          0    00001474    00000004     
                  00001474    00000004     pdmstream_pem3.oem3 (.const:xdc_runtime_System_maxAtexitHandlers__C)

.const:xdc_runtime_Text_charTab__C 
*          0    00001478    00000004     
                  00001478    00000004     pdmstream_pem3.oem3 (.const:xdc_runtime_Text_charTab__C)

.const:xdc_runtime_Text_nameEmpty__C 
*          0    0000147c    00000004     
                  0000147c    00000004     pdmstream_pem3.oem3 (.const:xdc_runtime_Text_nameEmpty__C)

.const:xdc_runtime_Text_nameStatic__C 
*          0    00001480    00000004     
                  00001480    00000004     pdmstream_pem3.oem3 (.const:xdc_runtime_Text_nameStatic__C)

.const:xdc_runtime_Text_nameUnknown__C 
*          0    00001484    00000004     
                  00001484    00000004     pdmstream_pem3.oem3 (.const:xdc_runtime_Text_nameUnknown__C)

.const:xdc_runtime_Main_Module__id__C 
*          0    00001488    00000002     
                  00001488    00000002     pdmstream_pem3.oem3 (.const:xdc_runtime_Main_Module__id__C)

.const:xdc_runtime_Memory_Module__id__C 
*          0    0000148a    00000002     
                  0000148a    00000002     pdmstream_pem3.oem3 (.const:xdc_runtime_Memory_Module__id__C)

.const:xdc_runtime_Text_charCnt__C 
*          0    0000148c    00000002     
                  0000148c    00000002     pdmstream_pem3.oem3 (.const:xdc_runtime_Text_charCnt__C)

.const:xdc_runtime_Text_isLoaded__C 
*          0    0000148e    00000002     
                  0000148e    00000002     pdmstream_pem3.oem3 (.const:xdc_runtime_Text_isLoaded__C)

.const:ti_sysbios_rom_ROM_AONRTCChannelEnable 
*          0    00001494    00000004     
                  00001494    00000004     pdmstream_pem3.oem3 (.const:ti_sysbios_rom_ROM_AONRTCChannelEnable)

.const:ti_sysbios_rom_ROM_AONRTCCompareValueSet 
*          0    00001498    00000004     
                  00001498    00000004     pdmstream_pem3.oem3 (.const:ti_sysbios_rom_ROM_AONRTCCompareValueSet)

.const:ti_sysbios_rom_ROM_AONRTCCurrentCompareValueGet 
*          0    0000149c    00000004     
                  0000149c    00000004     pdmstream_pem3.oem3 (.const:ti_sysbios_rom_ROM_AONRTCCurrentCompareValueGet)

.const:ti_sysbios_rom_ROM_AONRTCEventClear 
*          0    000014a0    00000004     
                  000014a0    00000004     pdmstream_pem3.oem3 (.const:ti_sysbios_rom_ROM_AONRTCEventClear)

.const:ti_sysbios_rom_ROM_ti_sysbios_family_arm_cc26xx_Timer_getCount64__E 
*          0    000014a4    00000004     
                  000014a4    00000004     pdmstream_pem3.oem3 (.const:ti_sysbios_rom_ROM_ti_sysbios_family_arm_cc26xx_Timer_getCount64__E)

.const:ti_sysbios_rom_ROM_ti_sysbios_family_arm_cc26xx_Timer_getCurrentTick__E 
*          0    000014a8    00000004     
                  000014a8    00000004     pdmstream_pem3.oem3 (.const:ti_sysbios_rom_ROM_ti_sysbios_family_arm_cc26xx_Timer_getCurrentTick__E)

.const:ti_sysbios_rom_ROM_ti_sysbios_family_arm_cc26xx_Timer_getMaxTicks__E 
*          0    000014ac    00000004     
                  000014ac    00000004     pdmstream_pem3.oem3 (.const:ti_sysbios_rom_ROM_ti_sysbios_family_arm_cc26xx_Timer_getMaxTicks__E)

.const:ti_sysbios_rom_ROM_ti_sysbios_family_arm_cc26xx_Timer_setNextTick__E 
*          0    000014b4    00000004     
                  000014b4    00000004     pdmstream_pem3.oem3 (.const:ti_sysbios_rom_ROM_ti_sysbios_family_arm_cc26xx_Timer_setNextTick__E)

.const:ti_sysbios_rom_ROM_ti_sysbios_family_arm_cc26xx_Timer_setThreshold__I 
*          0    000014b8    00000004     
                  000014b8    00000004     pdmstream_pem3.oem3 (.const:ti_sysbios_rom_ROM_ti_sysbios_family_arm_cc26xx_Timer_setThreshold__I)

.const:ti_sysbios_rom_ROM_ti_sysbios_family_arm_cc26xx_Timer_start__E 
*          0    000014bc    00000004     
                  000014bc    00000004     pdmstream_pem3.oem3 (.const:ti_sysbios_rom_ROM_ti_sysbios_family_arm_cc26xx_Timer_start__E)

.const:ti_sysbios_rom_ROM_ti_sysbios_family_arm_cc26xx_TimestampProvider_get32__E 
*          0    000014c0    00000004     
                  000014c0    00000004     pdmstream_pem3.oem3 (.const:ti_sysbios_rom_ROM_ti_sysbios_family_arm_cc26xx_TimestampProvider_get32__E)

.const:ti_sysbios_rom_ROM_xdc_runtime_Startup_getState__I 
*          0    000014c4    00000004     
                  000014c4    00000004     pdmstream_pem3.oem3 (.const:ti_sysbios_rom_ROM_xdc_runtime_Startup_getState__I)

.const:ti_sysbios_rom_ROM_xdc_runtime_System_SupportProxy_abort__E 
*          0    000014c8    00000004     
                  000014c8    00000004     pdmstream_pem3.oem3 (.const:ti_sysbios_rom_ROM_xdc_runtime_System_SupportProxy_abort__E)

.const:ti_sysbios_rom_ROM_xdc_runtime_System_SupportProxy_exit__E 
*          0    000014cc    00000004     
                  000014cc    00000004     pdmstream_pem3.oem3 (.const:ti_sysbios_rom_ROM_xdc_runtime_System_SupportProxy_exit__E)

.const:ti_sysbios_knl_Clock_Module_State_clockQ__O 
*          0    000014d4    00000004     
                  000014d4    00000004     pdmstream_pem3.oem3 (.const:ti_sysbios_knl_Clock_Module_State_clockQ__O)

.const:ti_sysbios_knl_Mailbox_Instance_State_dataSem__O 
*          0    000014dc    00000004     
                  000014dc    00000004     pdmstream_pem3.oem3 (.const:ti_sysbios_knl_Mailbox_Instance_State_dataSem__O)

.const:ti_sysbios_knl_Mailbox_Instance_State_freeQue__O 
*          0    000014e0    00000004     
                  000014e0    00000004     pdmstream_pem3.oem3 (.const:ti_sysbios_knl_Mailbox_Instance_State_freeQue__O)

.const:ti_sysbios_knl_Mailbox_Instance_State_freeSem__O 
*          0    000014e4    00000004     
                  000014e4    00000004     pdmstream_pem3.oem3 (.const:ti_sysbios_knl_Mailbox_Instance_State_freeSem__O)

.const:ti_sysbios_knl_Semaphore_Instance_State_pendQ__O 
*          0    000014e8    00000004     
                  000014e8    00000004     pdmstream_pem3.oem3 (.const:ti_sysbios_knl_Semaphore_Instance_State_pendQ__O)

.data:ti_sysbios_knl_Task_Module__state__V 
*          0    20000100    00000044     UNINITIALIZED
                  20000100    00000044     pdmstream_pem3.oem3 (.data:ti_sysbios_knl_Task_Module__state__V)

.data:ti_sysbios_family_arm_m3_Hwi_Module__state__V 
*          0    20000144    00000034     UNINITIALIZED
                  20000144    00000034     pdmstream_pem3.oem3 (.data:ti_sysbios_family_arm_m3_Hwi_Module__state__V)

.data:ti_sysbios_BIOS_Module__state__V 
*          0    200001a4    00000024     UNINITIALIZED
                  200001a4    00000024     pdmstream_pem3.oem3 (.data:ti_sysbios_BIOS_Module__state__V)

.data:ti_sysbios_knl_Swi_Module__state__V 
*          0    200001c8    0000001c     UNINITIALIZED
                  200001c8    0000001c     pdmstream_pem3.oem3 (.data:ti_sysbios_knl_Swi_Module__state__V)

.data:ti_sysbios_family_arm_cc26xx_Timer_Module__state__V 
*          0    200001e4    00000008     UNINITIALIZED
                  200001e4    00000008     pdmstream_pem3.oem3 (.data:ti_sysbios_family_arm_cc26xx_Timer_Module__state__V)

.data:xdc_runtime_System_Module__state__V 
*          0    200001f8    00000008     UNINITIALIZED
                  200001f8    00000008     pdmstream_pem3.oem3 (.data:xdc_runtime_System_Module__state__V)

.bss       0    20000208    00003377     UNINITIALIZED
                  20000208    00002000     (.common:ti_sysbios_heaps_HeapMem_Instance_State_0_buf__A)
                  20002208    00000300     drivers_cc13xxware.aem3 : PDMCC26XX.oem3 (.bss:pdmContinuousBuffer)
                  20002508    00000300     (.common:task0Stack)
                  20002808    00000200     pdmstream_pem3.oem3 (.bss:taskStackSection)
                  20002a08    000001f4     drivers_cc13xxware.aem3 : PDMCC26XX.oem3 (.bss:pdmTaskStack)
                  20002bfc    0000012c     (.common:uartCC26XXObjects)
                  20002d28    00000120     rtsv7M3_T_le_eabi.lib : trgmsg.c.obj (.bss:_CIOBUF_)
                  20002e48    00000100     pdm_cc13xxware.aem3 : pdm2pcm_ccs.oem3 (.bss)
                  20002f48    000000c8     (.common:ti_sysbios_family_arm_m3_Hwi_dispatchTable)
                  20003010    0000009c     (.common:pdmCC26XXI2SObjects)
                  200030ac    00000080     CC1350STK.obj (.bss:uartStringBuf)
                  2000312c    00000080     (.common:xdc_runtime_SysMin_Module_State_0_outbuf__A)
                  200031ac    0000007c     drivers_cc13xxware.aem3 : PINCC26XX.oem3 (.bss:PIN_HandleTable)
                  20003228    00000074     (.common:pdmCC26XXObjects)
                  2000329c    0000006c                             : PDMCC26XX.oem3 (.bss:decimationFilterInRAM)
                  20003308    00000050                             : PDMCC26XX.oem3 (.bss:pdmTask)
                  20003358    00000050     (.common:task0Struct)
                  200033a8    00000034                             : PINCC26XX.oem3 (.bss:PinSwi)
                  200033dc    00000024                             : PDMCC26XX.oem3 (.bss:pdmContMgtBuffer)
                  20003400    00000020     (.common:PinGpioConfigTable)
                  20003420    00000020     (.common:displayUartObject)
                  20003440    00000020     (.common:uartCC26XXRingBuffer)
                  20003460    0000001c     (.common:PinHwi)
                  2000347c    0000001c     (.common:PinSem)
                  20003498    0000001c     (.common:semStruct)
                  200034b4    00000018     (.common:g_ControlTable)
                  200034cc    00000014     driverlib.lib : osc.obj (.bss:oscHfGlobals)
                  200034e0    00000014     (.common:sPDMEvents)
                  200034f4    0000000c     pdmstream.obj (.bss:buttonPinState)
                  20003500    0000000c     pdmstream.obj (.bss:ledPinState)
                  2000350c    0000000c     (.common:i2sBlockAvailIn)
                  20003518    0000000c     (.common:i2sBlockReadyIn)
                  20003524    0000000c     (.common:pcmMsgReady)
                  20003530    00000009     pdmstream.obj (.bss)
                  20003539    00000001     (.common:Codec1_siEnc)
                  2000353a    00000002     (.common:Codec1_pvEnc)
                  2000353c    00000008     driverlib.lib : sys_ctrl.obj (.bss:powerQualGlobals)
                  20003544    00000008     (.common:parmbuf)
                  2000354c    00000008     (.common:pdmStream)
                  20003554    00000004     (.common:PIN_NumPins)
                  20003558    00000004     (.common:activePcmBuffer)
                  2000355c    00000004     (.common:g_pControlTable)
                  20003560    00000004     (.common:i2sBlockAvailInQueue)
                  20003564    00000004     (.common:i2sBlockReadyInQueue)
                  20003568    00000004     (.common:i2sHandle)
                  2000356c    00000004     (.common:pPinGpio)
                  20003570    00000004     (.common:pcmMsgReadyQueue)
                  20003574    00000004     (.common:pdmEvents)
                  20003578    00000004     (.common:saSem)
                  2000357c    00000001     (.common:driverlib_release_0_47020)
                  2000357d    00000001     (.common:uartRxPowerConstraint)
                  2000357e    00000001     (.common:uartTxPowerConstraint)

.data      0    20003580    0000046e     UNINITIALIZED
                  20003580    00000110     drivers_cc13xxware.aem3 : PowerCC26XX.oem3 (.data:PowerCC26XX_module)
                  20003690    00000080     pdmstream_pem3.oem3 (.data:ti_sysbios_knl_Swi_Module_State_0_readyQ__A)
                  20003710    0000004c     pdmstream_pem3.oem3 (.data:ti_sysbios_knl_Task_Object__table__V)
                  2000375c    00000004     drivers_cc13xxware.aem3 : UART.oem3 (.data)
                  20003760    00000048     pdmstream_pem3.oem3 (.data:ti_sysbios_family_arm_cc26xx_Timer_Object__table__V)
                  200037a8    00000040     drivers_cc13xxware.aem3 : PDMCC26XX.oem3 (.data:decimationState)
                  200037e8    00000038     pdmstream_pem3.oem3 (.data:ti_sysbios_gates_GateMutex_Object__table__V)
                  20003820    00000034     pdmstream.obj (.data)
                  20003854    00000030     pdmstream_pem3.oem3 (.data:ti_sysbios_knl_Swi_Object__table__V)
                  20003884    00000024     pdmstream.obj (.data:pdmParams)
                  200038a8    00000020     pdmstream_pem3.oem3 (.data:ti_sysbios_knl_Clock_Object__table__V)
                  200038c8    00000020     pdmstream_pem3.oem3 (.data:ti_sysbios_knl_Task_Module_State_0_readyQ__A)
                  200038e8    00000018     pdmstream_pem3.oem3 (.data:ti_sysbios_family_arm_m3_Hwi_Object__table__V)
                  20003900    00000018     pdmstream_pem3.oem3 (.data:ti_sysbios_heaps_HeapMem_Object__table__V)
                  20003918    00000010     drivers_cc13xxware.aem3 : PDMCC26XX.oem3 (.data)
                  20003928    00000010     pdmstream.obj (.data:volumeIndicator$3)
                  20003938    0000000c     pdmstream.obj (.data:buttonPinTable)
                  20003944    0000000c     pdmstream.obj (.data:ledPinTable)
                  20003950    0000000c     pdmstream_pem3.oem3 (.data:xdc_runtime_SysMin_Module__state__V)
                  2000395c    00000008     rtsv7M3_T_le_eabi.lib : _lock.c.obj (.data:$O1$$)
                  20003964    00000008     drivers_cc13xxware.aem3 : PDMCC26XX_util.oem3 (.data)
                  2000396c    00000008     pdmstream_pem3.oem3 (.data:ti_sysbios_family_arm_m3_Hwi_Module__root__V)
                  20003974    00000008     pdmstream_pem3.oem3 (.data:ti_sysbios_gates_GateHwi_Module__root__V)
                  2000397c    00000008     pdmstream_pem3.oem3 (.data:ti_sysbios_gates_GateMutex_Module__root__V)
                  20003984    00000008     pdmstream_pem3.oem3 (.data:ti_sysbios_hal_Hwi_Module__root__V)
                  2000398c    00000008     pdmstream_pem3.oem3 (.data:ti_sysbios_heaps_HeapMem_Module__root__V)
                  20003994    00000008     pdmstream_pem3.oem3 (.data:ti_sysbios_knl_Clock_Module__root__V)
                  2000399c    00000008     pdmstream_pem3.oem3 (.data:ti_sysbios_knl_Event_Module__root__V)
                  200039a4    00000008     pdmstream_pem3.oem3 (.data:ti_sysbios_knl_Mailbox_Module__root__V)
                  200039ac    00000008     pdmstream_pem3.oem3 (.data:ti_sysbios_knl_Queue_Module__root__V)
                  200039b4    00000008     pdmstream_pem3.oem3 (.data:ti_sysbios_knl_Semaphore_Module__root__V)
                  200039bc    00000008     pdmstream_pem3.oem3 (.data:ti_sysbios_knl_Swi_Module__root__V)
                  200039c4    00000008     pdmstream_pem3.oem3 (.data:ti_sysbios_knl_Task_Module__root__V)
                  200039cc    00000008     pdmstream_pem3.oem3 (.data:xdc_runtime_Registry_Module__state__V)
                  200039d4    00000008     pdmstream_pem3.oem3 (.data:xdc_runtime_System_Module_State_0_atexitHandlers__A)
                  200039dc    00000004     rtsv7M3_T_le_eabi.lib : stkdepth_vars.c.obj (.data)
                  200039e0    00000004     pdmstream_pem3.oem3 (.data:ti_sysbios_family_arm_m3_Hwi_Module_State_0_excContext__A)
                  200039e4    00000004     pdmstream_pem3.oem3 (.data:ti_sysbios_family_arm_m3_Hwi_Module_State_0_excStack__A)
                  200039e8    00000004     pdmstream_pem3.oem3 (.data:ti_sysbios_knl_Task_Module_State_0_idleTask__A)
                  200039ec    00000002     pdmstream_pem3.oem3 (.data:ti_sysbios_family_arm_m3_Hwi_Module_State_0_excActive__A)

.stack     0    20004d00    00000300     UNINITIALIZED
                  20004d00    00000300     --HOLE--

.const:xdc_runtime_Error_policy__C 
*          0    00001490    00000001     
                  00001490    00000001     pdmstream_pem3.oem3 (.const:xdc_runtime_Error_policy__C)

.const:ti_sysbios_rom_ROM_ti_sysbios_family_arm_cc26xx_Timer_initDevice__I 
*          0    000014b0    00000004     
                  000014b0    00000004     pdmstream_pem3.oem3 (.const:ti_sysbios_rom_ROM_ti_sysbios_family_arm_cc26xx_Timer_initDevice__I)

.const:ti_sysbios_gates_GateMutex_Instance_State_sem__O 
*          0    000014d0    00000004     
                  000014d0    00000004     pdmstream_pem3.oem3 (.const:ti_sysbios_gates_GateMutex_Instance_State_sem__O)

.const:ti_sysbios_knl_Mailbox_Instance_State_dataQue__O 
*          0    000014d8    00000004     
                  000014d8    00000004     pdmstream_pem3.oem3 (.const:ti_sysbios_knl_Mailbox_Instance_State_dataQue__O)

.const:ti_sysbios_knl_Task_Module_State_inactiveQ__O 
*          0    000014ec    00000004     
                  000014ec    00000004     pdmstream_pem3.oem3 (.const:ti_sysbios_knl_Task_Module_State_inactiveQ__O)

.data:ti_sysbios_knl_Clock_Module__state__V 
*          0    20000178    0000002c     UNINITIALIZED
                  20000178    0000002c     pdmstream_pem3.oem3 (.data:ti_sysbios_knl_Clock_Module__state__V)

.data:ti_sysbios_family_arm_cc26xx_TimestampProvider_Module__state__V 
*          0    200001ec    00000004     UNINITIALIZED
                  200001ec    00000004     pdmstream_pem3.oem3 (.data:ti_sysbios_family_arm_cc26xx_TimestampProvider_Module__state__V)

.data:xdc_runtime_Startup_Module__state__V 
*          0    200001f0    00000008     UNINITIALIZED
                  200001f0    00000008     pdmstream_pem3.oem3 (.data:xdc_runtime_Startup_Module__state__V)

.data:xdc_runtime_Memory_Module__state__V 
*          0    20000200    00000004     UNINITIALIZED
                  20000200    00000004     pdmstream_pem3.oem3 (.data:xdc_runtime_Memory_Module__state__V)

.bootVecs 
*          0    00000000    00000008     DSECT
                  00000000    00000008     boot.aem3 : boot.oem3 (.bootVecs)

.resetVecs 
*          0    00000000    0000003c     
                  00000000    0000003c     pdmstream_pem3.oem3 (.resetVecs)

.vecs      0    20000000    000000c8     NOLOAD SECTION
                  20000000    000000c8     pdmstream_pem3.oem3 (.vecs)

xdc.meta   0    00000000    000000fe     COPY SECTION
                  00000000    000000fe     pdmstream_pem3.oem3 (xdc.meta)

xdc.noload 
*          0    00000000    00000000     COPY SECTION

MODULE SUMMARY

       Module                            code    ro data   rw data
       ------                            ----    -------   -------
    .\
       pdmstream.obj                     2428    0         1041   
       CC1350STK.obj                     0       268       764    
       ccfg.obj                          0       88        0      
    +--+---------------------------------+-------+---------+---------+
       Total:                            2428    356       1805   
                                                                  
    E:\Projects\CCS\CC1310\WSFensterKontakt\pdmstream_CC1350STK_TI\Debug\configPkg\package\cfg\
       pdmstream_pem3.oem3               762     1551      10122  
    +--+---------------------------------+-------+---------+---------+
       Total:                            762     1551      10122  
                                                                  
    C:/ti/tirtos_cc13xx_cc26xx_2_21_00_06/products/cc13xxware_2_04_03_17272/driverlib/bin/ccs/driverlib.lib
       setup_rom.obj                     1472    0         0      
       sys_ctrl.obj                      748     0         8      
       osc.obj                           376     0         20     
       i2s.obj                           380     0         4      
       setup.obj                         360     0         0      
       chipinfo.obj                      230     0         0      
       prcm.obj                          48      0         0      
       aon_rtc.obj                       44      0         0      
       ddi.obj                           44      0         0      
       adi.obj                           40      0         0      
       aon_batmon.obj                    40      0         0      
       cpu.obj                           24      0         0      
       vims.obj                          14      0         0      
       driverlib_release.obj             0       0         1      
    +--+---------------------------------+-------+---------+---------+
       Total:                            3820    0         33     
                                                                  
    C:/ti/tirtos_cc13xx_cc26xx_2_21_00_06/products/tidrivers_cc13xx_cc26xx_2_21_00_04/packages/ti/drivers/lib/drivers_cc13xxware.aem3
       PDMCC26XX.oem3                    1790    154       1628   
       UARTCC26XX.oem3                   2664    104       2      
       PowerCC26XX.oem3                  2096    76        272    
       PDMCC26XX_util.oem3               1698    0         64     
       PINCC26XX.oem3                    1426    0         272    
       PowerCC26XX_calibrateRCOSC.oem3   1476    0         0      
       Codec1.oem3                       292     194       3      
       RingBuf.oem3                      152     0         0      
       UART.oem3                         92      36        4      
       List.oem3                         82      0         0      
    +--+---------------------------------+-------+---------+---------+
       Total:                            11768   564       2245   
                                                                  
    C:/ti/tirtos_cc13xx_cc26xx_2_21_00_06/products/tidrivers_cc13xx_cc26xx_2_21_00_04/packages/ti/drivers/lib/power_cc13xx_tirtos.aem3
       PowerCC26XX_tirtos.oem3           212     0         0      
    +--+---------------------------------+-------+---------+---------+
       Total:                            212     0         0      
                                                                  
    C:/ti/tirtos_cc13xx_cc26xx_2_21_00_06/products/tidrivers_cc13xx_cc26xx_2_21_00_04/packages/ti/drivers/pdm/lib/pdm_cc13xxware.aem3
       pdm2pcm_ccs.oem3                  2316    0         256    
    +--+---------------------------------+-------+---------+---------+
       Total:                            2316    0         256    
                                                                  
    C:/ti/tirtos_cc13xx_cc26xx_2_21_00_06/products/tidrivers_cc13xx_cc26xx_2_21_00_04/packages/ti/drivers/ports/lib/tirtosport.aem3
       HwiP_tirtos.oem3                  4       0         0      
    +--+---------------------------------+-------+---------+---------+
       Total:                            4       0         0      
                                                                  
    C:/ti/tirtos_cc13xx_cc26xx_2_21_00_06/products/tidrivers_cc13xx_cc26xx_2_21_00_04/packages/ti/mw/display/lib/display.aem3
       DisplayUart.oem3                  204     28        0      
       Display.oem3                      128     1         0      
    +--+---------------------------------+-------+---------+---------+
       Total:                            332     29        0      
                                                                  
    C:\ti81\ccsv8\tools\compiler\ti-cgt-arm_18.1.3.LTS\lib\rtsv7M3_T_le_eabi.lib
       trgmsg.c.obj                      108     0         288    
       memcpy_t2.asm.obj                 156     0         0      
       ull_div_t2.asm.obj                150     0         0      
       memset_t2.asm.obj                 122     0         0      
       copy_decompress_lzss.c.obj        104     0         0      
       hostwrite.c.obj                   88      0         0      
       cpy_tbl.c.obj                     76      0         0      
       u_divt2.asm.obj                   64      0         0      
       _lock.c.obj                       26      0         8      
       args_main.c.obj                   24      0         0      
       ll_mul_t2.asm.obj                 24      0         0      
       strlen.c.obj                      20      0         0      
       copy_decompress_none.c.obj        14      0         0      
       copy_zero_init.c.obj              12      0         0      
       hostopen.c.obj                    0       0         8      
       stkdepth_vars.c.obj               0       0         4      
       div0.asm.obj                      2       0         0      
    +--+---------------------------------+-------+---------+---------+
       Total:                            990     0         308    
                                                                  
    C:\ti\tirtos_cc13xx_cc26xx_2_21_00_06\products\bios_6_46_01_37\packages\ti\targets\arm\rtsarm\lib\auto_init.aem3
       auto_init.oem3                    160     0         0      
    +--+---------------------------------+-------+---------+---------+
       Total:                            160     0         0      
                                                                  
    C:\ti\tirtos_cc13xx_cc26xx_2_21_00_06\products\bios_6_46_01_37\packages\ti\targets\arm\rtsarm\lib\boot.aem3
       boot.oem3                         68      0         0      
    +--+---------------------------------+-------+---------+---------+
       Total:                            68      0         0      
                                                                  
    E:\Projects\CCS\CC1310\WSFensterKontakt\pdmstream_CC1350STK_TI\src\sysbios\rom_sysbios.aem3
       rom_sysbios.obj                   2995    0         0      
       rom_sysbios_config.obj            52      0         0      
    +--+---------------------------------+-------+---------+---------+
       Total:                            3047    0         0      
                                                                  
       Stack:                            0       0         768    
       Linker Generated:                 544     666       0      
    +--+---------------------------------+-------+---------+---------+
       Grand Total:                      26451   3166      15537  


LINKER GENERATED COPY TABLES

__TI_cinit_table @ 000006c8 records: 12, size/record: 8, table size: 96
	.data: load addr=00000488, load size=00000165 bytes, run addr=20003580, run size=0000046e bytes, compression=lzss
	.data:ti_sysbios_family_arm_m3_Hwi_Module__state__V: load addr=000005ed, load size=00000028 bytes, run addr=20000144, run size=00000034 bytes, compression=lzss
	.data:ti_sysbios_knl_Task_Module__state__V: load addr=00000615, load size=00000021 bytes, run addr=20000100, run size=00000044 bytes, compression=lzss
	.data:ti_sysbios_BIOS_Module__state__V: load addr=00000636, load size=0000001f bytes, run addr=200001a4, run size=00000024 bytes, compression=lzss
	.data:ti_sysbios_knl_Clock_Module__state__V: load addr=00000655, load size=0000001d bytes, run addr=20000178, run size=0000002c bytes, compression=lzss
	.data:ti_sysbios_knl_Swi_Module__state__V: load addr=00000672, load size=00000010 bytes, run addr=200001c8, run size=0000001c bytes, compression=lzss
	.data:ti_sysbios_family_arm_cc26xx_Timer_Module__state__V: load addr=00000690, load size=0000000b bytes, run addr=200001e4, run size=00000008 bytes, compression=lzss
	.data:xdc_runtime_System_Module__state__V: load addr=0000069b, load size=0000000b bytes, run addr=200001f8, run size=00000008 bytes, compression=lzss
	.bss: load addr=000006a8, load size=00000008 bytes, run addr=20000208, run size=00003377 bytes, compression=zero_init
	.data:xdc_runtime_Memory_Module__state__V: load addr=000006b0, load size=00000008 bytes, run addr=20000200, run size=00000004 bytes, compression=lzss
	.data:ti_sysbios_family_arm_cc26xx_TimestampProvider_Module__state__V: load addr=000006b8, load size=00000007 bytes, run addr=200001ec, run size=00000004 bytes, compression=lzss
	.data:xdc_runtime_Startup_Module__state__V: load addr=000006bf, load size=00000007 bytes, run addr=200001f0, run size=00000008 bytes, compression=lzss


LINKER GENERATED HANDLER TABLE

__TI_handler_table @ 00000684 records: 3, size/record: 4, table size: 12
	index: 0, handler: __TI_decompress_lzss
	index: 1, handler: __TI_decompress_none
	index: 2, handler: __TI_zero_init


FAR CALL TRAMPOLINES

callee name               trampoline name
   callee addr  tramp addr   call addr  call info
--------------  -----------  ---------  ----------------
xdc_runtime_Core_assignParams__I  $Tramp$TT$L$PI$$xdc_runtime_Core_assignParams__I
   1001c5ed     00007a28     00007970   pdmstream_pem3.oem3 (.text:ti_sysbios_knl_Event_Params__init__S)
xdc_runtime_Startup_startMods__I  $Tramp$TT$L$PI$$xdc_runtime_Startup_startMods__I
   1001c309     00007a30     0000786c   pdmstream_pem3.oem3 (.text:xdc_runtime_Startup_exec__I)
ti_sysbios_knl_Clock_logTick__E  $Tramp$TT$L$PI$$ti_sysbios_knl_Clock_logTick__E
   1001be63     00007a38     0000782a   pdmstream_pem3.oem3 (.text:ti_sysbios_knl_Clock_doTick__I)
ti_sysbios_BIOS_RtsGateProxy_leave__E  $Tramp$TT$L$PI$$ti_sysbios_BIOS_RtsGateProxy_leave__E
   1001c249     00007a40     00007732   pdmstream_pem3.oem3 (.text:ti_sysbios_BIOS_rtsUnlock__I)
ti_sysbios_BIOS_RtsGateProxy_enter__E  $Tramp$TT$L$PI$$ti_sysbios_BIOS_RtsGateProxy_enter__E
   1001c245     00007a48     0000736e   pdmstream_pem3.oem3 (.text:ti_sysbios_BIOS_rtsLock__I)
xdc_runtime_Memory_free__E  $Tramp$TT$L$PI$$xdc_runtime_Memory_free__E
   1001c7fd     00007a50     00007226   pdmstream.obj (.text:SA_audioFree)
xdc_runtime_Core_constructObject__I  $Tramp$TT$L$PI$$xdc_runtime_Core_constructObject__I
   1001c635     00007a58     00007090   pdmstream_pem3.oem3 (.text:ti_sysbios_knl_Event_construct)
ti_sysbios_knl_Task_startup__E  $Tramp$TT$L$PI$$ti_sysbios_knl_Task_startup__E
   1001c305     00007a60     00006f00   pdmstream_pem3.oem3 (.text:ti_sysbios_BIOS_startFunc__I)
ti_sysbios_knl_Swi_startup__E  $Tramp$TT$L$PI$$ti_sysbios_knl_Swi_startup__E
   1001c239     00007a68     00006efc   pdmstream_pem3.oem3 (.text:ti_sysbios_BIOS_startFunc__I)
ti_sysbios_hal_Hwi_startup__E  $Tramp$TT$L$PI$$ti_sysbios_hal_Hwi_startup__E
   1001c289     00007a70     00006ef8   pdmstream_pem3.oem3 (.text:ti_sysbios_BIOS_startFunc__I)
ti_sysbios_family_arm_cc26xx_Timer_startup__E  $Tramp$TT$L$PI$$ti_sysbios_family_arm_cc26xx_Timer_startup__E
   1001b791     00007a78     00006ef4   pdmstream_pem3.oem3 (.text:ti_sysbios_BIOS_startFunc__I)
xdc_runtime_System_atexit__E  $Tramp$TT$L$PI$$xdc_runtime_System_atexit__E
   1001c67d     00007a80     00006eec   pdmstream_pem3.oem3 (.text:ti_sysbios_BIOS_startFunc__I)
ti_sysbios_BIOS_setThreadType__E  $Tramp$TT$L$PI$$ti_sysbios_BIOS_setThreadType__E
   1001c041     00007a88     00006eb8   pdmstream_pem3.oem3 (.text:ti_sysbios_BIOS_atExitFunc__I)
                             0000778c   pdmstream_pem3.oem3 (.text:ti_sysbios_BIOS_exitFunc__I)
xdc_runtime_Memory_alloc__E  $Tramp$TT$L$PI$$xdc_runtime_Memory_alloc__E
   1001c485     00007a90     00006ace   pdmstream.obj (.text:SA_audioMalloc)
xdc_runtime_Error_init__E  $Tramp$TT$L$PI$$xdc_runtime_Error_init__E
   1001c83d     00007a98     00006ab0   pdmstream.obj (.text:SA_audioMalloc)
xdc_runtime_Gate_leaveSystem__E  $Tramp$TT$L$PI$$xdc_runtime_Gate_leaveSystem__E
   1001c875     00007aa0     000068a8   rom_sysbios.aem3 : rom_sysbios.obj (.text:xdc_runtime_SysMin_flush__E)
                             00006be4                    : rom_sysbios.obj (.text:xdc_runtime_SysMin_putch__E)
xdc_runtime_Gate_enterSystem__E  $Tramp$TT$L$PI$$xdc_runtime_Gate_enterSystem__E
   1001c881     00007aa8     0000687a   rom_sysbios.aem3 : rom_sysbios.obj (.text:xdc_runtime_SysMin_flush__E)
                             00006bc6                    : rom_sysbios.obj (.text:xdc_runtime_SysMin_putch__E)
xdc_runtime_System_exit__E  $Tramp$TT$L$PI$$xdc_runtime_System_exit__E
   1001c7cd     00007ab0     00006860   boot.aem3 : boot.oem3 (.text)
                             00007792   pdmstream_pem3.oem3 (.text:ti_sysbios_BIOS_exitFunc__I)
ti_sysbios_knl_Task_Params__init__S  $Tramp$TT$L$PI$$ti_sysbios_knl_Task_Params__init__S
   1001c1d5     00007ab8     00005ee0   drivers_cc13xxware.aem3 : PDMCC26XX.oem3 (.text:PDMCC26XX_init)
                             000077be   pdmstream.obj (.text:ti_sysbios_knl_Task_Params_init)
ti_sysbios_knl_Task_unblockI__E  $Tramp$TT$L$PI$$ti_sysbios_knl_Task_unblockI__E
   1001b9a1     00007ac0     00005b4e   rom_sysbios.aem3 : rom_sysbios.obj (.text:ti_sysbios_knl_Event_post__E)
                             000070c6                    : rom_sysbios.obj (.text:ti_sysbios_knl_Event_pendTimeout__I)
ti_sysbios_knl_Queue_remove__E  $Tramp$TT$L$PI$$ti_sysbios_knl_Queue_remove__E
   1001c11d     00007ac8     00005b3a   rom_sysbios.aem3 : rom_sysbios.obj (.text:ti_sysbios_knl_Event_post__E)
                             000070ba                    : rom_sysbios.obj (.text:ti_sysbios_knl_Event_pendTimeout__I)
ti_sysbios_knl_Queue_head__E  $Tramp$TT$L$PI$$ti_sysbios_knl_Queue_head__E
   1001c2d1     00007ad0     00005b22   rom_sysbios.aem3 : rom_sysbios.obj (.text:ti_sysbios_knl_Event_post__E)
ti_sysbios_knl_Clock_destruct  $Tramp$TT$L$PI$$ti_sysbios_knl_Clock_destruct
   1001c2b5     00007ad8     00005894   drivers_cc13xxware.aem3 : UARTCC26XX.oem3 (.text:UARTCC26XX_close)
ti_sysbios_knl_Swi_destruct  $Tramp$TT$L$PI$$ti_sysbios_knl_Swi_destruct
   1001c2e5     00007ae0     00005874   drivers_cc13xxware.aem3 : UARTCC26XX.oem3 (.text:UARTCC26XX_close)
ti_sysbios_knl_Semaphore_destruct  $Tramp$TT$L$PI$$ti_sysbios_knl_Semaphore_destruct
   1001c2dd     00007ae8     000056f6   drivers_cc13xxware.aem3 : PDMCC26XX_util.oem3 (.text:PDMCC26XX_I2S_close)
                             00005702                           : PDMCC26XX_util.oem3 (.text:PDMCC26XX_I2S_close)
                             00005880                           : UARTCC26XX.oem3 (.text:UARTCC26XX_close)
                             0000588c                           : UARTCC26XX.oem3 (.text:UARTCC26XX_close)
                             0000756c   display.aem3 : DisplayUart.oem3 (.text:DisplayUart_close)
ti_sysbios_family_arm_m3_Hwi_destruct  $Tramp$TT$L$PI$$ti_sysbios_family_arm_m3_Hwi_destruct
   1001c25d     00007af0     000056e8   drivers_cc13xxware.aem3 : PDMCC26XX_util.oem3 (.text:PDMCC26XX_I2S_close)
                             0000586c                           : UARTCC26XX.oem3 (.text:UARTCC26XX_close)
ti_sysbios_family_arm_m3_Hwi_disableInterrupt__E  $Tramp$TT$L$PI$$ti_sysbios_family_arm_m3_Hwi_disableInterrupt__E
   1001b251     00007af8     00005634   drivers_cc13xxware.aem3 : PDMCC26XX_util.oem3 (.text:PDMCC26XX_I2S_stopStream)
ti_sysbios_knl_Clock_scheduleNextTick__E  $Tramp$TT$L$PI$$ti_sysbios_knl_Clock_scheduleNextTick__E
   1001beb9     00007b00     000050a2   rom_sysbios.aem3 : rom_sysbios.obj (.text:ti_sysbios_knl_Clock_workFuncDynamic__E)
ti_sysbios_knl_Clock_walkQueueDynamic__E  $Tramp$TT$L$PI$$ti_sysbios_knl_Clock_walkQueueDynamic__E
   1001a809     00007b08     0000506a   rom_sysbios.aem3 : rom_sysbios.obj (.text:ti_sysbios_knl_Clock_workFuncDynamic__E)
                             00005086                    : rom_sysbios.obj (.text:ti_sysbios_knl_Clock_workFuncDynamic__E)
ti_sysbios_knl_Clock_TimerProxy_getCurrentTick__E  $Tramp$TT$L$PI$$ti_sysbios_knl_Clock_TimerProxy_getCurrentTick__E
   1001c091     00007b10     00005038   rom_sysbios.aem3 : rom_sysbios.obj (.text:ti_sysbios_knl_Clock_workFuncDynamic__E)
                             0000705e                    : rom_sysbios.obj (.text:ti_sysbios_knl_Clock_getTicksUntilInterrupt__E)
ti_sysbios_knl_Semaphore_post__E  $Tramp$TT$L$PI$$ti_sysbios_knl_Semaphore_post__E
   1001ac41     00007b18     00004a28   drivers_cc13xxware.aem3 : PDMCC26XX_util.oem3 (.text:PDMCC26XX_I2S_hwiFxn)
                             000051ce                           : PINCC26XX.oem3 (.text:PIN_open)
                             000056bc   pdmstream.obj (.text:SA_PDMCC26XX_callbackFxn)
                             00006260   display.aem3 : DisplayUart.oem3 (.text:DisplayUart_put5)
                             000063b2   pdmstream.obj (.text:buttonCallbackFxn)
                             000079ca   drivers_cc13xxware.aem3 : PDMCC26XX_util.oem3 (.text:PDMCC26XX_I2S_callback)
                             000079d2                           : UARTCC26XX.oem3 (.text:readSemCallback)
                             000079da                           : UARTCC26XX.oem3 (.text:writeSemCallback)
ti_sysbios_knl_Queue_get__E  $Tramp$TT$L$PI$$ti_sysbios_knl_Queue_get__E
   1001bf0d     00007b20     000049d0   drivers_cc13xxware.aem3 : PDMCC26XX_util.oem3 (.text:PDMCC26XX_I2S_hwiFxn)
                             000064f6                           : PDMCC26XX_util.oem3 (.text:PDMCC26XX_I2S_requestBuffer)
                             0000680c                           : PDMCC26XX.oem3 (.text:PDMCC26XX_requestBuffer)
ti_sysbios_knl_Queue_put__E  $Tramp$TT$L$PI$$ti_sysbios_knl_Queue_put__E
   1001bf29     00007b28     000049aa   drivers_cc13xxware.aem3 : PDMCC26XX_util.oem3 (.text:PDMCC26XX_I2S_hwiFxn)
                             00006572                           : PDMCC26XX.oem3 (.text:PDMCC26XX_setPcmBufferReady)
                             000077f4                           : PDMCC26XX_util.oem3 (.text:PDMCC26XX_I2S_releaseBuffer)
ti_sysbios_BIOS_getCpuFreq__E  $Tramp$TT$L$PI$$ti_sysbios_BIOS_getCpuFreq__E
   1001bff5     00007b30     00004908   drivers_cc13xxware.aem3 : UARTCC26XX.oem3 (.text:UARTCC26XX_initHw)
ti_sysbios_knl_Clock_removeI__E  $Tramp$TT$L$PI$$ti_sysbios_knl_Clock_removeI__E
   1001c2b9     00007b38     000042a8   rom_sysbios.aem3 : rom_sysbios.obj (.text:ti_sysbios_knl_Event_pend__E)
                             000042c8                    : rom_sysbios.obj (.text:ti_sysbios_knl_Event_pend__E)
ti_sysbios_knl_Clock_startI__E  $Tramp$TT$L$PI$$ti_sysbios_knl_Clock_startI__E
   1001a715     00007b40     0000428e   rom_sysbios.aem3 : rom_sysbios.obj (.text:ti_sysbios_knl_Event_pend__E)
ti_sysbios_knl_Task_blockI__E  $Tramp$TT$L$PI$$ti_sysbios_knl_Task_blockI__E
   1001b611     00007b48     0000427e   rom_sysbios.aem3 : rom_sysbios.obj (.text:ti_sysbios_knl_Event_pend__E)
ti_sysbios_knl_Task_self__E  $Tramp$TT$L$PI$$ti_sysbios_knl_Task_self__E
   1001c1e1     00007b50     0000423c   rom_sysbios.aem3 : rom_sysbios.obj (.text:ti_sysbios_knl_Event_pend__E)
ti_sysbios_knl_Clock_addI__E  $Tramp$TT$L$PI$$ti_sysbios_knl_Clock_addI__E
   1001ba1d     00007b58     0000421c   rom_sysbios.aem3 : rom_sysbios.obj (.text:ti_sysbios_knl_Event_pend__E)
ti_sysbios_family_arm_m3_Hwi_enableInterrupt__E  $Tramp$TT$L$PI$$ti_sysbios_family_arm_m3_Hwi_enableInterrupt__E
   1001b295     00007b60     00003ef2   drivers_cc13xxware.aem3 : PDMCC26XX_util.oem3 (.text:PDMCC26XX_I2S_startStream)
ti_sysbios_knl_Swi_post__E  $Tramp$TT$L$PI$$ti_sysbios_knl_Swi_post__E
   1001b31d     00007b68     00003cf0   drivers_cc13xxware.aem3 : UARTCC26XX.oem3 (.text:UARTCC26XX_read)
                             00003d70                           : UARTCC26XX.oem3 (.text:UARTCC26XX_hwiIntFxn)
                             00007750   rom_sysbios.aem3 : rom_sysbios.obj (.text:ti_sysbios_knl_Swi_or__E)
                             00007832   pdmstream_pem3.oem3 (.text:ti_sysbios_knl_Clock_doTick__I)
ti_sysbios_knl_Clock_setTimeout__E  $Tramp$TT$L$PI$$ti_sysbios_knl_Clock_setTimeout__E
   1001c2bd     00007b70     00003ba6   drivers_cc13xxware.aem3 : PowerCC26XX.oem3 (.text:Power_init)
                             000045b6   power_cc13xx_tirtos.aem3 : PowerCC26XX_tirtos.oem3 (.text:PowerCC26XX_standbyPolicy)
                             00005262   drivers_cc13xxware.aem3 : UARTCC26XX.oem3 (.text:writeFinishedDoCallback)
                             0000535c                           : PowerCC26XX.oem3 (.text:switchXOSCHFclockFunc)
                             000054ea                           : PowerCC26XX.oem3 (.text:disableLFClockQualifiers)
                             00006454                           : PowerCC26XX.oem3 (.text:configureXOSCHF)
                             0000662c                           : UARTCC26XX.oem3 (.text:startTxFifoEmptyClk)
ti_sysbios_knl_Clock_construct  $Tramp$TT$L$PI$$ti_sysbios_knl_Clock_construct
   1001b575     00007b78     00003806   drivers_cc13xxware.aem3 : UARTCC26XX.oem3 (.text:UARTCC26XX_open)
                             00003b02                           : PowerCC26XX.oem3 (.text:Power_init)
                             00003b10                           : PowerCC26XX.oem3 (.text:Power_init)
                             00003b1e                           : PowerCC26XX.oem3 (.text:Power_init)
                             00005c88                           : PowerCC26XX.oem3 (.text:PowerCC26XX_calibrate)
ti_sysbios_knl_Clock_Params__init__S  $Tramp$TT$L$PI$$ti_sysbios_knl_Clock_Params__init__S
   1001c181     00007b80     000037ee   drivers_cc13xxware.aem3 : UARTCC26XX.oem3 (.text:UARTCC26XX_open)
                             00003aea                           : PowerCC26XX.oem3 (.text:Power_init)
                             00005c70                           : PowerCC26XX.oem3 (.text:PowerCC26XX_calibrate)
ti_sysbios_knl_Clock_start__E  $Tramp$TT$L$PI$$ti_sysbios_knl_Clock_start__E
   1001bfdf     00007b88     0000367e   drivers_cc13xxware.aem3 : PowerCC26XX_calibrateRCOSC.oem3 (.text:PowerCC26XX_doCalibrate)
                             00003bac                           : PowerCC26XX.oem3 (.text:Power_init)
                             000045bc   power_cc13xx_tirtos.aem3 : PowerCC26XX_tirtos.oem3 (.text:PowerCC26XX_standbyPolicy)
                             00005268   drivers_cc13xxware.aem3 : UARTCC26XX.oem3 (.text:writeFinishedDoCallback)
                             00005362                           : PowerCC26XX.oem3 (.text:switchXOSCHFclockFunc)
                             000054f0                           : PowerCC26XX.oem3 (.text:disableLFClockQualifiers)
                             0000645a                           : PowerCC26XX.oem3 (.text:configureXOSCHF)
                             00006632                           : UARTCC26XX.oem3 (.text:startTxFifoEmptyClk)
                             000073ba   rom_sysbios.aem3 : rom_sysbios.obj (.text:ti_sysbios_knl_Clock_stop__E)
xdc_runtime_System_abortSpin__E  $Tramp$TT$L$PI$$xdc_runtime_System_abortSpin__E
   1001c895     00007b90     000035f0   drivers_cc13xxware.aem3 : PowerCC26XX_calibrateRCOSC.oem3 (.text:PowerCC26XX_doCalibrate)
                             00006002                           : PowerCC26XX_calibrateRCOSC.oem3 (.text:PowerCC26XX_RCOSC_clockFunc)
ti_sysbios_knl_Queue_enqueue__E  $Tramp$TT$L$PI$$ti_sysbios_knl_Queue_enqueue__E
   1001c1b1     00007b98     0000346a   drivers_cc13xxware.aem3 : PDMCC26XX_util.oem3 (.text:PDMCC26XX_I2S_open)
                             00004278   rom_sysbios.aem3 : rom_sysbios.obj (.text:ti_sysbios_knl_Event_pend__E)
                             00006e02   drivers_cc13xxware.aem3 : PDMCC26XX_util.oem3 (.text:PDMCC26XX_I2S_cleanUpQueues)
ti_sysbios_knl_Queue_construct  $Tramp$TT$L$PI$$ti_sysbios_knl_Queue_construct
   1001b8f1     00007ba0     0000343a   drivers_cc13xxware.aem3 : PDMCC26XX_util.oem3 (.text:PDMCC26XX_I2S_open)
                             0000344c                           : PDMCC26XX_util.oem3 (.text:PDMCC26XX_I2S_open)
                             0000391a                           : PDMCC26XX.oem3 (.text:PDMCC26XX_open)
                             00007848   rom_sysbios.aem3 : rom_sysbios.obj (.text:ti_sysbios_knl_Event_Instance_init__E)
ti_sysbios_family_arm_m3_Hwi_restoreFxn__E  $Tramp$TT$L$PI$$ti_sysbios_family_arm_m3_Hwi_restoreFxn__E
   1001c215     00007ba8     00003366   drivers_cc13xxware.aem3 : PDMCC26XX_util.oem3 (.text:PDMCC26XX_I2S_open)
                             00003374                           : PDMCC26XX_util.oem3 (.text:PDMCC26XX_I2S_open)
                             0000341a                           : PDMCC26XX_util.oem3 (.text:PDMCC26XX_I2S_open)
                             000036c6                           : UARTCC26XX.oem3 (.text:UARTCC26XX_open)
                             000036d6                           : UARTCC26XX.oem3 (.text:UARTCC26XX_open)
                             0000375c                           : UARTCC26XX.oem3 (.text:UARTCC26XX_open)
                             00003864                           : PDMCC26XX.oem3 (.text:PDMCC26XX_open)
                             00003874                           : PDMCC26XX.oem3 (.text:PDMCC26XX_open)
                             00003c8c                           : UARTCC26XX.oem3 (.text:UARTCC26XX_read)
                             00003cca                           : UARTCC26XX.oem3 (.text:UARTCC26XX_read)
                             00003e28                           : PDMCC26XX_util.oem3 (.text:PDMCC26XX_I2S_startStream)
                             00003e3c                           : PDMCC26XX_util.oem3 (.text:PDMCC26XX_I2S_startStream)
                             00003f46                           : UARTCC26XX.oem3 (.text:UARTCC26XX_write)
                             00003f62                           : UARTCC26XX.oem3 (.text:UARTCC26XX_write)
                             00004000                           : UARTCC26XX.oem3 (.text:UARTCC26XX_write)
                             0000439a                           : PINCC26XX.oem3 (.text:PINCC26XX_setIoCfg)
                             00004702                           : PowerCC26XX.oem3 (.text:Power_releaseDependency)
                             000047d2                           : PowerCC26XX.oem3 (.text:Power_setDependency)
                             00004b72                           : PDMCC26XX.oem3 (.text:PDMCC26XX_startStream)
                             00004b8a                           : PDMCC26XX.oem3 (.text:PDMCC26XX_startStream)
                             0000521e                           : UARTCC26XX.oem3 (.text:writeFinishedDoCallback)
                             0000538a                           : PowerCC26XX.oem3 (.text:switchXOSCHFclockFunc)
                             00005446                           : UARTCC26XX.oem3 (.text:UARTCC26XX_writeCancel)
                             00005452                           : UARTCC26XX.oem3 (.text:UARTCC26XX_writeCancel)
                             00005494                           : UARTCC26XX.oem3 (.text:UARTCC26XX_writeCancel)
                             000055e6                           : PDMCC26XX_util.oem3 (.text:PDMCC26XX_I2S_stopStream)
                             00005602                           : PDMCC26XX_util.oem3 (.text:PDMCC26XX_I2S_stopStream)
                             00005616                           : PDMCC26XX_util.oem3 (.text:PDMCC26XX_I2S_stopStream)
                             0000572c                           : PDMCC26XX_util.oem3 (.text:PDMCC26XX_I2S_close)
                             000058a0                           : UARTCC26XX.oem3 (.text:UARTCC26XX_close)
                             00005ce4                           : UARTCC26XX.oem3 (.text:UARTCC26XX_readCancel)
                             00005cf0                           : UARTCC26XX.oem3 (.text:UARTCC26XX_readCancel)
                             00005cfa                           : UARTCC26XX.oem3 (.text:UARTCC26XX_readCancel)
                             00005f62                           : UARTCC26XX.oem3 (.text:UARTCC26XX_control)
                             0000630a                           : PDMCC26XX.oem3 (.text:PDMCC26XX_rollbackDriverInitialisation)
                             0000633e                           : PowerCC26XX_calibrateRCOSC.oem3 (.text:PowerCC26XX_initiateCalibration)
                             000063d8                           : PDMCC26XX.oem3 (.text:PDMCC26XX_stopStream)
                             000063e6                           : PDMCC26XX.oem3 (.text:PDMCC26XX_stopStream)
                             00006702                           : PINCC26XX.oem3 (.text:PIN_setOutputEnable)
                             000067bc                           : RingBuf.oem3 (.text:RingBuf_put)
                             000067e6                           : RingBuf.oem3 (.text:RingBuf_put)
                             0000692e                           : RingBuf.oem3 (.text:RingBuf_get)
                             00006936                           : RingBuf.oem3 (.text:RingBuf_get)
                             00006a16                           : UARTCC26XX.oem3 (.text:UARTCC26XX_swiIntFxn)
                             00006e40                           : PowerCC26XX.oem3 (.text:Power_releaseConstraint)
                             00006e70                           : PowerCC26XX.oem3 (.text:Power_setConstraint)
                             000071e2                           : List.oem3 (.text:List_put)
                             0000735c                           : PowerCC26XX.oem3 (.text:Power_unregisterNotify)
ti_sysbios_family_arm_m3_Hwi_disableFxn__E  $Tramp$TT$L$PI$$ti_sysbios_family_arm_m3_Hwi_disableFxn__E
   1001c145     00007bb0     0000335a   drivers_cc13xxware.aem3 : PDMCC26XX_util.oem3 (.text:PDMCC26XX_I2S_open)
                             00003412                           : PDMCC26XX_util.oem3 (.text:PDMCC26XX_I2S_open)
                             000036bc                           : UARTCC26XX.oem3 (.text:UARTCC26XX_open)
                             00003756                           : UARTCC26XX.oem3 (.text:UARTCC26XX_open)
                             00003858                           : PDMCC26XX.oem3 (.text:PDMCC26XX_open)
                             00003c74                           : UARTCC26XX.oem3 (.text:UARTCC26XX_read)
                             00003cb6                           : UARTCC26XX.oem3 (.text:UARTCC26XX_read)
                             00003e1e                           : PDMCC26XX_util.oem3 (.text:PDMCC26XX_I2S_startStream)
                             00003f28                           : UARTCC26XX.oem3 (.text:UARTCC26XX_write)
                             00003f4a                           : UARTCC26XX.oem3 (.text:UARTCC26XX_write)
                             00003fa2                           : UARTCC26XX.oem3 (.text:UARTCC26XX_write)
                             00003fec                           : UARTCC26XX.oem3 (.text:UARTCC26XX_write)
                             0000437c                           : PINCC26XX.oem3 (.text:PINCC26XX_setIoCfg)
                             0000464e                           : PowerCC26XX.oem3 (.text:Power_releaseDependency)
                             00004722                           : PowerCC26XX.oem3 (.text:Power_setDependency)
                             00004b0c                           : PDMCC26XX.oem3 (.text:PDMCC26XX_startStream)
                             00005206                           : UARTCC26XX.oem3 (.text:writeFinishedDoCallback)
                             00005314                           : PowerCC26XX.oem3 (.text:switchXOSCHFclockFunc)
                             00005436                           : UARTCC26XX.oem3 (.text:UARTCC26XX_writeCancel)
                             0000547e                           : UARTCC26XX.oem3 (.text:UARTCC26XX_writeCancel)
                             000055d0                           : PDMCC26XX_util.oem3 (.text:PDMCC26XX_I2S_stopStream)
                             00005724                           : PDMCC26XX_util.oem3 (.text:PDMCC26XX_I2S_close)
                             00005898                           : UARTCC26XX.oem3 (.text:UARTCC26XX_close)
                             00005ccc                           : UARTCC26XX.oem3 (.text:UARTCC26XX_readCancel)
                             00005ce8                           : UARTCC26XX.oem3 (.text:UARTCC26XX_readCancel)
                             00005f3a                           : UARTCC26XX.oem3 (.text:UARTCC26XX_control)
                             00006300                           : PDMCC26XX.oem3 (.text:PDMCC26XX_rollbackDriverInitialisation)
                             0000632a                           : PowerCC26XX_calibrateRCOSC.oem3 (.text:PowerCC26XX_initiateCalibration)
                             000063ce                           : PDMCC26XX.oem3 (.text:PDMCC26XX_stopStream)
                             000066ec                           : PINCC26XX.oem3 (.text:PIN_setOutputEnable)
                             000067ae                           : RingBuf.oem3 (.text:RingBuf_put)
                             00006906                           : RingBuf.oem3 (.text:RingBuf_get)
                             000069fe                           : UARTCC26XX.oem3 (.text:UARTCC26XX_swiIntFxn)
                             00006e20                           : PowerCC26XX.oem3 (.text:Power_releaseConstraint)
                             00006e50                           : PowerCC26XX.oem3 (.text:Power_setConstraint)
                             0000734c                           : PowerCC26XX.oem3 (.text:Power_unregisterNotify)
                             00007a04   tirtosport.aem3 : HwiP_tirtos.oem3 (.text:HwiP_disable)
ti_sysbios_knl_Swi_construct  $Tramp$TT$L$PI$$ti_sysbios_knl_Swi_construct
   1001b085     00007bb8     000032e4   drivers_cc13xxware.aem3 : PINCC26XX.oem3 (.text:PIN_init)
                             000037aa                           : UARTCC26XX.oem3 (.text:UARTCC26XX_open)
ti_sysbios_knl_Swi_Params__init__S  $Tramp$TT$L$PI$$ti_sysbios_knl_Swi_Params__init__S
   1001c1c9     00007bc0     000032d2   drivers_cc13xxware.aem3 : PINCC26XX.oem3 (.text:PIN_init)
                             00003794                           : UARTCC26XX.oem3 (.text:UARTCC26XX_open)
ti_sysbios_family_arm_m3_Hwi_construct  $Tramp$TT$L$PI$$ti_sysbios_family_arm_m3_Hwi_construct
   1001af29     00007bc8     000032c6   drivers_cc13xxware.aem3 : PINCC26XX.oem3 (.text:PIN_init)
                             0000349e                           : PDMCC26XX_util.oem3 (.text:PDMCC26XX_I2S_open)
                             00003788                           : UARTCC26XX.oem3 (.text:UARTCC26XX_open)
                             00005c98                           : PowerCC26XX.oem3 (.text:PowerCC26XX_calibrate)
ti_sysbios_family_arm_m3_Hwi_Params__init__S  $Tramp$TT$L$PI$$ti_sysbios_family_arm_m3_Hwi_Params__init__S
   1001c139     00007bd0     000032b0   drivers_cc13xxware.aem3 : PINCC26XX.oem3 (.text:PIN_init)
                             00003482                           : PDMCC26XX_util.oem3 (.text:PDMCC26XX_I2S_open)
                             0000376c                           : UARTCC26XX.oem3 (.text:UARTCC26XX_open)
ti_sysbios_knl_Semaphore_Params__init__S  $Tramp$TT$L$PI$$ti_sysbios_knl_Semaphore_Params__init__S
   1001c1bd     00007bd8     0000323c   drivers_cc13xxware.aem3 : PINCC26XX.oem3 (.text:PIN_init)
                             000034aa                           : PDMCC26XX_util.oem3 (.text:PDMCC26XX_I2S_open)
                             000034cc                           : PDMCC26XX_util.oem3 (.text:PDMCC26XX_I2S_open)
                             000037b6                           : UARTCC26XX.oem3 (.text:UARTCC26XX_open)
                             00006534   display.aem3 : DisplayUart.oem3 (.text:DisplayUart_open)
                             000077a8   pdmstream.obj (.text:ti_sysbios_knl_Semaphore_Params_init)
ti_sysbios_knl_Task_restore__E  $Tramp$TT$L$PI$$ti_sysbios_knl_Task_restore__E
   1001ba45     00007be0     00002f58   drivers_cc13xxware.aem3 : PowerCC26XX.oem3 (.text:Power_sleep)
                             00004298   rom_sysbios.aem3 : rom_sysbios.obj (.text:ti_sysbios_knl_Event_pend__E)
                             00005b58                    : rom_sysbios.obj (.text:ti_sysbios_knl_Event_post__E)
ti_sysbios_knl_Swi_restore__E  $Tramp$TT$L$PI$$ti_sysbios_knl_Swi_restore__E
   1001b5dd     00007be8     00002f4e   drivers_cc13xxware.aem3 : PowerCC26XX.oem3 (.text:Power_sleep)
ti_sysbios_knl_Swi_disable__E  $Tramp$TT$L$PI$$ti_sysbios_knl_Swi_disable__E
   1001c0d1     00007bf0     00002daa   drivers_cc13xxware.aem3 : PowerCC26XX.oem3 (.text:Power_sleep)
                             00006eae   pdmstream_pem3.oem3 (.text:ti_sysbios_BIOS_atExitFunc__I)
ti_sysbios_knl_Task_disable__E  $Tramp$TT$L$PI$$ti_sysbios_knl_Task_disable__E
   1001c0f1     00007bf8     00002d92   drivers_cc13xxware.aem3 : PowerCC26XX.oem3 (.text:Power_sleep)
                             00004268   rom_sysbios.aem3 : rom_sysbios.obj (.text:ti_sysbios_knl_Event_pend__E)
                             00005b1a                    : rom_sysbios.obj (.text:ti_sysbios_knl_Event_post__E)
                             00006eb2   pdmstream_pem3.oem3 (.text:ti_sysbios_BIOS_atExitFunc__I)
ti_sysbios_BIOS_start__E  $Tramp$TT$L$PI$$ti_sysbios_BIOS_start__E
   1001c051     00007c00     000029c2   pdmstream.obj (.text:main)
ti_sysbios_knl_Semaphore_construct  $Tramp$TT$L$PI$$ti_sysbios_knl_Semaphore_construct
   1001b705     00007c08     000029a0   pdmstream.obj (.text:main)
                             0000324e   drivers_cc13xxware.aem3 : PINCC26XX.oem3 (.text:PIN_init)
                             000034bc                           : PDMCC26XX_util.oem3 (.text:PDMCC26XX_I2S_open)
                             000034dc                           : PDMCC26XX_util.oem3 (.text:PDMCC26XX_I2S_open)
                             000037ca                           : UARTCC26XX.oem3 (.text:UARTCC26XX_open)
                             000037de                           : UARTCC26XX.oem3 (.text:UARTCC26XX_open)
                             00006542   display.aem3 : DisplayUart.oem3 (.text:DisplayUart_open)
ti_sysbios_knl_Task_construct  $Tramp$TT$L$PI$$ti_sysbios_knl_Task_construct
   1001b125     00007c10     0000293c   pdmstream.obj (.text:main)
                             00005efa   drivers_cc13xxware.aem3 : PDMCC26XX.oem3 (.text:PDMCC26XX_init)
xdc_runtime_System_abort__E  $Tramp$TT$L$PI$$xdc_runtime_System_abort__E
   1001c745     00007c18     0000291c   pdmstream.obj (.text:main)
                             0000295a   pdmstream.obj (.text:main)
                             0000297e   pdmstream.obj (.text:main)
                             00002990   pdmstream.obj (.text:main)
ti_sysbios_knl_Task_sleep__E  $Tramp$TT$L$PI$$ti_sysbios_knl_Task_sleep__E
   1001a9d9     00007c20     00002794   pdmstream.obj (.text:taskFxn)
ti_sysbios_knl_Semaphore_pend__E  $Tramp$TT$L$PI$$ti_sysbios_knl_Semaphore_pend__E
   1001a001     00007c28     00002712   pdmstream.obj (.text:taskFxn)
                             00003cae   drivers_cc13xxware.aem3 : UARTCC26XX.oem3 (.text:UARTCC26XX_read)
                             00003f8e                           : UARTCC26XX.oem3 (.text:UARTCC26XX_write)
                             00003fca                           : UARTCC26XX.oem3 (.text:UARTCC26XX_write)
                             00005166                           : PINCC26XX.oem3 (.text:PIN_open)
                             0000560e                           : PDMCC26XX_util.oem3 (.text:PDMCC26XX_I2S_stopStream)
                             00005a5a                           : UARTCC26XX.oem3 (.text:writeTxFifoFlush)
                             0000621c   display.aem3 : DisplayUart.oem3 (.text:DisplayUart_put5)
                             000064d4   drivers_cc13xxware.aem3 : PDMCC26XX_util.oem3 (.text:PDMCC26XX_I2S_requestBuffer)
ti_sysbios_knl_Queue_destruct  $Tramp$TT$L$PI$$ti_sysbios_knl_Queue_destruct
   1001c2cd     00007c30     000023d4   drivers_cc13xxware.aem3 : PDMCC26XX.oem3 (.text:PDMCC26XX_taskFxn)
                             00005712                           : PDMCC26XX_util.oem3 (.text:PDMCC26XX_I2S_close)
                             00005718                           : PDMCC26XX_util.oem3 (.text:PDMCC26XX_I2S_close)
ti_sysbios_knl_Queue_empty__E  $Tramp$TT$L$PI$$ti_sysbios_knl_Queue_empty__E
   1001c10f     00007c38     000023ca   drivers_cc13xxware.aem3 : PDMCC26XX.oem3 (.text:PDMCC26XX_taskFxn)
                             000049c8                           : PDMCC26XX_util.oem3 (.text:PDMCC26XX_I2S_hwiFxn)
                             00004b56                           : PDMCC26XX.oem3 (.text:PDMCC26XX_startStream)
                             00005b14   rom_sysbios.aem3 : rom_sysbios.obj (.text:ti_sysbios_knl_Event_post__E)
                             000064ee   drivers_cc13xxware.aem3 : PDMCC26XX_util.oem3 (.text:PDMCC26XX_I2S_requestBuffer)
                             000067fe                           : PDMCC26XX.oem3 (.text:PDMCC26XX_requestBuffer)
                             00006e08                           : PDMCC26XX_util.oem3 (.text:PDMCC26XX_I2S_cleanUpQueues)
ti_sysbios_knl_Queue_dequeue__E  $Tramp$TT$L$PI$$ti_sysbios_knl_Queue_dequeue__E
   1001c1a5     00007c40     000023ae   drivers_cc13xxware.aem3 : PDMCC26XX.oem3 (.text:PDMCC26XX_taskFxn)
                             00003e74                           : PDMCC26XX_util.oem3 (.text:PDMCC26XX_I2S_startStream)
                             00003e90                           : PDMCC26XX_util.oem3 (.text:PDMCC26XX_I2S_startStream)
                             00004b3c                           : PDMCC26XX.oem3 (.text:PDMCC26XX_startStream)
                             00006dfa                           : PDMCC26XX_util.oem3 (.text:PDMCC26XX_I2S_cleanUpQueues)

[68 trampolines]
[254 trampoline calls]


GLOBAL SYMBOLS: SORTED ALPHABETICALLY BY Name 

address   name                                                                      
-------   ----                                                                      
0000015c  BoardGpioInitTable                                                        
00006b0b  C$$IO$$                                                                   
000057c9  Codec1_encodeBuff                                                         
00004bb5  Codec1_encodeSingle                                                       
000048b7  DisplayUart_clear                                                         
00004eeb  DisplayUart_clearLines                                                    
0000755b  DisplayUart_close                                                         
000079e7  DisplayUart_control                                                       
0000036c  DisplayUart_fxnTable                                                      
000079ed  DisplayUart_getType                                                       
00006511  DisplayUart_open                                                          
00006211  DisplayUart_put5                                                          
00000388  Display_config                                                            
00000486  Display_defaultParams                                                     
000078ff  Display_doClear                                                           
00006641  Display_doOpen                                                            
000079f3  Display_doParamsInit                                                      
0000719d  Display_doPut5                                                            
00006269  HOSTwrite                                                                 
00007a05  HwiP_disable                                                              
1001c215  HwiP_restore                                                              
000079a9  List_empty                                                                
00007a09  List_head                                                                 
00007a0d  List_next                                                                 
000071c3  List_put                                                                  
0000750d  List_remove                                                               
000070fd  NOROM_AONBatMonTemperatureGetDegC                                         
000077c5  NOROM_AONRTCCurrent64BitValueGet                                          
00007575  NOROM_AONRTCCurrentCompareValueGet                                        
0000790b  NOROM_CPUcpsid                                                            
00007917  NOROM_CPUcpsie                                                            
00006689  NOROM_ChipInfo_GetChipFamily                                              
00005a89  NOROM_ChipInfo_GetHwRevision                                              
0000758d  NOROM_ChipInfo_GetPackageType                                             
00006f9d  NOROM_DDI32RegWrite                                                       
00007309  NOROM_I2SAudioFormatConfigure                                             
000075a5  NOROM_I2SBufferConfig                                                     
000043c5  NOROM_I2SChannelConfigure                                                 
00007125  NOROM_I2SEnable                                                           
000077d9  NOROM_I2SPointerSet                                                       
00006d5d  NOROM_I2SSampleStampConfigure                                             
00006fc9  NOROM_OSCClockSourceGet                                                   
00005f81  NOROM_OSCClockSourceSet                                                   
00005e55  NOROM_OSCHF_AttemptToSwitchToXosc                                         
00006bf5  NOROM_OSCHF_SwitchToRcOscTurnOffXosc                                      
000075bd  NOROM_OSCHF_TurnOnXosc                                                    
00006981  NOROM_OSC_HPOSCRelativeFrequencyOffsetGet                                 
00006d8d  NOROM_PRCMAudioClockConfigSetOverride                                     
00004d09  NOROM_SetupAfterColdResetWakeupFromShutDownCfg1                           
0000410d  NOROM_SetupAfterColdResetWakeupFromShutDownCfg2                           
0000398d  NOROM_SetupAfterColdResetWakeupFromShutDownCfg3                           
000075d5  NOROM_SetupGetTrimForAdcShModeEn                                          
000075ed  NOROM_SetupGetTrimForAdcShVbufEn                                          
00005bd9  NOROM_SetupGetTrimForAmpcompCtrl                                          
00007605  NOROM_SetupGetTrimForAmpcompTh1                                           
00007465  NOROM_SetupGetTrimForAmpcompTh2                                           
00005d1d  NOROM_SetupGetTrimForAnabypassValue1                                      
0000761d  NOROM_SetupGetTrimForDblrLoopFilterResetVoltage                           
00006ff5  NOROM_SetupGetTrimForRadcExtCfg                                           
00007635  NOROM_SetupGetTrimForRcOscLfIBiasTrim                                     
00007481  NOROM_SetupGetTrimForRcOscLfRtuneCtuneTrim                                
00007329  NOROM_SetupGetTrimForXoscHfCtl                                            
00007875  NOROM_SetupGetTrimForXoscHfFastStart                                      
00007885  NOROM_SetupGetTrimForXoscHfIbiastherm                                     
0000764d  NOROM_SetupGetTrimForXoscLfRegulatorAndCmirrwrRatio                       
00006dbd  NOROM_SetupSetAonRtcSubSecInc                                             
00006471  NOROM_SetupSetCacheModeAccordingToCcfgSetting                             
000058b9  NOROM_SetupSetVddrLevel                                                   
00004c61  NOROM_SetupTrimDevice                                                     
000060a1  NOROM_SysCtrlAdjustRechargeAfterPowerDown                                 
00002b49  NOROM_SysCtrlSetRechargeBeforePowerDown                                   
00005d85  NOROM_SysCtrl_DCDC_VoltageConditionalControl                              
0000776d  NOROM_ThisCodeIsBuiltForCC13xxHwRev20AndLater_HaltIfViolated              
000078d5  NOROM_VIMSModeGet                                                         
000056d1  PDMCC26XX_I2S_close                                                       
00000408  PDMCC26XX_I2S_config                                                      
00007665  PDMCC26XX_I2S_init                                                        
00003349  PDMCC26XX_I2S_open                                                        
000077ed  PDMCC26XX_I2S_releaseBuffer                                               
000064c1  PDMCC26XX_I2S_requestBuffer                                               
00003e15  PDMCC26XX_I2S_startStream                                                 
000055cd  PDMCC26XX_I2S_stopStream                                                  
00007895  PDMCC26XX_close                                                           
0000044c  PDMCC26XX_config                                                          
00005eb9  PDMCC26XX_init                                                            
00003849  PDMCC26XX_open                                                            
000067f1  PDMCC26XX_requestBuffer                                                   
00004b05  PDMCC26XX_startStream                                                     
000063c9  PDMCC26XX_stopStream                                                      
000071e9  PINCC26XX_getPinCount                                                     
00000454  PINCC26XX_hwAttrs                                                         
00007021  PINCC26XX_setMux                                                          
200031ac  PIN_HandleTable                                                           
20003554  PIN_NumPins                                                               
00007429  PIN_close                                                                 
00007801  PIN_getInputValue                                                         
00003185  PIN_init                                                                  
00005155  PIN_open                                                                  
00007923  PIN_registerIntCb                                                         
000060fd  PIN_remove                                                                
00006c29  PIN_setConfig                                                             
00006a6d  PIN_setInterrupt                                                          
000066d1  PIN_setOutputEnable                                                       
000069bd  PIN_setOutputValue                                                        
00005fe1  PowerCC26XX_RCOSC_clockFunc                                               
0000592d  PowerCC26XX_auxISR                                                        
00005c45  PowerCC26XX_calibrate                                                     
00000418  PowerCC26XX_config                                                        
00003509  PowerCC26XX_doCalibrate                                                   
00006319  PowerCC26XX_initiateCalibration                                           
20003580  PowerCC26XX_module                                                        
00004575  PowerCC26XX_standbyPolicy                                                 
00007931  Power_getConstraintMask                                                   
0000793d  Power_getDependencyCount                                                  
00007447  Power_getTransitionLatency                                                
00007695  Power_idleFunc                                                            
00003abd  Power_init                                                                
0000714d  Power_registerNotify                                                      
00006e1d  Power_releaseConstraint                                                   
00004649  Power_releaseDependency                                                   
00006e4d  Power_setConstraint                                                       
0000471d  Power_setDependency                                                       
00002d71  Power_sleep                                                               
00007349  Power_unregisterNotify                                                    
00006835  ResetISR                                                                  
00007851  RingBuf_construct                                                         
00006901  RingBuf_get                                                               
000067a9  RingBuf_put                                                               
UNDEFED   SHT$$INIT_ARRAY$$Base                                                     
UNDEFED   SHT$$INIT_ARRAY$$Limit                                                    
00007175  SafeHapiVoid                                                              
00005841  UARTCC26XX_close                                                          
00005f1d  UARTCC26XX_control                                                        
00000294  UARTCC26XX_fxnTable                                                       
00003d05  UARTCC26XX_hwiIntFxn                                                      
000076ad  UARTCC26XX_init                                                           
000036a9  UARTCC26XX_open                                                           
00003be9  UARTCC26XX_read                                                           
00005cb1  UARTCC26XX_readCancel                                                     
000079f9  UARTCC26XX_readPolling                                                    
000069f9  UARTCC26XX_swiIntFxn                                                      
00003f19  UARTCC26XX_write                                                          
0000542d  UARTCC26XX_writeCancel                                                    
000079ff  UARTCC26XX_writePolling                                                   
000076c5  UART_Params_init                                                          
000079b3  UART_close                                                                
000003a0  UART_config                                                               
00000308  UART_defaultParams                                                        
00006e7d  UART_open                                                                 
000079bd  UART_write                                                                
00000000  __ASM__                                                                   
20002d28  __CIOBUF_                                                                 
00000078  __ISA__                                                                   
0000008a  __PLAT__                                                                  
20005000  __STACK_END                                                               
00000300  __STACK_SIZE                                                              
20005000  __STACK_TOP                                                               
000000b1  __TARG__                                                                  
000006c8  __TI_CINIT_Base                                                           
00000728  __TI_CINIT_Limit                                                          
00000684  __TI_Handler_Table_Base                                                   
00000690  __TI_Handler_Table_Limit                                                  
00004dad  __TI_auto_init                                                            
00005ded  __TI_decompress_lzss                                                      
000078e3  __TI_decompress_none                                                      
ffffffff  __TI_pprof_out_hndl                                                       
ffffffff  __TI_prof_data_size                                                       
ffffffff  __TI_prof_data_start                                                      
00006c5d  __TI_readmsg                                                              
00000000  __TI_static_base__                                                        
00006add  __TI_writemsg                                                             
00007961  __TI_zero_init                                                            
000000d6  __TRDR__                                                                  
00005bd7  __aeabi_idiv0                                                             
00005bd7  __aeabi_ldiv0                                                             
0000770d  __aeabi_lmul                                                              
0000574d  __aeabi_memclr                                                            
0000574d  __aeabi_memclr4                                                           
0000574d  __aeabi_memclr8                                                           
00004f89  __aeabi_memcpy                                                            
00004f89  __aeabi_memcpy4                                                           
00004f89  __aeabi_memcpy8                                                           
0000574f  __aeabi_memset                                                            
0000574f  __aeabi_memset4                                                           
0000574f  __aeabi_memset8                                                           
00006941  __aeabi_uidiv                                                             
00006941  __aeabi_uidivmod                                                          
000050bd  __aeabi_uldivmod                                                          
ffffffff  __binit__                                                                 
ffffffff  __c_args__                                                                
0001ffa8  __ccfg                                                                    
20004d00  __stack                                                                   
000076dd  _args_main                                                                
00006835  _c_int00                                                                  
2000395c  _lock                                                                     
00005153  _nop                                                                      
00007949  _register_lock                                                            
00007955  _register_unlock                                                          
20003960  _unlock                                                                   
ffffffff  binit                                                                     
00006371  buttonCallbackFxn                                                         
20003938  buttonPinTable                                                            
000065a9  copy_in                                                                   
000003d0  displayUartHWAttrs                                                        
20003420  displayUartObject                                                         
2000357c  driverlib_release_0_47020                                                 
200034b4  g_ControlTable                                                            
2000355c  g_pControlTable                                                           
20003944  ledPinTable                                                               
00002909  main                                                                      
200039dc  main_func_sp                                                              
00004f89  memcpy                                                                    
00005755  memset                                                                    
20003544  parmbuf                                                                   
000014f1  pdm2pcm16k                                                                
00000428  pdmC26XXI2SHWAttrs                                                        
0000045c  pdmCC26XXHWAttrs                                                          
20003010  pdmCC26XXI2SObjects                                                       
20003228  pdmCC26XXObjects                                                          
20003884  pdmParams                                                                 
000001c0  resourceDB                                                                
20003578  saSem                                                                     
20003498  semStruct                                                                 
20003920  streamNotification                                                        
00007815  strlen                                                                    
20002508  task0Stack                                                                
20003358  task0Struct                                                               
00002699  taskFxn                                                                   
200001a4  ti_sysbios_BIOS_Module__state__V                                          
1001bc25  ti_sysbios_BIOS_RtsGateProxy_Handle__label__S                             
1001bc25  ti_sysbios_BIOS_RtsGateProxy_Handle__label__S__mangled__                  
1001bab5  ti_sysbios_BIOS_RtsGateProxy_Object__delete__S                            
1001bab5  ti_sysbios_BIOS_RtsGateProxy_Object__delete__S__mangled__                 
1001c175  ti_sysbios_BIOS_RtsGateProxy_Params__init__S                              
1001c175  ti_sysbios_BIOS_RtsGateProxy_Params__init__S__mangled__                   
1001c245  ti_sysbios_BIOS_RtsGateProxy_enter__E                                     
1001c249  ti_sysbios_BIOS_RtsGateProxy_leave__E                                     
1001c271  ti_sysbios_BIOS_RtsGateProxy_query__E                                     
1001c271  ti_sysbios_BIOS_RtsGateProxy_query__E__mangled__                          
00006ead  ti_sysbios_BIOS_atExitFunc__I                                             
00007783  ti_sysbios_BIOS_exitFunc__I                                               
1001c031  ti_sysbios_BIOS_exit__E                                                   
1001bff5  ti_sysbios_BIOS_getCpuFreq__E                                             
000067ef  ti_sysbios_BIOS_linkedWithIncorrectBootLibrary__E                         
000070fb  ti_sysbios_BIOS_nullFunc__I                                               
00007255  ti_sysbios_BIOS_registerRTSLock__I                                        
00007279  ti_sysbios_BIOS_removeRTSLock__I                                          
00007369  ti_sysbios_BIOS_rtsLock__I                                                
00007725  ti_sysbios_BIOS_rtsUnlock__I                                              
1001c041  ti_sysbios_BIOS_setThreadType__E                                          
00006edd  ti_sysbios_BIOS_startFunc__I                                              
1001c051  ti_sysbios_BIOS_start__E                                                  
00004c61  ti_sysbios_family_arm_cc26xx_Boot_trimDevice                              
00001406  ti_sysbios_family_arm_cc26xx_Timer_Module__id__C                          
1001bb45  ti_sysbios_family_arm_cc26xx_Timer_Module__startupDone__S                 
200001e4  ti_sysbios_family_arm_cc26xx_Timer_Module__state__V                       
1001ba6d  ti_sysbios_family_arm_cc26xx_Timer_Module_startup__E                      
20003760  ti_sysbios_family_arm_cc26xx_Timer_Object__table__V                       
00007389  ti_sysbios_family_arm_cc26xx_Timer_dynamicStub__E                         
00007a15  ti_sysbios_family_arm_cc26xx_Timer_getCount64__E                          
00006b4d  ti_sysbios_family_arm_cc26xx_Timer_getCurrentTick__E                      
1001c24d  ti_sysbios_family_arm_cc26xx_Timer_getExpiredTicks__E                     
0000729d  ti_sysbios_family_arm_cc26xx_Timer_getMaxTicks__E                         
1001c251  ti_sysbios_family_arm_cc26xx_Timer_getPeriod__E                           
00006cc5  ti_sysbios_family_arm_cc26xx_Timer_initDevice__I                          
1001a465  ti_sysbios_family_arm_cc26xx_Timer_periodicStub__E                        
1001b765  ti_sysbios_family_arm_cc26xx_Timer_postInit__I                            
00006d2b  ti_sysbios_family_arm_cc26xx_Timer_setNextTick__E                         
1001c255  ti_sysbios_family_arm_cc26xx_Timer_setPeriod__E                           
00006f0d  ti_sysbios_family_arm_cc26xx_Timer_setThreshold__I                        
000059a1  ti_sysbios_family_arm_cc26xx_Timer_start__E                               
00001384  ti_sysbios_family_arm_cc26xx_Timer_startupNeeded__C                       
1001b791  ti_sysbios_family_arm_cc26xx_Timer_startup__E                             
200001ec  ti_sysbios_family_arm_cc26xx_TimestampProvider_Module__state__V           
1001bb65  ti_sysbios_family_arm_cc26xx_TimestampProvider_Module_startup__E          
000078f1  ti_sysbios_family_arm_cc26xx_TimestampProvider_get32__E                   
1001b9cd  ti_sysbios_family_arm_cc26xx_TimestampProvider_get64__E                   
1001c12b  ti_sysbios_family_arm_cc26xx_TimestampProvider_getFreq__E                 
00001408  ti_sysbios_family_arm_cc26xx_TimestampProvider_useClockTimer__C           
00001388  ti_sysbios_family_arm_m3_Hwi_E_alreadyDefined__C                          
0000138c  ti_sysbios_family_arm_m3_Hwi_E_hwiLimitExceeded__C                        
1001aed1  ti_sysbios_family_arm_m3_Hwi_Instance_finalize__E                         
1001a3c5  ti_sysbios_family_arm_m3_Hwi_Instance_init__E                             
200039ec  ti_sysbios_family_arm_m3_Hwi_Module_State_0_excActive__A                  
200039e0  ti_sysbios_family_arm_m3_Hwi_Module_State_0_excContext__A                 
200039e4  ti_sysbios_family_arm_m3_Hwi_Module_State_0_excStack__A                   
0000140a  ti_sysbios_family_arm_m3_Hwi_Module__id__C                                
2000396c  ti_sysbios_family_arm_m3_Hwi_Module__root__V                              
1001bb85  ti_sysbios_family_arm_m3_Hwi_Module__startupDone__S                       
20000144  ti_sysbios_family_arm_m3_Hwi_Module__state__V                             
1001b1c1  ti_sysbios_family_arm_m3_Hwi_Module_startup__E                            
00001390  ti_sysbios_family_arm_m3_Hwi_NUM_INTERRUPTS__C                            
000011d0  ti_sysbios_family_arm_m3_Hwi_Object__DESC__C                              
00001070  ti_sysbios_family_arm_m3_Hwi_Object__PARAMS__C                            
00001394  ti_sysbios_family_arm_m3_Hwi_Object__count__C                             
1001aab1  ti_sysbios_family_arm_m3_Hwi_Object__create__S                            
1001bba5  ti_sysbios_family_arm_m3_Hwi_Object__delete__S                            
1001be65  ti_sysbios_family_arm_m3_Hwi_Object__destruct__S                          
1001b7bd  ti_sysbios_family_arm_m3_Hwi_Object__get__S                               
00001398  ti_sysbios_family_arm_m3_Hwi_Object__table__C                             
200038e8  ti_sysbios_family_arm_m3_Hwi_Object__table__V                             
1001c139  ti_sysbios_family_arm_m3_Hwi_Params__init__S                              
0000139c  ti_sysbios_family_arm_m3_Hwi_ccr__C                                       
000074d5  ti_sysbios_family_arm_m3_Hwi_clearInterrupt__E                            
1001af29  ti_sysbios_family_arm_m3_Hwi_construct                                    
1001ab15  ti_sysbios_family_arm_m3_Hwi_create                                       
1001c259  ti_sysbios_family_arm_m3_Hwi_delete                                       
1001c25d  ti_sysbios_family_arm_m3_Hwi_destruct                                     
1001c145  ti_sysbios_family_arm_m3_Hwi_disableFxn__E                                
1001b251  ti_sysbios_family_arm_m3_Hwi_disableInterrupt__E                          
1001aa49  ti_sysbios_family_arm_m3_Hwi_dispatchC__I                                 
20002f48  ti_sysbios_family_arm_m3_Hwi_dispatchTable                                
1001c899  ti_sysbios_family_arm_m3_Hwi_dispatch__I                                  
1001c1f7  ti_sysbios_family_arm_m3_Hwi_doSwiRestore__I                              
1001c20f  ti_sysbios_family_arm_m3_Hwi_doTaskRestore__I                             
1001c151  ti_sysbios_family_arm_m3_Hwi_enableFxn__E                                 
1001b295  ti_sysbios_family_arm_m3_Hwi_enableInterrupt__E                           
1001c9fd  ti_sysbios_family_arm_m3_Hwi_excHandlerAsm__I                             
000013a0  ti_sysbios_family_arm_m3_Hwi_excHandlerFunc__C                            
1001bbc5  ti_sysbios_family_arm_m3_Hwi_excHandler__I                                
1001b461  ti_sysbios_family_arm_m3_Hwi_getStackInfo__E                              
1001a695  ti_sysbios_family_arm_m3_Hwi_initNVIC__E                                  
1001c9b5  ti_sysbios_family_arm_m3_Hwi_initStacks__E                                
000013a4  ti_sysbios_family_arm_m3_Hwi_nullIsrFunc__C                               
000013a8  ti_sysbios_family_arm_m3_Hwi_numSparseInterrupts__C                       
e000e000  ti_sysbios_family_arm_m3_Hwi_nvic                                         
1001ca3b  ti_sysbios_family_arm_m3_Hwi_pendSV__I                                    
1001c061  ti_sysbios_family_arm_m3_Hwi_plug__E                                      
1001a315  ti_sysbios_family_arm_m3_Hwi_postInit__I                                  
000013ac  ti_sysbios_family_arm_m3_Hwi_priGroup__C                                  
20000000  ti_sysbios_family_arm_m3_Hwi_ramVectors                                   
00000000  ti_sysbios_family_arm_m3_Hwi_resetVectors                                 
1001c215  ti_sysbios_family_arm_m3_Hwi_restoreFxn__E                                
1001ca53  ti_sysbios_family_arm_m3_Hwi_return                                       
1001be81  ti_sysbios_family_arm_m3_Hwi_setPriority__E                               
1001c1ff  ti_sysbios_family_arm_m3_Hwi_startup__E                                   
1001c009  ti_sysbios_family_arm_m3_Hwi_switchFromBootStack__E                       
1001c261  ti_sysbios_family_arm_m3_TaskSupport_Module__startupDone__S               
1001c969  ti_sysbios_family_arm_m3_TaskSupport_buildTaskStack                       
1001c15d  ti_sysbios_family_arm_m3_TaskSupport_getStackAlignment__E                 
1001ca55  ti_sysbios_family_arm_m3_TaskSupport_glue                                 
000013b0  ti_sysbios_family_arm_m3_TaskSupport_stackAlignment__C                    
1001b499  ti_sysbios_family_arm_m3_TaskSupport_start__E                             
1001ca65  ti_sysbios_family_arm_m3_TaskSupport_swap__E                              
1001ca1d  ti_sysbios_family_xxx_Hwi_switchAndRunFunc                                
1001bbe5  ti_sysbios_gates_GateHwi_Handle__label__S                                 
1001b45f  ti_sysbios_gates_GateHwi_Instance_init__E                                 
0000111c  ti_sysbios_gates_GateHwi_Module__FXNS__C                                  
0000140c  ti_sysbios_gates_GateHwi_Module__id__C                                    
20003974  ti_sysbios_gates_GateHwi_Module__root__V                                  
000011f0  ti_sysbios_gates_GateHwi_Object__DESC__C                                  
00001330  ti_sysbios_gates_GateHwi_Object__PARAMS__C                                
1001ba91  ti_sysbios_gates_GateHwi_Object__create__S                                
1001bc05  ti_sysbios_gates_GateHwi_Object__delete__S                                
1001c169  ti_sysbios_gates_GateHwi_enter__E                                         
1001c21b  ti_sysbios_gates_GateHwi_leave__E                                         
1001c265  ti_sysbios_gates_GateHwi_query__E                                         
1001bc25  ti_sysbios_gates_GateMutex_Handle__label__S                               
000014d0  ti_sysbios_gates_GateMutex_Instance_State_sem__O                          
1001c071  ti_sysbios_gates_GateMutex_Instance_finalize__E                           
1001be9d  ti_sysbios_gates_GateMutex_Instance_init__E                               
00001140  ti_sysbios_gates_GateMutex_Module__FXNS__C                                
0000140e  ti_sysbios_gates_GateMutex_Module__id__C                                  
2000397c  ti_sysbios_gates_GateMutex_Module__root__V                                
00001210  ti_sysbios_gates_GateMutex_Object__DESC__C                                
00001348  ti_sysbios_gates_GateMutex_Object__PARAMS__C                              
1001b645  ti_sysbios_gates_GateMutex_Object__create__S                              
1001bab5  ti_sysbios_gates_GateMutex_Object__delete__S                              
1001bc45  ti_sysbios_gates_GateMutex_Object__destruct__S                            
200037e8  ti_sysbios_gates_GateMutex_Object__table__V                               
1001c175  ti_sysbios_gates_GateMutex_Params__init__S                                
1001b7e9  ti_sysbios_gates_GateMutex_construct                                      
1001b675  ti_sysbios_gates_GateMutex_create                                         
1001c269  ti_sysbios_gates_GateMutex_delete                                         
1001c26d  ti_sysbios_gates_GateMutex_destruct                                       
1001b6a5  ti_sysbios_gates_GateMutex_enter__E                                       
1001bf99  ti_sysbios_gates_GateMutex_leave__E                                       
1001c271  ti_sysbios_gates_GateMutex_query__E                                       
1001c275  ti_sysbios_hal_Hwi_HwiProxy_Module__startupDone__S                        
1001bb85  ti_sysbios_hal_Hwi_HwiProxy_Module__startupDone__S__mangled__             
1001c081  ti_sysbios_hal_Hwi_HwiProxy_Object__create__S                             
1001bba5  ti_sysbios_hal_Hwi_HwiProxy_Object__delete__S                             
1001bba5  ti_sysbios_hal_Hwi_HwiProxy_Object__delete__S__mangled__                  
1001c139  ti_sysbios_hal_Hwi_HwiProxy_Params__init__S                               
1001c139  ti_sysbios_hal_Hwi_HwiProxy_Params__init__S__mangled__                    
000074d5  ti_sysbios_hal_Hwi_HwiProxy_clearInterrupt__E                             
1001be45  ti_sysbios_hal_Hwi_HwiProxy_create                                        
1001c279  ti_sysbios_hal_Hwi_HwiProxy_delete                                        
1001c27d  ti_sysbios_hal_Hwi_HwiProxy_disableInterrupt__E                           
1001b251  ti_sysbios_hal_Hwi_HwiProxy_disableInterrupt__E__mangled__                
1001c281  ti_sysbios_hal_Hwi_HwiProxy_enableInterrupt__E                            
1001b295  ti_sysbios_hal_Hwi_HwiProxy_enableInterrupt__E__mangled__                 
1001c285  ti_sysbios_hal_Hwi_HwiProxy_getStackInfo__E                               
1001b461  ti_sysbios_hal_Hwi_HwiProxy_getStackInfo__E__mangled__                    
1001c289  ti_sysbios_hal_Hwi_HwiProxy_startup__E                                    
1001c1ff  ti_sysbios_hal_Hwi_HwiProxy_startup__E__mangled__                         
1001c28d  ti_sysbios_hal_Hwi_HwiProxy_switchFromBootStack__E                        
1001c009  ti_sysbios_hal_Hwi_HwiProxy_switchFromBootStack__E__mangled__             
1001c1ed  ti_sysbios_hal_Hwi_Instance_finalize__E                                   
1001b9f5  ti_sysbios_hal_Hwi_Instance_init__E                                       
20003984  ti_sysbios_hal_Hwi_Module__root__V                                        
1001c01d  ti_sysbios_hal_Hwi_Module_startup__E                                      
00001230  ti_sysbios_hal_Hwi_Object__DESC__C                                        
000010a0  ti_sysbios_hal_Hwi_Object__PARAMS__C                                      
1001bc65  ti_sysbios_hal_Hwi_Object__delete__S                                      
000074d5  ti_sysbios_hal_Hwi_clearInterrupt__E                                      
1001ab79  ti_sysbios_hal_Hwi_create                                                 
1001c291  ti_sysbios_hal_Hwi_delete                                                 
1001c27d  ti_sysbios_hal_Hwi_disableInterrupt__E                                    
1001c27d  ti_sysbios_hal_Hwi_disableInterrupt__E                                    
1001c281  ti_sysbios_hal_Hwi_enableInterrupt__E                                     
1001c281  ti_sysbios_hal_Hwi_enableInterrupt__E                                     
1001c285  ti_sysbios_hal_Hwi_getStackInfo__E                                        
1001c285  ti_sysbios_hal_Hwi_getStackInfo__E                                        
1001b815  ti_sysbios_hal_Hwi_initStack                                              
1001c289  ti_sysbios_hal_Hwi_startup__E                                             
1001c289  ti_sysbios_hal_Hwi_startup__E                                             
1001c295  ti_sysbios_hal_Hwi_switchFromBootStack__E                                 
1001c295  ti_sysbios_hal_Hwi_switchFromBootStack__E                                 
000013b4  ti_sysbios_heaps_HeapMem_E_memory__C                                      
1001bc85  ti_sysbios_heaps_HeapMem_Handle__label__S                                 
20000208  ti_sysbios_heaps_HeapMem_Instance_State_0_buf__A                          
1001b4d1  ti_sysbios_heaps_HeapMem_Instance_init__E                                 
1001bc25  ti_sysbios_heaps_HeapMem_Module_GateProxy_Handle__label__S                
1001bc25  ti_sysbios_heaps_HeapMem_Module_GateProxy_Handle__label__S__mangled__     
1001bab5  ti_sysbios_heaps_HeapMem_Module_GateProxy_Object__delete__S               
1001bab5  ti_sysbios_heaps_HeapMem_Module_GateProxy_Object__delete__S__mangled__    
1001c175  ti_sysbios_heaps_HeapMem_Module_GateProxy_Params__init__S                 
1001c175  ti_sysbios_heaps_HeapMem_Module_GateProxy_Params__init__S__mangled__      
1001c299  ti_sysbios_heaps_HeapMem_Module_GateProxy_enter__E                        
1001c29d  ti_sysbios_heaps_HeapMem_Module_GateProxy_leave__E                        
1001c271  ti_sysbios_heaps_HeapMem_Module_GateProxy_query__E                        
1001c271  ti_sysbios_heaps_HeapMem_Module_GateProxy_query__E__mangled__             
000010cc  ti_sysbios_heaps_HeapMem_Module__FXNS__C                                  
000013b8  ti_sysbios_heaps_HeapMem_Module__gateObj__C                               
00001410  ti_sysbios_heaps_HeapMem_Module__id__C                                    
2000398c  ti_sysbios_heaps_HeapMem_Module__root__V                                  
00001250  ti_sysbios_heaps_HeapMem_Object__DESC__C                                  
00001164  ti_sysbios_heaps_HeapMem_Object__PARAMS__C                                
000013bc  ti_sysbios_heaps_HeapMem_Object__count__C                                 
1001b841  ti_sysbios_heaps_HeapMem_Object__create__S                                
1001bca5  ti_sysbios_heaps_HeapMem_Object__delete__S                                
1001b86d  ti_sysbios_heaps_HeapMem_Object__get__S                                   
000013c0  ti_sysbios_heaps_HeapMem_Object__table__C                                 
20003900  ti_sysbios_heaps_HeapMem_Object__table__V                                 
1001a195  ti_sysbios_heaps_HeapMem_alloc__E                                         
1001a791  ti_sysbios_heaps_HeapMem_free__E                                          
1001b209  ti_sysbios_heaps_HeapMem_getStats__E                                      
1001b541  ti_sysbios_heaps_HeapMem_init__I                                          
1001c2a1  ti_sysbios_heaps_HeapMem_isBlocking__E                                    
000013c4  ti_sysbios_heaps_HeapMem_reqAlign__C                                      
1001c101  ti_sysbios_heaps_HeapMem_restore__E                                       
1001bfc9  ti_sysbios_knl_Clock_Instance_finalize__E                                 
1001b509  ti_sysbios_knl_Clock_Instance_init__E                                     
000014d4  ti_sysbios_knl_Clock_Module_State_clockQ__O                               
20003994  ti_sysbios_knl_Clock_Module__root__V                                      
20000178  ti_sysbios_knl_Clock_Module__state__V                                     
1001bcc5  ti_sysbios_knl_Clock_Module_startup__E                                    
00001270  ti_sysbios_knl_Clock_Object__DESC__C                                      
00001188  ti_sysbios_knl_Clock_Object__PARAMS__C                                    
1001bad9  ti_sysbios_knl_Clock_Object__delete__S                                    
1001bce5  ti_sysbios_knl_Clock_Object__destruct__S                                  
200038a8  ti_sysbios_knl_Clock_Object__table__V                                     
1001c181  ti_sysbios_knl_Clock_Params__init__S                                      
1001c2a5  ti_sysbios_knl_Clock_TimerProxy_Module__startupDone__S                    
1001bb45  ti_sysbios_knl_Clock_TimerProxy_Module__startupDone__S__mangled__         
1001c091  ti_sysbios_knl_Clock_TimerProxy_getCurrentTick__E                         
1001c2a9  ti_sysbios_knl_Clock_TimerProxy_getExpiredTicks__E                        
1001c0a1  ti_sysbios_knl_Clock_TimerProxy_getMaxTicks__E                            
1001c2ad  ti_sysbios_knl_Clock_TimerProxy_getPeriod__E                              
1001c0b1  ti_sysbios_knl_Clock_TimerProxy_setNextTick__E                            
1001b791  ti_sysbios_knl_Clock_TimerProxy_startup__E                                
1001b791  ti_sysbios_knl_Clock_TimerProxy_startup__E__mangled__                     
1001ba1d  ti_sysbios_knl_Clock_addI__E                                              
1001b575  ti_sysbios_knl_Clock_construct                                            
1001b3e9  ti_sysbios_knl_Clock_create                                               
1001c2b1  ti_sysbios_knl_Clock_delete                                               
1001c2b5  ti_sysbios_knl_Clock_destruct                                             
00007829  ti_sysbios_knl_Clock_doTick__I                                            
0000704d  ti_sysbios_knl_Clock_getTicksUntilInterrupt__E                            
1001b6d5  ti_sysbios_knl_Clock_getTicks__E                                          
1001c18d  ti_sysbios_knl_Clock_getTimerHandle__E                                    
1001be63  ti_sysbios_knl_Clock_logTick__E                                           
1001c2b9  ti_sysbios_knl_Clock_removeI__E                                           
1001beb9  ti_sysbios_knl_Clock_scheduleNextTick__E                                  
000013c8  ti_sysbios_knl_Clock_serviceMargin__C                                     
1001c2bd  ti_sysbios_knl_Clock_setTimeout__E                                        
1001a715  ti_sysbios_knl_Clock_startI__E                                            
1001bfdf  ti_sysbios_knl_Clock_start__E                                             
000073a9  ti_sysbios_knl_Clock_stop__E                                              
00001414  ti_sysbios_knl_Clock_tickMode__C                                          
00000464  ti_sysbios_knl_Clock_tickPeriod__C                                        
00000468  ti_sysbios_knl_Clock_triggerClock__C                                      
00007307  ti_sysbios_knl_Clock_triggerFunc__I                                       
1001a809  ti_sysbios_knl_Clock_walkQueueDynamic__E                                  
00005025  ti_sysbios_knl_Clock_workFuncDynamic__E                                   
1001a881  ti_sysbios_knl_Clock_workFunc__E                                          
0000046c  ti_sysbios_knl_Event_Instance_State_pendQ__O                              
0000783d  ti_sysbios_knl_Event_Instance_init__E                                     
2000399c  ti_sysbios_knl_Event_Module__root__V                                      
0000032c  ti_sysbios_knl_Event_Object__DESC__C                                      
000003b8  ti_sysbios_knl_Event_Object__PARAMS__C                                    
0000796d  ti_sysbios_knl_Event_Params__init__S                                      
000073c9  ti_sysbios_knl_Event_checkEvents__I                                       
00007079  ti_sysbios_knl_Event_construct                                            
000070a5  ti_sysbios_knl_Event_pendTimeout__I                                       
000041fd  ti_sysbios_knl_Event_pend__E                                              
00005af9  ti_sysbios_knl_Event_post__E                                              
00000470  ti_sysbios_knl_Idle_funcList__A                                           
00001378  ti_sysbios_knl_Idle_funcList__C                                           
1001c207  ti_sysbios_knl_Idle_loop__E                                               
1001bd05  ti_sysbios_knl_Idle_run__E                                                
000014d8  ti_sysbios_knl_Mailbox_Instance_State_dataQue__O                          
000014dc  ti_sysbios_knl_Mailbox_Instance_State_dataSem__O                          
000014e0  ti_sysbios_knl_Mailbox_Instance_State_freeQue__O                          
000014e4  ti_sysbios_knl_Mailbox_Instance_State_freeSem__O                          
1001a8f9  ti_sysbios_knl_Mailbox_Instance_finalize__E                               
1001a0cd  ti_sysbios_knl_Mailbox_Instance_init__E                                   
200039a4  ti_sysbios_knl_Mailbox_Module__root__V                                    
1001b2d9  ti_sysbios_knl_Mailbox_Module_startup__E                                  
00001290  ti_sysbios_knl_Mailbox_Object__DESC__C                                    
0000103c  ti_sysbios_knl_Mailbox_Object__PARAMS__C                                  
000013cc  ti_sysbios_knl_Mailbox_Object__count__C                                   
1001bd25  ti_sysbios_knl_Mailbox_Object__delete__S                                  
1001bed5  ti_sysbios_knl_Mailbox_Object__destruct__S                                
1001b899  ti_sysbios_knl_Mailbox_Object__get__S                                     
000013d0  ti_sysbios_knl_Mailbox_Object__table__C                                   
1001c199  ti_sysbios_knl_Mailbox_Params__init__S                                    
1001af81  ti_sysbios_knl_Mailbox_construct                                          
1001abdd  ti_sysbios_knl_Mailbox_create                                             
1001c2c1  ti_sysbios_knl_Mailbox_delete                                             
1001c2c5  ti_sysbios_knl_Mailbox_destruct                                           
000013d4  ti_sysbios_knl_Mailbox_maxTypeAlign__C                                    
1001a969  ti_sysbios_knl_Mailbox_pend__E                                            
1001b8c5  ti_sysbios_knl_Mailbox_postInit__I                                        
1001a58d  ti_sysbios_knl_Mailbox_post__E                                            
1001c227  ti_sysbios_knl_Queue_Instance_init__E                                     
200039ac  ti_sysbios_knl_Queue_Module__root__V                                      
000012b0  ti_sysbios_knl_Queue_Object__DESC__C                                      
00001360  ti_sysbios_knl_Queue_Object__PARAMS__C                                    
000013d8  ti_sysbios_knl_Queue_Object__count__C                                     
1001bd45  ti_sysbios_knl_Queue_Object__delete__S                                    
1001bef1  ti_sysbios_knl_Queue_Object__destruct__S                                  
1001bd65  ti_sysbios_knl_Queue_Object__get__S                                       
000013dc  ti_sysbios_knl_Queue_Object__table__C                                     
1001b8f1  ti_sysbios_knl_Queue_construct                                            
1001b91d  ti_sysbios_knl_Queue_create                                               
1001c2c9  ti_sysbios_knl_Queue_delete                                               
1001c1a5  ti_sysbios_knl_Queue_dequeue__E                                           
1001c2cd  ti_sysbios_knl_Queue_destruct                                             
1001c22d  ti_sysbios_knl_Queue_elemClear__E                                         
1001c10f  ti_sysbios_knl_Queue_empty__E                                             
1001c1b1  ti_sysbios_knl_Queue_enqueue__E                                           
1001bf0d  ti_sysbios_knl_Queue_get__E                                               
1001c2d1  ti_sysbios_knl_Queue_head__E                                              
1001c2d5  ti_sysbios_knl_Queue_next__E                                              
1001bf29  ti_sysbios_knl_Queue_put__E                                               
1001c11d  ti_sysbios_knl_Queue_remove__E                                            
000014e8  ti_sysbios_knl_Semaphore_Instance_State_pendQ__O                          
1001c0c1  ti_sysbios_knl_Semaphore_Instance_finalize__E                             
1001bafd  ti_sysbios_knl_Semaphore_Instance_init__E                                 
200039b4  ti_sysbios_knl_Semaphore_Module__root__V                                  
000012d0  ti_sysbios_knl_Semaphore_Object__DESC__C                                  
000011ac  ti_sysbios_knl_Semaphore_Object__PARAMS__C                                
1001bb21  ti_sysbios_knl_Semaphore_Object__delete__S                                
1001bd85  ti_sysbios_knl_Semaphore_Object__destruct__S                              
1001c1bd  ti_sysbios_knl_Semaphore_Params__init__S                                  
1001b705  ti_sysbios_knl_Semaphore_construct                                        
1001b5a9  ti_sysbios_knl_Semaphore_create                                           
1001c2d9  ti_sysbios_knl_Semaphore_delete                                           
1001c2dd  ti_sysbios_knl_Semaphore_destruct                                         
00007a19  ti_sysbios_knl_Semaphore_getCount__E                                      
1001b949  ti_sysbios_knl_Semaphore_pendTimeout__I                                   
1001a001  ti_sysbios_knl_Semaphore_pend__E                                          
1001ac41  ti_sysbios_knl_Semaphore_post__E                                          
1001bf97  ti_sysbios_knl_Swi_Instance_finalize__E                                   
1001aca5  ti_sysbios_knl_Swi_Instance_init__E                                       
20003690  ti_sysbios_knl_Swi_Module_State_0_readyQ__A                               
200039bc  ti_sysbios_knl_Swi_Module__root__V                                        
200001c8  ti_sysbios_knl_Swi_Module__state__V                                       
1001c233  ti_sysbios_knl_Swi_Module_startup__E                                      
000012f0  ti_sysbios_knl_Swi_Object__DESC__C                                        
000010f4  ti_sysbios_knl_Swi_Object__PARAMS__C                                      
000013e0  ti_sysbios_knl_Swi_Object__count__C                                       
1001bda5  ti_sysbios_knl_Swi_Object__delete__S                                      
1001bf45  ti_sysbios_knl_Swi_Object__destruct__S                                    
1001b975  ti_sysbios_knl_Swi_Object__get__S                                         
000013e4  ti_sysbios_knl_Swi_Object__table__C                                       
20003854  ti_sysbios_knl_Swi_Object__table__V                                       
1001c1c9  ti_sysbios_knl_Swi_Params__init__S                                        
1001b085  ti_sysbios_knl_Swi_construct                                              
1001ad05  ti_sysbios_knl_Swi_create                                                 
1001c2e1  ti_sysbios_knl_Swi_delete                                                 
1001c2e5  ti_sysbios_knl_Swi_destruct                                               
1001c0d1  ti_sysbios_knl_Swi_disable__E                                             
1001c0e1  ti_sysbios_knl_Swi_enabled__E                                             
00007985  ti_sysbios_knl_Swi_getTrigger__E                                          
000013e8  ti_sysbios_knl_Swi_numPriorities__C                                       
0000773d  ti_sysbios_knl_Swi_or__E                                                  
1001c2e9  ti_sysbios_knl_Swi_postInit__I                                            
1001b31d  ti_sysbios_knl_Swi_post__E                                                
1001ad61  ti_sysbios_knl_Swi_restoreHwi__E                                          
1001b5dd  ti_sysbios_knl_Swi_restore__E                                             
1001b0d5  ti_sysbios_knl_Swi_runLoop__I                                             
1001afd9  ti_sysbios_knl_Swi_run__I                                                 
1001b031  ti_sysbios_knl_Swi_schedule__I                                            
1001c239  ti_sysbios_knl_Swi_startup__E                                             
20002808  ti_sysbios_knl_Task_Instance_State_0_stack__A                             
1001a4f9  ti_sysbios_knl_Task_Instance_finalize__E                                  
1001a259  ti_sysbios_knl_Task_Instance_init__E                                      
200039e8  ti_sysbios_knl_Task_Module_State_0_idleTask__A                            
200038c8  ti_sysbios_knl_Task_Module_State_0_readyQ__A                              
000014ec  ti_sysbios_knl_Task_Module_State_inactiveQ__O                             
200039c4  ti_sysbios_knl_Task_Module__root__V                                       
20000100  ti_sysbios_knl_Task_Module__state__V                                      
1001adbd  ti_sysbios_knl_Task_Module_startup__E                                     
00001310  ti_sysbios_knl_Task_Object__DESC__C                                       
00001000  ti_sysbios_knl_Task_Object__PARAMS__C                                     
000013ec  ti_sysbios_knl_Task_Object__count__C                                      
1001bdc5  ti_sysbios_knl_Task_Object__delete__S                                     
1001bf61  ti_sysbios_knl_Task_Object__destruct__S                                   
1001bde5  ti_sysbios_knl_Task_Object__get__S                                        
000013f0  ti_sysbios_knl_Task_Object__table__C                                      
20003710  ti_sysbios_knl_Task_Object__table__V                                      
1001c1d5  ti_sysbios_knl_Task_Params__init__S                                       
1001c2ed  ti_sysbios_knl_Task_SupportProxy_Module__startupDone__S                   
1001c261  ti_sysbios_knl_Task_SupportProxy_Module__startupDone__S__mangled__        
1001c2f1  ti_sysbios_knl_Task_SupportProxy_getStackAlignment__E                     
1001c15d  ti_sysbios_knl_Task_SupportProxy_getStackAlignment__E__mangled__          
1001c2f5  ti_sysbios_knl_Task_SupportProxy_start__E                                 
1001b499  ti_sysbios_knl_Task_SupportProxy_start__E__mangled__                      
1001c2f9  ti_sysbios_knl_Task_SupportProxy_swap__E                                  
1001ca65  ti_sysbios_knl_Task_SupportProxy_swap__E__mangled__                       
000013f4  ti_sysbios_knl_Task_allBlockedFunc__C                                     
1001b361  ti_sysbios_knl_Task_allBlockedFunction__I                                 
1001b611  ti_sysbios_knl_Task_blockI__E                                             
1001b125  ti_sysbios_knl_Task_construct                                             
1001ae19  ti_sysbios_knl_Task_create                                                
000013f8  ti_sysbios_knl_Task_defaultStackHeap__C                                   
000013fc  ti_sysbios_knl_Task_defaultStackSize__C                                   
1001c2fd  ti_sysbios_knl_Task_delete                                                
1001c301  ti_sysbios_knl_Task_destruct                                              
1001c0f1  ti_sysbios_knl_Task_disable__E                                            
1001c23f  ti_sysbios_knl_Task_enable__E                                             
1001be05  ti_sysbios_knl_Task_enter__I                                              
1001b425  ti_sysbios_knl_Task_exit__E                                               
00001412  ti_sysbios_knl_Task_initStackFlag__C                                      
00001400  ti_sysbios_knl_Task_numConstructedTasks__C                                
1001a611  ti_sysbios_knl_Task_postInit__I                                           
1001b735  ti_sysbios_knl_Task_processVitalTaskFlag__I                               
1001be25  ti_sysbios_knl_Task_restoreHwi__E                                         
1001ba45  ti_sysbios_knl_Task_restore__E                                            
1001b175  ti_sysbios_knl_Task_schedule__I                                           
1001c1e1  ti_sysbios_knl_Task_self__E                                               
1001bf7d  ti_sysbios_knl_Task_sleepTimeout__I                                       
1001a9d9  ti_sysbios_knl_Task_sleep__E                                              
1001ae75  ti_sysbios_knl_Task_startCore__E                                          
1001c305  ti_sysbios_knl_Task_startup__E                                            
1001ca6d  ti_sysbios_knl_Task_swapReturn                                            
1001b9a1  ti_sysbios_knl_Task_unblockI__E                                           
1001bfb1  ti_sysbios_knl_Task_unblock__E                                            
1001b3a5  ti_sysbios_knl_Task_yield__E                                              
00001494  ti_sysbios_rom_ROM_AONRTCChannelEnable                                    
00001498  ti_sysbios_rom_ROM_AONRTCCompareValueSet                                  
0000149c  ti_sysbios_rom_ROM_AONRTCCurrentCompareValueGet                           
000014a0  ti_sysbios_rom_ROM_AONRTCEventClear                                       
000014a4  ti_sysbios_rom_ROM_ti_sysbios_family_arm_cc26xx_Timer_getCount64__E       
000014a8  ti_sysbios_rom_ROM_ti_sysbios_family_arm_cc26xx_Timer_getCurrentTick__E   
000014ac  ti_sysbios_rom_ROM_ti_sysbios_family_arm_cc26xx_Timer_getMaxTicks__E      
000014b0  ti_sysbios_rom_ROM_ti_sysbios_family_arm_cc26xx_Timer_initDevice__I       
000014b4  ti_sysbios_rom_ROM_ti_sysbios_family_arm_cc26xx_Timer_setNextTick__E      
000014b8  ti_sysbios_rom_ROM_ti_sysbios_family_arm_cc26xx_Timer_setThreshold__I     
000014bc  ti_sysbios_rom_ROM_ti_sysbios_family_arm_cc26xx_Timer_start__E            
000014c0  ti_sysbios_rom_ROM_ti_sysbios_family_arm_cc26xx_TimestampProvider_get32__E
000014c4  ti_sysbios_rom_ROM_xdc_runtime_Startup_getState__I                        
000014c8  ti_sysbios_rom_ROM_xdc_runtime_System_SupportProxy_abort__E               
000014cc  ti_sysbios_rom_ROM_xdc_runtime_System_SupportProxy_exit__E                
00007573  ti_sysbios_rom_cortexm_cc13xx_CC13xx_badRomRevision__E                    
00007755  ti_sysbios_rom_cortexm_cc13xx_CC13xx_checkRevision__E                     
1001ca97  ti_sysbios_rom_cortexm_cc13xx_CC13xx_getRevision__E                       
0000034c  uartCC26XXHWAttrs                                                         
20002bfc  uartCC26XXObjects                                                         
20003440  uartCC26XXRingBuffer                                                      
00001428  xdc_runtime_Assert_E_assertFailed__C                                      
1001c5a5  xdc_runtime_Assert_raise__I                                               
1001c6e9  xdc_runtime_Core_assignLabel__I                                           
1001c5ed  xdc_runtime_Core_assignParams__I                                          
1001c635  xdc_runtime_Core_constructObject__I                                       
1001c401  xdc_runtime_Core_createObject__I                                          
1001c4f5  xdc_runtime_Core_deleteObject__I                                          
1001c79d  xdc_runtime_Core_destructObject__I                                        
0000142c  xdc_runtime_Error_E_memory__C                                             
1001c7b5  xdc_runtime_Error_check__E                                                
1001c83d  xdc_runtime_Error_init__E                                                 
00001430  xdc_runtime_Error_policyFxn__C                                            
1001c483  xdc_runtime_Error_policySpin__E                                           
00001490  xdc_runtime_Error_policy__C                                               
1001c765  xdc_runtime_Error_raiseX__E                                               
1001c881  xdc_runtime_Gate_enterSystem__E                                           
1001c875  xdc_runtime_Gate_leaveSystem__E                                           
00001434  xdc_runtime_IGateProvider_Interface__BASE__C                              
00001438  xdc_runtime_IHeap_Interface__BASE__C                                      
0000143c  xdc_runtime_IModule_Interface__BASE__C                                    
1001bbe5  xdc_runtime_Main_Module_GateProxy_Handle__label__S                        
1001bc05  xdc_runtime_Main_Module_GateProxy_Object__delete__S                       
1001c265  xdc_runtime_Main_Module_GateProxy_query__E                                
00001440  xdc_runtime_Main_Module__diagsEnabled__C                                  
00001444  xdc_runtime_Main_Module__diagsIncluded__C                                 
00001448  xdc_runtime_Main_Module__diagsMask__C                                     
00001488  xdc_runtime_Main_Module__id__C                                            
1001bc85  xdc_runtime_Memory_HeapProxy_Handle__label__S                             
1001bc85  xdc_runtime_Memory_HeapProxy_Handle__label__S__mangled__                  
1001bca5  xdc_runtime_Memory_HeapProxy_Object__delete__S                            
1001bca5  xdc_runtime_Memory_HeapProxy_Object__delete__S__mangled__                 
1001c885  xdc_runtime_Memory_HeapProxy_alloc__E                                     
1001c889  xdc_runtime_Memory_HeapProxy_free__E                                      
0000148a  xdc_runtime_Memory_Module__id__C                                          
20000200  xdc_runtime_Memory_Module__state__V                                       
1001c485  xdc_runtime_Memory_alloc__E                                               
1001c849  xdc_runtime_Memory_calloc__E                                              
0000144c  xdc_runtime_Memory_defaultHeapInstance__C                                 
1001c7fd  xdc_runtime_Memory_free__E                                                
1001c855  xdc_runtime_Memory_getMaxDefaultTypeAlign__E                              
1001c781  xdc_runtime_Memory_valloc__E                                              
200039cc  xdc_runtime_Registry_Module__state__V                                     
000073e9  xdc_runtime_Registry_findById__E                                          
200001f0  xdc_runtime_Startup_Module__state__V                                      
00000001  xdc_runtime_Startup__EXECFXN__C                                           
00000001  xdc_runtime_Startup__RESETFXN__C                                          
00001450  xdc_runtime_Startup_execImpl__C                                           
1001c555  xdc_runtime_Startup_exec__E                                               
00007863  xdc_runtime_Startup_exec__I                                               
00000434  xdc_runtime_Startup_firstFxns__A                                          
00001418  xdc_runtime_Startup_firstFxns__C                                          
00006159  xdc_runtime_Startup_getState__I                                           
00001420  xdc_runtime_Startup_lastFxns__C                                           
00001454  xdc_runtime_Startup_maxPasses__C                                          
00007991  xdc_runtime_Startup_reset__I                                              
0000799d  xdc_runtime_Startup_rtsDone__E                                            
000003e4  xdc_runtime_Startup_sfxnRts__A                                            
00001458  xdc_runtime_Startup_sfxnRts__C                                            
000002bc  xdc_runtime_Startup_sfxnTab__A                                            
0000145c  xdc_runtime_Startup_sfxnTab__C                                            
00001460  xdc_runtime_Startup_startModsFxn__C                                       
1001c309  xdc_runtime_Startup_startMods__I                                          
00001464  xdc_runtime_SysCallback_abortFxn__C                                       
1001c80d  xdc_runtime_SysCallback_abort__E                                          
0000792f  xdc_runtime_SysCallback_defaultAbort                                      
00007a25  xdc_runtime_SysCallback_defaultExit                                       
00001468  xdc_runtime_SysCallback_exitFxn__C                                        
1001c81d  xdc_runtime_SysCallback_exit__E                                           
2000312c  xdc_runtime_SysMin_Module_State_0_outbuf__A                               
20003950  xdc_runtime_SysMin_Module__state__V                                       
00007409  xdc_runtime_SysMin_Module_startup__E                                      
00006f3d  xdc_runtime_SysMin_abort__E                                               
00000474  xdc_runtime_SysMin_bufSize__C                                             
000074f1  xdc_runtime_SysMin_exit__E                                                
000000ee  xdc_runtime_SysMin_flushAtExit__C                                         
00006879  xdc_runtime_SysMin_flush__E                                               
00000478  xdc_runtime_SysMin_outputFunc__C                                          
000072e5  xdc_runtime_SysMin_output__I                                              
00006bbd  xdc_runtime_SysMin_putch__E                                               
000078b5  xdc_runtime_SysMin_ready__E                                               
1001bbe5  xdc_runtime_System_Module_GateProxy_Handle__label__S                      
1001bbe5  xdc_runtime_System_Module_GateProxy_Handle__label__S__mangled__           
1001bc05  xdc_runtime_System_Module_GateProxy_Object__delete__S                     
1001bc05  xdc_runtime_System_Module_GateProxy_Object__delete__S__mangled__          
1001c88d  xdc_runtime_System_Module_GateProxy_enter__E                              
1001c891  xdc_runtime_System_Module_GateProxy_leave__E                              
1001c265  xdc_runtime_System_Module_GateProxy_query__E                              
1001c265  xdc_runtime_System_Module_GateProxy_query__E__mangled__                   
200039d4  xdc_runtime_System_Module_State_0_atexitHandlers__A                       
200001f8  xdc_runtime_System_Module__state__V                                       
1001c87b  xdc_runtime_System_Module_startup__E                                      
00006f3d  xdc_runtime_System_SupportProxy_abort__E                                  
000074f1  xdc_runtime_System_SupportProxy_exit__E                                   
00006879  xdc_runtime_System_SupportProxy_flush__E                                  
00006bbd  xdc_runtime_System_SupportProxy_putch__E                                  
000078b5  xdc_runtime_System_SupportProxy_ready__E                                  
0000146c  xdc_runtime_System_abortFxn__C                                            
1001c895  xdc_runtime_System_abortSpin__E                                           
1001c745  xdc_runtime_System_abort__E                                               
1001c67d  xdc_runtime_System_atexit__E                                              
00001dfd  xdc_runtime_System_doPrint__I                                             
00001470  xdc_runtime_System_exitFxn__C                                             
1001c897  xdc_runtime_System_exitSpin__E                                            
1001c7cd  xdc_runtime_System_exit__E                                                
0000047c  xdc_runtime_System_extendFxn__C                                           
00006879  xdc_runtime_System_flush__E                                               
00005b69  xdc_runtime_System_formatNum__I                                           
00001474  xdc_runtime_System_maxAtexitHandlers__C                                   
00004015  xdc_runtime_System_printfExtend__I                                        
00007527  xdc_runtime_System_printf__E                                              
00007a1d  xdc_runtime_System_printf_va__F                                           
1001c6b5  xdc_runtime_System_processAtExit__E                                       
000070d1  xdc_runtime_System_putchar__I                                             
00007541  xdc_runtime_System_snprintf__E                                            
00007a21  xdc_runtime_System_snprintf_va__F                                         
000072c1  xdc_runtime_System_vprintf__E                                             
000078c5  xdc_runtime_System_vsnprintf__E                                           
0000148c  xdc_runtime_Text_charCnt__C                                               
00000487  xdc_runtime_Text_charTab__A                                               
00001478  xdc_runtime_Text_charTab__C                                               
1001c719  xdc_runtime_Text_cordText__E                                              
0000148e  xdc_runtime_Text_isLoaded__C                                              
0000147c  xdc_runtime_Text_nameEmpty__C                                             
00001480  xdc_runtime_Text_nameStatic__C                                            
00001484  xdc_runtime_Text_nameUnknown__C                                           
00006f6d  xdc_runtime_Text_printVisFxn__I                                           
000061b5  xdc_runtime_Text_putLab__E                                                
0000527d  xdc_runtime_Text_putMod__E                                                
00004e4d  xdc_runtime_Text_putSite__E                                               
0000044a  xdc_runtime_Text_registryModsLastId__C                                    
1001c7e5  xdc_runtime_Text_ropeText__E                                              
00000484  xdc_runtime_Text_unnamedModsLastId__C                                     
00000480  xdc_runtime_Text_visitRopeFxn__C                                          
000079df  xdc_runtime_Text_visitRope__I                                             
000068bd  xdc_runtime_Text_xprintf__I                                               
1001c82d  xdc_runtime_Timestamp_SupportProxy_get32__E                               
000078f1  xdc_runtime_Timestamp_SupportProxy_get32__E__mangled__                    
1001b9cd  xdc_runtime_Timestamp_SupportProxy_get64__E                               
1001b9cd  xdc_runtime_Timestamp_SupportProxy_get64__E__mangled__                    
1001c12b  xdc_runtime_Timestamp_SupportProxy_getFreq__E                             
1001c12b  xdc_runtime_Timestamp_SupportProxy_getFreq__E__mangled__                  
1001c82d  xdc_runtime_Timestamp_get32__E                                            
1001c82d  xdc_runtime_Timestamp_get32__E                                            
1001b9cd  xdc_runtime_Timestamp_get64__E                                            
1001b9cd  xdc_runtime_Timestamp_get64__E                                            
1001c12b  xdc_runtime_Timestamp_getFreq__E                                          
1001c12b  xdc_runtime_Timestamp_getFreq__E                                          


GLOBAL SYMBOLS: SORTED BY Symbol Address 

address   name                                                                      
-------   ----                                                                      
00000000  __ASM__                                                                   
00000000  __TI_static_base__                                                        
00000000  ti_sysbios_family_arm_m3_Hwi_resetVectors                                 
00000001  xdc_runtime_Startup__EXECFXN__C                                           
00000001  xdc_runtime_Startup__RESETFXN__C                                          
00000078  __ISA__                                                                   
0000008a  __PLAT__                                                                  
000000b1  __TARG__                                                                  
000000d6  __TRDR__                                                                  
000000ee  xdc_runtime_SysMin_flushAtExit__C                                         
0000015c  BoardGpioInitTable                                                        
000001c0  resourceDB                                                                
00000294  UARTCC26XX_fxnTable                                                       
000002bc  xdc_runtime_Startup_sfxnTab__A                                            
00000300  __STACK_SIZE                                                              
00000308  UART_defaultParams                                                        
0000032c  ti_sysbios_knl_Event_Object__DESC__C                                      
0000034c  uartCC26XXHWAttrs                                                         
0000036c  DisplayUart_fxnTable                                                      
00000388  Display_config                                                            
000003a0  UART_config                                                               
000003b8  ti_sysbios_knl_Event_Object__PARAMS__C                                    
000003d0  displayUartHWAttrs                                                        
000003e4  xdc_runtime_Startup_sfxnRts__A                                            
00000408  PDMCC26XX_I2S_config                                                      
00000418  PowerCC26XX_config                                                        
00000428  pdmC26XXI2SHWAttrs                                                        
00000434  xdc_runtime_Startup_firstFxns__A                                          
0000044a  xdc_runtime_Text_registryModsLastId__C                                    
0000044c  PDMCC26XX_config                                                          
00000454  PINCC26XX_hwAttrs                                                         
0000045c  pdmCC26XXHWAttrs                                                          
00000464  ti_sysbios_knl_Clock_tickPeriod__C                                        
00000468  ti_sysbios_knl_Clock_triggerClock__C                                      
0000046c  ti_sysbios_knl_Event_Instance_State_pendQ__O                              
00000470  ti_sysbios_knl_Idle_funcList__A                                           
00000474  xdc_runtime_SysMin_bufSize__C                                             
00000478  xdc_runtime_SysMin_outputFunc__C                                          
0000047c  xdc_runtime_System_extendFxn__C                                           
00000480  xdc_runtime_Text_visitRopeFxn__C                                          
00000484  xdc_runtime_Text_unnamedModsLastId__C                                     
00000486  Display_defaultParams                                                     
00000487  xdc_runtime_Text_charTab__A                                               
00000684  __TI_Handler_Table_Base                                                   
00000690  __TI_Handler_Table_Limit                                                  
000006c8  __TI_CINIT_Base                                                           
00000728  __TI_CINIT_Limit                                                          
00001000  ti_sysbios_knl_Task_Object__PARAMS__C                                     
0000103c  ti_sysbios_knl_Mailbox_Object__PARAMS__C                                  
00001070  ti_sysbios_family_arm_m3_Hwi_Object__PARAMS__C                            
000010a0  ti_sysbios_hal_Hwi_Object__PARAMS__C                                      
000010cc  ti_sysbios_heaps_HeapMem_Module__FXNS__C                                  
000010f4  ti_sysbios_knl_Swi_Object__PARAMS__C                                      
0000111c  ti_sysbios_gates_GateHwi_Module__FXNS__C                                  
00001140  ti_sysbios_gates_GateMutex_Module__FXNS__C                                
00001164  ti_sysbios_heaps_HeapMem_Object__PARAMS__C                                
00001188  ti_sysbios_knl_Clock_Object__PARAMS__C                                    
000011ac  ti_sysbios_knl_Semaphore_Object__PARAMS__C                                
000011d0  ti_sysbios_family_arm_m3_Hwi_Object__DESC__C                              
000011f0  ti_sysbios_gates_GateHwi_Object__DESC__C                                  
00001210  ti_sysbios_gates_GateMutex_Object__DESC__C                                
00001230  ti_sysbios_hal_Hwi_Object__DESC__C                                        
00001250  ti_sysbios_heaps_HeapMem_Object__DESC__C                                  
00001270  ti_sysbios_knl_Clock_Object__DESC__C                                      
00001290  ti_sysbios_knl_Mailbox_Object__DESC__C                                    
000012b0  ti_sysbios_knl_Queue_Object__DESC__C                                      
000012d0  ti_sysbios_knl_Semaphore_Object__DESC__C                                  
000012f0  ti_sysbios_knl_Swi_Object__DESC__C                                        
00001310  ti_sysbios_knl_Task_Object__DESC__C                                       
00001330  ti_sysbios_gates_GateHwi_Object__PARAMS__C                                
00001348  ti_sysbios_gates_GateMutex_Object__PARAMS__C                              
00001360  ti_sysbios_knl_Queue_Object__PARAMS__C                                    
00001378  ti_sysbios_knl_Idle_funcList__C                                           
00001384  ti_sysbios_family_arm_cc26xx_Timer_startupNeeded__C                       
00001388  ti_sysbios_family_arm_m3_Hwi_E_alreadyDefined__C                          
0000138c  ti_sysbios_family_arm_m3_Hwi_E_hwiLimitExceeded__C                        
00001390  ti_sysbios_family_arm_m3_Hwi_NUM_INTERRUPTS__C                            
00001394  ti_sysbios_family_arm_m3_Hwi_Object__count__C                             
00001398  ti_sysbios_family_arm_m3_Hwi_Object__table__C                             
0000139c  ti_sysbios_family_arm_m3_Hwi_ccr__C                                       
000013a0  ti_sysbios_family_arm_m3_Hwi_excHandlerFunc__C                            
000013a4  ti_sysbios_family_arm_m3_Hwi_nullIsrFunc__C                               
000013a8  ti_sysbios_family_arm_m3_Hwi_numSparseInterrupts__C                       
000013ac  ti_sysbios_family_arm_m3_Hwi_priGroup__C                                  
000013b0  ti_sysbios_family_arm_m3_TaskSupport_stackAlignment__C                    
000013b4  ti_sysbios_heaps_HeapMem_E_memory__C                                      
000013b8  ti_sysbios_heaps_HeapMem_Module__gateObj__C                               
000013bc  ti_sysbios_heaps_HeapMem_Object__count__C                                 
000013c0  ti_sysbios_heaps_HeapMem_Object__table__C                                 
000013c4  ti_sysbios_heaps_HeapMem_reqAlign__C                                      
000013c8  ti_sysbios_knl_Clock_serviceMargin__C                                     
000013cc  ti_sysbios_knl_Mailbox_Object__count__C                                   
000013d0  ti_sysbios_knl_Mailbox_Object__table__C                                   
000013d4  ti_sysbios_knl_Mailbox_maxTypeAlign__C                                    
000013d8  ti_sysbios_knl_Queue_Object__count__C                                     
000013dc  ti_sysbios_knl_Queue_Object__table__C                                     
000013e0  ti_sysbios_knl_Swi_Object__count__C                                       
000013e4  ti_sysbios_knl_Swi_Object__table__C                                       
000013e8  ti_sysbios_knl_Swi_numPriorities__C                                       
000013ec  ti_sysbios_knl_Task_Object__count__C                                      
000013f0  ti_sysbios_knl_Task_Object__table__C                                      
000013f4  ti_sysbios_knl_Task_allBlockedFunc__C                                     
000013f8  ti_sysbios_knl_Task_defaultStackHeap__C                                   
000013fc  ti_sysbios_knl_Task_defaultStackSize__C                                   
00001400  ti_sysbios_knl_Task_numConstructedTasks__C                                
00001406  ti_sysbios_family_arm_cc26xx_Timer_Module__id__C                          
00001408  ti_sysbios_family_arm_cc26xx_TimestampProvider_useClockTimer__C           
0000140a  ti_sysbios_family_arm_m3_Hwi_Module__id__C                                
0000140c  ti_sysbios_gates_GateHwi_Module__id__C                                    
0000140e  ti_sysbios_gates_GateMutex_Module__id__C                                  
00001410  ti_sysbios_heaps_HeapMem_Module__id__C                                    
00001412  ti_sysbios_knl_Task_initStackFlag__C                                      
00001414  ti_sysbios_knl_Clock_tickMode__C                                          
00001418  xdc_runtime_Startup_firstFxns__C                                          
00001420  xdc_runtime_Startup_lastFxns__C                                           
00001428  xdc_runtime_Assert_E_assertFailed__C                                      
0000142c  xdc_runtime_Error_E_memory__C                                             
00001430  xdc_runtime_Error_policyFxn__C                                            
00001434  xdc_runtime_IGateProvider_Interface__BASE__C                              
00001438  xdc_runtime_IHeap_Interface__BASE__C                                      
0000143c  xdc_runtime_IModule_Interface__BASE__C                                    
00001440  xdc_runtime_Main_Module__diagsEnabled__C                                  
00001444  xdc_runtime_Main_Module__diagsIncluded__C                                 
00001448  xdc_runtime_Main_Module__diagsMask__C                                     
0000144c  xdc_runtime_Memory_defaultHeapInstance__C                                 
00001450  xdc_runtime_Startup_execImpl__C                                           
00001454  xdc_runtime_Startup_maxPasses__C                                          
00001458  xdc_runtime_Startup_sfxnRts__C                                            
0000145c  xdc_runtime_Startup_sfxnTab__C                                            
00001460  xdc_runtime_Startup_startModsFxn__C                                       
00001464  xdc_runtime_SysCallback_abortFxn__C                                       
00001468  xdc_runtime_SysCallback_exitFxn__C                                        
0000146c  xdc_runtime_System_abortFxn__C                                            
00001470  xdc_runtime_System_exitFxn__C                                             
00001474  xdc_runtime_System_maxAtexitHandlers__C                                   
00001478  xdc_runtime_Text_charTab__C                                               
0000147c  xdc_runtime_Text_nameEmpty__C                                             
00001480  xdc_runtime_Text_nameStatic__C                                            
00001484  xdc_runtime_Text_nameUnknown__C                                           
00001488  xdc_runtime_Main_Module__id__C                                            
0000148a  xdc_runtime_Memory_Module__id__C                                          
0000148c  xdc_runtime_Text_charCnt__C                                               
0000148e  xdc_runtime_Text_isLoaded__C                                              
00001490  xdc_runtime_Error_policy__C                                               
00001494  ti_sysbios_rom_ROM_AONRTCChannelEnable                                    
00001498  ti_sysbios_rom_ROM_AONRTCCompareValueSet                                  
0000149c  ti_sysbios_rom_ROM_AONRTCCurrentCompareValueGet                           
000014a0  ti_sysbios_rom_ROM_AONRTCEventClear                                       
000014a4  ti_sysbios_rom_ROM_ti_sysbios_family_arm_cc26xx_Timer_getCount64__E       
000014a8  ti_sysbios_rom_ROM_ti_sysbios_family_arm_cc26xx_Timer_getCurrentTick__E   
000014ac  ti_sysbios_rom_ROM_ti_sysbios_family_arm_cc26xx_Timer_getMaxTicks__E      
000014b0  ti_sysbios_rom_ROM_ti_sysbios_family_arm_cc26xx_Timer_initDevice__I       
000014b4  ti_sysbios_rom_ROM_ti_sysbios_family_arm_cc26xx_Timer_setNextTick__E      
000014b8  ti_sysbios_rom_ROM_ti_sysbios_family_arm_cc26xx_Timer_setThreshold__I     
000014bc  ti_sysbios_rom_ROM_ti_sysbios_family_arm_cc26xx_Timer_start__E            
000014c0  ti_sysbios_rom_ROM_ti_sysbios_family_arm_cc26xx_TimestampProvider_get32__E
000014c4  ti_sysbios_rom_ROM_xdc_runtime_Startup_getState__I                        
000014c8  ti_sysbios_rom_ROM_xdc_runtime_System_SupportProxy_abort__E               
000014cc  ti_sysbios_rom_ROM_xdc_runtime_System_SupportProxy_exit__E                
000014d0  ti_sysbios_gates_GateMutex_Instance_State_sem__O                          
000014d4  ti_sysbios_knl_Clock_Module_State_clockQ__O                               
000014d8  ti_sysbios_knl_Mailbox_Instance_State_dataQue__O                          
000014dc  ti_sysbios_knl_Mailbox_Instance_State_dataSem__O                          
000014e0  ti_sysbios_knl_Mailbox_Instance_State_freeQue__O                          
000014e4  ti_sysbios_knl_Mailbox_Instance_State_freeSem__O                          
000014e8  ti_sysbios_knl_Semaphore_Instance_State_pendQ__O                          
000014ec  ti_sysbios_knl_Task_Module_State_inactiveQ__O                             
000014f1  pdm2pcm16k                                                                
00001dfd  xdc_runtime_System_doPrint__I                                             
00002699  taskFxn                                                                   
00002909  main                                                                      
00002b49  NOROM_SysCtrlSetRechargeBeforePowerDown                                   
00002d71  Power_sleep                                                               
00003185  PIN_init                                                                  
00003349  PDMCC26XX_I2S_open                                                        
00003509  PowerCC26XX_doCalibrate                                                   
000036a9  UARTCC26XX_open                                                           
00003849  PDMCC26XX_open                                                            
0000398d  NOROM_SetupAfterColdResetWakeupFromShutDownCfg3                           
00003abd  Power_init                                                                
00003be9  UARTCC26XX_read                                                           
00003d05  UARTCC26XX_hwiIntFxn                                                      
00003e15  PDMCC26XX_I2S_startStream                                                 
00003f19  UARTCC26XX_write                                                          
00004015  xdc_runtime_System_printfExtend__I                                        
0000410d  NOROM_SetupAfterColdResetWakeupFromShutDownCfg2                           
000041fd  ti_sysbios_knl_Event_pend__E                                              
000043c5  NOROM_I2SChannelConfigure                                                 
00004575  PowerCC26XX_standbyPolicy                                                 
00004649  Power_releaseDependency                                                   
0000471d  Power_setDependency                                                       
000048b7  DisplayUart_clear                                                         
00004b05  PDMCC26XX_startStream                                                     
00004bb5  Codec1_encodeSingle                                                       
00004c61  NOROM_SetupTrimDevice                                                     
00004c61  ti_sysbios_family_arm_cc26xx_Boot_trimDevice                              
00004d09  NOROM_SetupAfterColdResetWakeupFromShutDownCfg1                           
00004dad  __TI_auto_init                                                            
00004e4d  xdc_runtime_Text_putSite__E                                               
00004eeb  DisplayUart_clearLines                                                    
00004f89  __aeabi_memcpy                                                            
00004f89  __aeabi_memcpy4                                                           
00004f89  __aeabi_memcpy8                                                           
00004f89  memcpy                                                                    
00005025  ti_sysbios_knl_Clock_workFuncDynamic__E                                   
000050bd  __aeabi_uldivmod                                                          
00005153  _nop                                                                      
00005155  PIN_open                                                                  
0000527d  xdc_runtime_Text_putMod__E                                                
0000542d  UARTCC26XX_writeCancel                                                    
000055cd  PDMCC26XX_I2S_stopStream                                                  
000056d1  PDMCC26XX_I2S_close                                                       
0000574d  __aeabi_memclr                                                            
0000574d  __aeabi_memclr4                                                           
0000574d  __aeabi_memclr8                                                           
0000574f  __aeabi_memset                                                            
0000574f  __aeabi_memset4                                                           
0000574f  __aeabi_memset8                                                           
00005755  memset                                                                    
000057c9  Codec1_encodeBuff                                                         
00005841  UARTCC26XX_close                                                          
000058b9  NOROM_SetupSetVddrLevel                                                   
0000592d  PowerCC26XX_auxISR                                                        
000059a1  ti_sysbios_family_arm_cc26xx_Timer_start__E                               
00005a89  NOROM_ChipInfo_GetHwRevision                                              
00005af9  ti_sysbios_knl_Event_post__E                                              
00005b69  xdc_runtime_System_formatNum__I                                           
00005bd7  __aeabi_idiv0                                                             
00005bd7  __aeabi_ldiv0                                                             
00005bd9  NOROM_SetupGetTrimForAmpcompCtrl                                          
00005c45  PowerCC26XX_calibrate                                                     
00005cb1  UARTCC26XX_readCancel                                                     
00005d1d  NOROM_SetupGetTrimForAnabypassValue1                                      
00005d85  NOROM_SysCtrl_DCDC_VoltageConditionalControl                              
00005ded  __TI_decompress_lzss                                                      
00005e55  NOROM_OSCHF_AttemptToSwitchToXosc                                         
00005eb9  PDMCC26XX_init                                                            
00005f1d  UARTCC26XX_control                                                        
00005f81  NOROM_OSCClockSourceSet                                                   
00005fe1  PowerCC26XX_RCOSC_clockFunc                                               
000060a1  NOROM_SysCtrlAdjustRechargeAfterPowerDown                                 
000060fd  PIN_remove                                                                
00006159  xdc_runtime_Startup_getState__I                                           
000061b5  xdc_runtime_Text_putLab__E                                                
00006211  DisplayUart_put5                                                          
00006269  HOSTwrite                                                                 
00006319  PowerCC26XX_initiateCalibration                                           
00006371  buttonCallbackFxn                                                         
000063c9  PDMCC26XX_stopStream                                                      
00006471  NOROM_SetupSetCacheModeAccordingToCcfgSetting                             
000064c1  PDMCC26XX_I2S_requestBuffer                                               
00006511  DisplayUart_open                                                          
000065a9  copy_in                                                                   
00006641  Display_doOpen                                                            
00006689  NOROM_ChipInfo_GetChipFamily                                              
000066d1  PIN_setOutputEnable                                                       
000067a9  RingBuf_put                                                               
000067ef  ti_sysbios_BIOS_linkedWithIncorrectBootLibrary__E                         
000067f1  PDMCC26XX_requestBuffer                                                   
00006835  ResetISR                                                                  
00006835  _c_int00                                                                  
00006879  xdc_runtime_SysMin_flush__E                                               
00006879  xdc_runtime_System_SupportProxy_flush__E                                  
00006879  xdc_runtime_System_flush__E                                               
000068bd  xdc_runtime_Text_xprintf__I                                               
00006901  RingBuf_get                                                               
00006941  __aeabi_uidiv                                                             
00006941  __aeabi_uidivmod                                                          
00006981  NOROM_OSC_HPOSCRelativeFrequencyOffsetGet                                 
000069bd  PIN_setOutputValue                                                        
000069f9  UARTCC26XX_swiIntFxn                                                      
00006a6d  PIN_setInterrupt                                                          
00006add  __TI_writemsg                                                             
00006b0b  C$$IO$$                                                                   
00006b4d  ti_sysbios_family_arm_cc26xx_Timer_getCurrentTick__E                      
00006bbd  xdc_runtime_SysMin_putch__E                                               
00006bbd  xdc_runtime_System_SupportProxy_putch__E                                  
00006bf5  NOROM_OSCHF_SwitchToRcOscTurnOffXosc                                      
00006c29  PIN_setConfig                                                             
00006c5d  __TI_readmsg                                                              
00006cc5  ti_sysbios_family_arm_cc26xx_Timer_initDevice__I                          
00006d2b  ti_sysbios_family_arm_cc26xx_Timer_setNextTick__E                         
00006d5d  NOROM_I2SSampleStampConfigure                                             
00006d8d  NOROM_PRCMAudioClockConfigSetOverride                                     
00006dbd  NOROM_SetupSetAonRtcSubSecInc                                             
00006e1d  Power_releaseConstraint                                                   
00006e4d  Power_setConstraint                                                       
00006e7d  UART_open                                                                 
00006ead  ti_sysbios_BIOS_atExitFunc__I                                             
00006edd  ti_sysbios_BIOS_startFunc__I                                              
00006f0d  ti_sysbios_family_arm_cc26xx_Timer_setThreshold__I                        
00006f3d  xdc_runtime_SysMin_abort__E                                               
00006f3d  xdc_runtime_System_SupportProxy_abort__E                                  
00006f6d  xdc_runtime_Text_printVisFxn__I                                           
00006f9d  NOROM_DDI32RegWrite                                                       
00006fc9  NOROM_OSCClockSourceGet                                                   
00006ff5  NOROM_SetupGetTrimForRadcExtCfg                                           
00007021  PINCC26XX_setMux                                                          
0000704d  ti_sysbios_knl_Clock_getTicksUntilInterrupt__E                            
00007079  ti_sysbios_knl_Event_construct                                            
000070a5  ti_sysbios_knl_Event_pendTimeout__I                                       
000070d1  xdc_runtime_System_putchar__I                                             
000070fb  ti_sysbios_BIOS_nullFunc__I                                               
000070fd  NOROM_AONBatMonTemperatureGetDegC                                         
00007125  NOROM_I2SEnable                                                           
0000714d  Power_registerNotify                                                      
00007175  SafeHapiVoid                                                              
0000719d  Display_doPut5                                                            
000071c3  List_put                                                                  
000071e9  PINCC26XX_getPinCount                                                     
00007255  ti_sysbios_BIOS_registerRTSLock__I                                        
00007279  ti_sysbios_BIOS_removeRTSLock__I                                          
0000729d  ti_sysbios_family_arm_cc26xx_Timer_getMaxTicks__E                         
000072c1  xdc_runtime_System_vprintf__E                                             
000072e5  xdc_runtime_SysMin_output__I                                              
00007307  ti_sysbios_knl_Clock_triggerFunc__I                                       
00007309  NOROM_I2SAudioFormatConfigure                                             
00007329  NOROM_SetupGetTrimForXoscHfCtl                                            
00007349  Power_unregisterNotify                                                    
00007369  ti_sysbios_BIOS_rtsLock__I                                                
00007389  ti_sysbios_family_arm_cc26xx_Timer_dynamicStub__E                         
000073a9  ti_sysbios_knl_Clock_stop__E                                              
000073c9  ti_sysbios_knl_Event_checkEvents__I                                       
000073e9  xdc_runtime_Registry_findById__E                                          
00007409  xdc_runtime_SysMin_Module_startup__E                                      
00007429  PIN_close                                                                 
00007447  Power_getTransitionLatency                                                
00007465  NOROM_SetupGetTrimForAmpcompTh2                                           
00007481  NOROM_SetupGetTrimForRcOscLfRtuneCtuneTrim                                
000074d5  ti_sysbios_family_arm_m3_Hwi_clearInterrupt__E                            
000074d5  ti_sysbios_hal_Hwi_HwiProxy_clearInterrupt__E                             
000074d5  ti_sysbios_hal_Hwi_clearInterrupt__E                                      
000074f1  xdc_runtime_SysMin_exit__E                                                
000074f1  xdc_runtime_System_SupportProxy_exit__E                                   
0000750d  List_remove                                                               
00007527  xdc_runtime_System_printf__E                                              
00007541  xdc_runtime_System_snprintf__E                                            
0000755b  DisplayUart_close                                                         
00007573  ti_sysbios_rom_cortexm_cc13xx_CC13xx_badRomRevision__E                    
00007575  NOROM_AONRTCCurrentCompareValueGet                                        
0000758d  NOROM_ChipInfo_GetPackageType                                             
000075a5  NOROM_I2SBufferConfig                                                     
000075bd  NOROM_OSCHF_TurnOnXosc                                                    
000075d5  NOROM_SetupGetTrimForAdcShModeEn                                          
000075ed  NOROM_SetupGetTrimForAdcShVbufEn                                          
00007605  NOROM_SetupGetTrimForAmpcompTh1                                           
0000761d  NOROM_SetupGetTrimForDblrLoopFilterResetVoltage                           
00007635  NOROM_SetupGetTrimForRcOscLfIBiasTrim                                     
0000764d  NOROM_SetupGetTrimForXoscLfRegulatorAndCmirrwrRatio                       
00007665  PDMCC26XX_I2S_init                                                        
00007695  Power_idleFunc                                                            
000076ad  UARTCC26XX_init                                                           
000076c5  UART_Params_init                                                          
000076dd  _args_main                                                                
0000770d  __aeabi_lmul                                                              
00007725  ti_sysbios_BIOS_rtsUnlock__I                                              
0000773d  ti_sysbios_knl_Swi_or__E                                                  
00007755  ti_sysbios_rom_cortexm_cc13xx_CC13xx_checkRevision__E                     
0000776d  NOROM_ThisCodeIsBuiltForCC13xxHwRev20AndLater_HaltIfViolated              
00007783  ti_sysbios_BIOS_exitFunc__I                                               
000077c5  NOROM_AONRTCCurrent64BitValueGet                                          
000077d9  NOROM_I2SPointerSet                                                       
000077ed  PDMCC26XX_I2S_releaseBuffer                                               
00007801  PIN_getInputValue                                                         
00007815  strlen                                                                    
00007829  ti_sysbios_knl_Clock_doTick__I                                            
0000783d  ti_sysbios_knl_Event_Instance_init__E                                     
00007851  RingBuf_construct                                                         
00007863  xdc_runtime_Startup_exec__I                                               
00007875  NOROM_SetupGetTrimForXoscHfFastStart                                      
00007885  NOROM_SetupGetTrimForXoscHfIbiastherm                                     
00007895  PDMCC26XX_close                                                           
000078b5  xdc_runtime_SysMin_ready__E                                               
000078b5  xdc_runtime_System_SupportProxy_ready__E                                  
000078c5  xdc_runtime_System_vsnprintf__E                                           
000078d5  NOROM_VIMSModeGet                                                         
000078e3  __TI_decompress_none                                                      
000078f1  ti_sysbios_family_arm_cc26xx_TimestampProvider_get32__E                   
000078f1  xdc_runtime_Timestamp_SupportProxy_get32__E__mangled__                    
000078ff  Display_doClear                                                           
0000790b  NOROM_CPUcpsid                                                            
00007917  NOROM_CPUcpsie                                                            
00007923  PIN_registerIntCb                                                         
0000792f  xdc_runtime_SysCallback_defaultAbort                                      
00007931  Power_getConstraintMask                                                   
0000793d  Power_getDependencyCount                                                  
00007949  _register_lock                                                            
00007955  _register_unlock                                                          
00007961  __TI_zero_init                                                            
0000796d  ti_sysbios_knl_Event_Params__init__S                                      
00007985  ti_sysbios_knl_Swi_getTrigger__E                                          
00007991  xdc_runtime_Startup_reset__I                                              
0000799d  xdc_runtime_Startup_rtsDone__E                                            
000079a9  List_empty                                                                
000079b3  UART_close                                                                
000079bd  UART_write                                                                
000079df  xdc_runtime_Text_visitRope__I                                             
000079e7  DisplayUart_control                                                       
000079ed  DisplayUart_getType                                                       
000079f3  Display_doParamsInit                                                      
000079f9  UARTCC26XX_readPolling                                                    
000079ff  UARTCC26XX_writePolling                                                   
00007a05  HwiP_disable                                                              
00007a09  List_head                                                                 
00007a0d  List_next                                                                 
00007a15  ti_sysbios_family_arm_cc26xx_Timer_getCount64__E                          
00007a19  ti_sysbios_knl_Semaphore_getCount__E                                      
00007a1d  xdc_runtime_System_printf_va__F                                           
00007a21  xdc_runtime_System_snprintf_va__F                                         
00007a25  xdc_runtime_SysCallback_defaultExit                                       
0001ffa8  __ccfg                                                                    
1001a001  ti_sysbios_knl_Semaphore_pend__E                                          
1001a0cd  ti_sysbios_knl_Mailbox_Instance_init__E                                   
1001a195  ti_sysbios_heaps_HeapMem_alloc__E                                         
1001a259  ti_sysbios_knl_Task_Instance_init__E                                      
1001a315  ti_sysbios_family_arm_m3_Hwi_postInit__I                                  
1001a3c5  ti_sysbios_family_arm_m3_Hwi_Instance_init__E                             
1001a465  ti_sysbios_family_arm_cc26xx_Timer_periodicStub__E                        
1001a4f9  ti_sysbios_knl_Task_Instance_finalize__E                                  
1001a58d  ti_sysbios_knl_Mailbox_post__E                                            
1001a611  ti_sysbios_knl_Task_postInit__I                                           
1001a695  ti_sysbios_family_arm_m3_Hwi_initNVIC__E                                  
1001a715  ti_sysbios_knl_Clock_startI__E                                            
1001a791  ti_sysbios_heaps_HeapMem_free__E                                          
1001a809  ti_sysbios_knl_Clock_walkQueueDynamic__E                                  
1001a881  ti_sysbios_knl_Clock_workFunc__E                                          
1001a8f9  ti_sysbios_knl_Mailbox_Instance_finalize__E                               
1001a969  ti_sysbios_knl_Mailbox_pend__E                                            
1001a9d9  ti_sysbios_knl_Task_sleep__E                                              
1001aa49  ti_sysbios_family_arm_m3_Hwi_dispatchC__I                                 
1001aab1  ti_sysbios_family_arm_m3_Hwi_Object__create__S                            
1001ab15  ti_sysbios_family_arm_m3_Hwi_create                                       
1001ab79  ti_sysbios_hal_Hwi_create                                                 
1001abdd  ti_sysbios_knl_Mailbox_create                                             
1001ac41  ti_sysbios_knl_Semaphore_post__E                                          
1001aca5  ti_sysbios_knl_Swi_Instance_init__E                                       
1001ad05  ti_sysbios_knl_Swi_create                                                 
1001ad61  ti_sysbios_knl_Swi_restoreHwi__E                                          
1001adbd  ti_sysbios_knl_Task_Module_startup__E                                     
1001ae19  ti_sysbios_knl_Task_create                                                
1001ae75  ti_sysbios_knl_Task_startCore__E                                          
1001aed1  ti_sysbios_family_arm_m3_Hwi_Instance_finalize__E                         
1001af29  ti_sysbios_family_arm_m3_Hwi_construct                                    
1001af81  ti_sysbios_knl_Mailbox_construct                                          
1001afd9  ti_sysbios_knl_Swi_run__I                                                 
1001b031  ti_sysbios_knl_Swi_schedule__I                                            
1001b085  ti_sysbios_knl_Swi_construct                                              
1001b0d5  ti_sysbios_knl_Swi_runLoop__I                                             
1001b125  ti_sysbios_knl_Task_construct                                             
1001b175  ti_sysbios_knl_Task_schedule__I                                           
1001b1c1  ti_sysbios_family_arm_m3_Hwi_Module_startup__E                            
1001b209  ti_sysbios_heaps_HeapMem_getStats__E                                      
1001b251  ti_sysbios_family_arm_m3_Hwi_disableInterrupt__E                          
1001b251  ti_sysbios_hal_Hwi_HwiProxy_disableInterrupt__E__mangled__                
1001b295  ti_sysbios_family_arm_m3_Hwi_enableInterrupt__E                           
1001b295  ti_sysbios_hal_Hwi_HwiProxy_enableInterrupt__E__mangled__                 
1001b2d9  ti_sysbios_knl_Mailbox_Module_startup__E                                  
1001b31d  ti_sysbios_knl_Swi_post__E                                                
1001b361  ti_sysbios_knl_Task_allBlockedFunction__I                                 
1001b3a5  ti_sysbios_knl_Task_yield__E                                              
1001b3e9  ti_sysbios_knl_Clock_create                                               
1001b425  ti_sysbios_knl_Task_exit__E                                               
1001b45f  ti_sysbios_gates_GateHwi_Instance_init__E                                 
1001b461  ti_sysbios_family_arm_m3_Hwi_getStackInfo__E                              
1001b461  ti_sysbios_hal_Hwi_HwiProxy_getStackInfo__E__mangled__                    
1001b499  ti_sysbios_family_arm_m3_TaskSupport_start__E                             
1001b499  ti_sysbios_knl_Task_SupportProxy_start__E__mangled__                      
1001b4d1  ti_sysbios_heaps_HeapMem_Instance_init__E                                 
1001b509  ti_sysbios_knl_Clock_Instance_init__E                                     
1001b541  ti_sysbios_heaps_HeapMem_init__I                                          
1001b575  ti_sysbios_knl_Clock_construct                                            
1001b5a9  ti_sysbios_knl_Semaphore_create                                           
1001b5dd  ti_sysbios_knl_Swi_restore__E                                             
1001b611  ti_sysbios_knl_Task_blockI__E                                             
1001b645  ti_sysbios_gates_GateMutex_Object__create__S                              
1001b675  ti_sysbios_gates_GateMutex_create                                         
1001b6a5  ti_sysbios_gates_GateMutex_enter__E                                       
1001b6d5  ti_sysbios_knl_Clock_getTicks__E                                          
1001b705  ti_sysbios_knl_Semaphore_construct                                        
1001b735  ti_sysbios_knl_Task_processVitalTaskFlag__I                               
1001b765  ti_sysbios_family_arm_cc26xx_Timer_postInit__I                            
1001b791  ti_sysbios_family_arm_cc26xx_Timer_startup__E                             
1001b791  ti_sysbios_knl_Clock_TimerProxy_startup__E                                
1001b791  ti_sysbios_knl_Clock_TimerProxy_startup__E__mangled__                     
1001b7bd  ti_sysbios_family_arm_m3_Hwi_Object__get__S                               
1001b7e9  ti_sysbios_gates_GateMutex_construct                                      
1001b815  ti_sysbios_hal_Hwi_initStack                                              
1001b841  ti_sysbios_heaps_HeapMem_Object__create__S                                
1001b86d  ti_sysbios_heaps_HeapMem_Object__get__S                                   
1001b899  ti_sysbios_knl_Mailbox_Object__get__S                                     
1001b8c5  ti_sysbios_knl_Mailbox_postInit__I                                        
1001b8f1  ti_sysbios_knl_Queue_construct                                            
1001b91d  ti_sysbios_knl_Queue_create                                               
1001b949  ti_sysbios_knl_Semaphore_pendTimeout__I                                   
1001b975  ti_sysbios_knl_Swi_Object__get__S                                         
1001b9a1  ti_sysbios_knl_Task_unblockI__E                                           
1001b9cd  ti_sysbios_family_arm_cc26xx_TimestampProvider_get64__E                   
1001b9cd  xdc_runtime_Timestamp_SupportProxy_get64__E                               
1001b9cd  xdc_runtime_Timestamp_SupportProxy_get64__E__mangled__                    
1001b9cd  xdc_runtime_Timestamp_get64__E                                            
1001b9cd  xdc_runtime_Timestamp_get64__E                                            
1001b9f5  ti_sysbios_hal_Hwi_Instance_init__E                                       
1001ba1d  ti_sysbios_knl_Clock_addI__E                                              
1001ba45  ti_sysbios_knl_Task_restore__E                                            
1001ba6d  ti_sysbios_family_arm_cc26xx_Timer_Module_startup__E                      
1001ba91  ti_sysbios_gates_GateHwi_Object__create__S                                
1001bab5  ti_sysbios_BIOS_RtsGateProxy_Object__delete__S                            
1001bab5  ti_sysbios_BIOS_RtsGateProxy_Object__delete__S__mangled__                 
1001bab5  ti_sysbios_gates_GateMutex_Object__delete__S                              
1001bab5  ti_sysbios_heaps_HeapMem_Module_GateProxy_Object__delete__S               
1001bab5  ti_sysbios_heaps_HeapMem_Module_GateProxy_Object__delete__S__mangled__    
1001bad9  ti_sysbios_knl_Clock_Object__delete__S                                    
1001bafd  ti_sysbios_knl_Semaphore_Instance_init__E                                 
1001bb21  ti_sysbios_knl_Semaphore_Object__delete__S                                
1001bb45  ti_sysbios_family_arm_cc26xx_Timer_Module__startupDone__S                 
1001bb45  ti_sysbios_knl_Clock_TimerProxy_Module__startupDone__S__mangled__         
1001bb65  ti_sysbios_family_arm_cc26xx_TimestampProvider_Module_startup__E          
1001bb85  ti_sysbios_family_arm_m3_Hwi_Module__startupDone__S                       
1001bb85  ti_sysbios_hal_Hwi_HwiProxy_Module__startupDone__S__mangled__             
1001bba5  ti_sysbios_family_arm_m3_Hwi_Object__delete__S                            
1001bba5  ti_sysbios_hal_Hwi_HwiProxy_Object__delete__S                             
1001bba5  ti_sysbios_hal_Hwi_HwiProxy_Object__delete__S__mangled__                  
1001bbc5  ti_sysbios_family_arm_m3_Hwi_excHandler__I                                
1001bbe5  ti_sysbios_gates_GateHwi_Handle__label__S                                 
1001bbe5  xdc_runtime_Main_Module_GateProxy_Handle__label__S                        
1001bbe5  xdc_runtime_System_Module_GateProxy_Handle__label__S                      
1001bbe5  xdc_runtime_System_Module_GateProxy_Handle__label__S__mangled__           
1001bc05  ti_sysbios_gates_GateHwi_Object__delete__S                                
1001bc05  xdc_runtime_Main_Module_GateProxy_Object__delete__S                       
1001bc05  xdc_runtime_System_Module_GateProxy_Object__delete__S                     
1001bc05  xdc_runtime_System_Module_GateProxy_Object__delete__S__mangled__          
1001bc25  ti_sysbios_BIOS_RtsGateProxy_Handle__label__S                             
1001bc25  ti_sysbios_BIOS_RtsGateProxy_Handle__label__S__mangled__                  
1001bc25  ti_sysbios_gates_GateMutex_Handle__label__S                               
1001bc25  ti_sysbios_heaps_HeapMem_Module_GateProxy_Handle__label__S                
1001bc25  ti_sysbios_heaps_HeapMem_Module_GateProxy_Handle__label__S__mangled__     
1001bc45  ti_sysbios_gates_GateMutex_Object__destruct__S                            
1001bc65  ti_sysbios_hal_Hwi_Object__delete__S                                      
1001bc85  ti_sysbios_heaps_HeapMem_Handle__label__S                                 
1001bc85  xdc_runtime_Memory_HeapProxy_Handle__label__S                             
1001bc85  xdc_runtime_Memory_HeapProxy_Handle__label__S__mangled__                  
1001bca5  ti_sysbios_heaps_HeapMem_Object__delete__S                                
1001bca5  xdc_runtime_Memory_HeapProxy_Object__delete__S                            
1001bca5  xdc_runtime_Memory_HeapProxy_Object__delete__S__mangled__                 
1001bcc5  ti_sysbios_knl_Clock_Module_startup__E                                    
1001bce5  ti_sysbios_knl_Clock_Object__destruct__S                                  
1001bd05  ti_sysbios_knl_Idle_run__E                                                
1001bd25  ti_sysbios_knl_Mailbox_Object__delete__S                                  
1001bd45  ti_sysbios_knl_Queue_Object__delete__S                                    
1001bd65  ti_sysbios_knl_Queue_Object__get__S                                       
1001bd85  ti_sysbios_knl_Semaphore_Object__destruct__S                              
1001bda5  ti_sysbios_knl_Swi_Object__delete__S                                      
1001bdc5  ti_sysbios_knl_Task_Object__delete__S                                     
1001bde5  ti_sysbios_knl_Task_Object__get__S                                        
1001be05  ti_sysbios_knl_Task_enter__I                                              
1001be25  ti_sysbios_knl_Task_restoreHwi__E                                         
1001be45  ti_sysbios_hal_Hwi_HwiProxy_create                                        
1001be63  ti_sysbios_knl_Clock_logTick__E                                           
1001be65  ti_sysbios_family_arm_m3_Hwi_Object__destruct__S                          
1001be81  ti_sysbios_family_arm_m3_Hwi_setPriority__E                               
1001be9d  ti_sysbios_gates_GateMutex_Instance_init__E                               
1001beb9  ti_sysbios_knl_Clock_scheduleNextTick__E                                  
1001bed5  ti_sysbios_knl_Mailbox_Object__destruct__S                                
1001bef1  ti_sysbios_knl_Queue_Object__destruct__S                                  
1001bf0d  ti_sysbios_knl_Queue_get__E                                               
1001bf29  ti_sysbios_knl_Queue_put__E                                               
1001bf45  ti_sysbios_knl_Swi_Object__destruct__S                                    
1001bf61  ti_sysbios_knl_Task_Object__destruct__S                                   
1001bf7d  ti_sysbios_knl_Task_sleepTimeout__I                                       
1001bf97  ti_sysbios_knl_Swi_Instance_finalize__E                                   
1001bf99  ti_sysbios_gates_GateMutex_leave__E                                       
1001bfb1  ti_sysbios_knl_Task_unblock__E                                            
1001bfc9  ti_sysbios_knl_Clock_Instance_finalize__E                                 
1001bfdf  ti_sysbios_knl_Clock_start__E                                             
1001bff5  ti_sysbios_BIOS_getCpuFreq__E                                             
1001c009  ti_sysbios_family_arm_m3_Hwi_switchFromBootStack__E                       
1001c009  ti_sysbios_hal_Hwi_HwiProxy_switchFromBootStack__E__mangled__             
1001c01d  ti_sysbios_hal_Hwi_Module_startup__E                                      
1001c031  ti_sysbios_BIOS_exit__E                                                   
1001c041  ti_sysbios_BIOS_setThreadType__E                                          
1001c051  ti_sysbios_BIOS_start__E                                                  
1001c061  ti_sysbios_family_arm_m3_Hwi_plug__E                                      
1001c071  ti_sysbios_gates_GateMutex_Instance_finalize__E                           
1001c081  ti_sysbios_hal_Hwi_HwiProxy_Object__create__S                             
1001c091  ti_sysbios_knl_Clock_TimerProxy_getCurrentTick__E                         
1001c0a1  ti_sysbios_knl_Clock_TimerProxy_getMaxTicks__E                            
1001c0b1  ti_sysbios_knl_Clock_TimerProxy_setNextTick__E                            
1001c0c1  ti_sysbios_knl_Semaphore_Instance_finalize__E                             
1001c0d1  ti_sysbios_knl_Swi_disable__E                                             
1001c0e1  ti_sysbios_knl_Swi_enabled__E                                             
1001c0f1  ti_sysbios_knl_Task_disable__E                                            
1001c101  ti_sysbios_heaps_HeapMem_restore__E                                       
1001c10f  ti_sysbios_knl_Queue_empty__E                                             
1001c11d  ti_sysbios_knl_Queue_remove__E                                            
1001c12b  ti_sysbios_family_arm_cc26xx_TimestampProvider_getFreq__E                 
1001c12b  xdc_runtime_Timestamp_SupportProxy_getFreq__E                             
1001c12b  xdc_runtime_Timestamp_SupportProxy_getFreq__E__mangled__                  
1001c12b  xdc_runtime_Timestamp_getFreq__E                                          
1001c12b  xdc_runtime_Timestamp_getFreq__E                                          
1001c139  ti_sysbios_family_arm_m3_Hwi_Params__init__S                              
1001c139  ti_sysbios_hal_Hwi_HwiProxy_Params__init__S                               
1001c139  ti_sysbios_hal_Hwi_HwiProxy_Params__init__S__mangled__                    
1001c145  ti_sysbios_family_arm_m3_Hwi_disableFxn__E                                
1001c151  ti_sysbios_family_arm_m3_Hwi_enableFxn__E                                 
1001c15d  ti_sysbios_family_arm_m3_TaskSupport_getStackAlignment__E                 
1001c15d  ti_sysbios_knl_Task_SupportProxy_getStackAlignment__E__mangled__          
1001c169  ti_sysbios_gates_GateHwi_enter__E                                         
1001c175  ti_sysbios_BIOS_RtsGateProxy_Params__init__S                              
1001c175  ti_sysbios_BIOS_RtsGateProxy_Params__init__S__mangled__                   
1001c175  ti_sysbios_gates_GateMutex_Params__init__S                                
1001c175  ti_sysbios_heaps_HeapMem_Module_GateProxy_Params__init__S                 
1001c175  ti_sysbios_heaps_HeapMem_Module_GateProxy_Params__init__S__mangled__      
1001c181  ti_sysbios_knl_Clock_Params__init__S                                      
1001c18d  ti_sysbios_knl_Clock_getTimerHandle__E                                    
1001c199  ti_sysbios_knl_Mailbox_Params__init__S                                    
1001c1a5  ti_sysbios_knl_Queue_dequeue__E                                           
1001c1b1  ti_sysbios_knl_Queue_enqueue__E                                           
1001c1bd  ti_sysbios_knl_Semaphore_Params__init__S                                  
1001c1c9  ti_sysbios_knl_Swi_Params__init__S                                        
1001c1d5  ti_sysbios_knl_Task_Params__init__S                                       
1001c1e1  ti_sysbios_knl_Task_self__E                                               
1001c1ed  ti_sysbios_hal_Hwi_Instance_finalize__E                                   
1001c1f7  ti_sysbios_family_arm_m3_Hwi_doSwiRestore__I                              
1001c1ff  ti_sysbios_family_arm_m3_Hwi_startup__E                                   
1001c1ff  ti_sysbios_hal_Hwi_HwiProxy_startup__E__mangled__                         
1001c207  ti_sysbios_knl_Idle_loop__E                                               
1001c20f  ti_sysbios_family_arm_m3_Hwi_doTaskRestore__I                             
1001c215  HwiP_restore                                                              
1001c215  ti_sysbios_family_arm_m3_Hwi_restoreFxn__E                                
1001c21b  ti_sysbios_gates_GateHwi_leave__E                                         
1001c227  ti_sysbios_knl_Queue_Instance_init__E                                     
1001c22d  ti_sysbios_knl_Queue_elemClear__E                                         
1001c233  ti_sysbios_knl_Swi_Module_startup__E                                      
1001c239  ti_sysbios_knl_Swi_startup__E                                             
1001c23f  ti_sysbios_knl_Task_enable__E                                             
1001c245  ti_sysbios_BIOS_RtsGateProxy_enter__E                                     
1001c249  ti_sysbios_BIOS_RtsGateProxy_leave__E                                     
1001c24d  ti_sysbios_family_arm_cc26xx_Timer_getExpiredTicks__E                     
1001c251  ti_sysbios_family_arm_cc26xx_Timer_getPeriod__E                           
1001c255  ti_sysbios_family_arm_cc26xx_Timer_setPeriod__E                           
1001c259  ti_sysbios_family_arm_m3_Hwi_delete                                       
1001c25d  ti_sysbios_family_arm_m3_Hwi_destruct                                     
1001c261  ti_sysbios_family_arm_m3_TaskSupport_Module__startupDone__S               
1001c261  ti_sysbios_knl_Task_SupportProxy_Module__startupDone__S__mangled__        
1001c265  ti_sysbios_gates_GateHwi_query__E                                         
1001c265  xdc_runtime_Main_Module_GateProxy_query__E                                
1001c265  xdc_runtime_System_Module_GateProxy_query__E                              
1001c265  xdc_runtime_System_Module_GateProxy_query__E__mangled__                   
1001c269  ti_sysbios_gates_GateMutex_delete                                         
1001c26d  ti_sysbios_gates_GateMutex_destruct                                       
1001c271  ti_sysbios_BIOS_RtsGateProxy_query__E                                     
1001c271  ti_sysbios_BIOS_RtsGateProxy_query__E__mangled__                          
1001c271  ti_sysbios_gates_GateMutex_query__E                                       
1001c271  ti_sysbios_heaps_HeapMem_Module_GateProxy_query__E                        
1001c271  ti_sysbios_heaps_HeapMem_Module_GateProxy_query__E__mangled__             
1001c275  ti_sysbios_hal_Hwi_HwiProxy_Module__startupDone__S                        
1001c279  ti_sysbios_hal_Hwi_HwiProxy_delete                                        
1001c27d  ti_sysbios_hal_Hwi_HwiProxy_disableInterrupt__E                           
1001c27d  ti_sysbios_hal_Hwi_disableInterrupt__E                                    
1001c27d  ti_sysbios_hal_Hwi_disableInterrupt__E                                    
1001c281  ti_sysbios_hal_Hwi_HwiProxy_enableInterrupt__E                            
1001c281  ti_sysbios_hal_Hwi_enableInterrupt__E                                     
1001c281  ti_sysbios_hal_Hwi_enableInterrupt__E                                     
1001c285  ti_sysbios_hal_Hwi_HwiProxy_getStackInfo__E                               
1001c285  ti_sysbios_hal_Hwi_getStackInfo__E                                        
1001c285  ti_sysbios_hal_Hwi_getStackInfo__E                                        
1001c289  ti_sysbios_hal_Hwi_HwiProxy_startup__E                                    
1001c289  ti_sysbios_hal_Hwi_startup__E                                             
1001c289  ti_sysbios_hal_Hwi_startup__E                                             
1001c28d  ti_sysbios_hal_Hwi_HwiProxy_switchFromBootStack__E                        
1001c291  ti_sysbios_hal_Hwi_delete                                                 
1001c295  ti_sysbios_hal_Hwi_switchFromBootStack__E                                 
1001c295  ti_sysbios_hal_Hwi_switchFromBootStack__E                                 
1001c299  ti_sysbios_heaps_HeapMem_Module_GateProxy_enter__E                        
1001c29d  ti_sysbios_heaps_HeapMem_Module_GateProxy_leave__E                        
1001c2a1  ti_sysbios_heaps_HeapMem_isBlocking__E                                    
1001c2a5  ti_sysbios_knl_Clock_TimerProxy_Module__startupDone__S                    
1001c2a9  ti_sysbios_knl_Clock_TimerProxy_getExpiredTicks__E                        
1001c2ad  ti_sysbios_knl_Clock_TimerProxy_getPeriod__E                              
1001c2b1  ti_sysbios_knl_Clock_delete                                               
1001c2b5  ti_sysbios_knl_Clock_destruct                                             
1001c2b9  ti_sysbios_knl_Clock_removeI__E                                           
1001c2bd  ti_sysbios_knl_Clock_setTimeout__E                                        
1001c2c1  ti_sysbios_knl_Mailbox_delete                                             
1001c2c5  ti_sysbios_knl_Mailbox_destruct                                           
1001c2c9  ti_sysbios_knl_Queue_delete                                               
1001c2cd  ti_sysbios_knl_Queue_destruct                                             
1001c2d1  ti_sysbios_knl_Queue_head__E                                              
1001c2d5  ti_sysbios_knl_Queue_next__E                                              
1001c2d9  ti_sysbios_knl_Semaphore_delete                                           
1001c2dd  ti_sysbios_knl_Semaphore_destruct                                         
1001c2e1  ti_sysbios_knl_Swi_delete                                                 
1001c2e5  ti_sysbios_knl_Swi_destruct                                               
1001c2e9  ti_sysbios_knl_Swi_postInit__I                                            
1001c2ed  ti_sysbios_knl_Task_SupportProxy_Module__startupDone__S                   
1001c2f1  ti_sysbios_knl_Task_SupportProxy_getStackAlignment__E                     
1001c2f5  ti_sysbios_knl_Task_SupportProxy_start__E                                 
1001c2f9  ti_sysbios_knl_Task_SupportProxy_swap__E                                  
1001c2fd  ti_sysbios_knl_Task_delete                                                
1001c301  ti_sysbios_knl_Task_destruct                                              
1001c305  ti_sysbios_knl_Task_startup__E                                            
1001c309  xdc_runtime_Startup_startMods__I                                          
1001c401  xdc_runtime_Core_createObject__I                                          
1001c483  xdc_runtime_Error_policySpin__E                                           
1001c485  xdc_runtime_Memory_alloc__E                                               
1001c4f5  xdc_runtime_Core_deleteObject__I                                          
1001c555  xdc_runtime_Startup_exec__E                                               
1001c5a5  xdc_runtime_Assert_raise__I                                               
1001c5ed  xdc_runtime_Core_assignParams__I                                          
1001c635  xdc_runtime_Core_constructObject__I                                       
1001c67d  xdc_runtime_System_atexit__E                                              
1001c6b5  xdc_runtime_System_processAtExit__E                                       
1001c6e9  xdc_runtime_Core_assignLabel__I                                           
1001c719  xdc_runtime_Text_cordText__E                                              
1001c745  xdc_runtime_System_abort__E                                               
1001c765  xdc_runtime_Error_raiseX__E                                               
1001c781  xdc_runtime_Memory_valloc__E                                              
1001c79d  xdc_runtime_Core_destructObject__I                                        
1001c7b5  xdc_runtime_Error_check__E                                                
1001c7cd  xdc_runtime_System_exit__E                                                
1001c7e5  xdc_runtime_Text_ropeText__E                                              
1001c7fd  xdc_runtime_Memory_free__E                                                
1001c80d  xdc_runtime_SysCallback_abort__E                                          
1001c81d  xdc_runtime_SysCallback_exit__E                                           
1001c82d  xdc_runtime_Timestamp_SupportProxy_get32__E                               
1001c82d  xdc_runtime_Timestamp_get32__E                                            
1001c82d  xdc_runtime_Timestamp_get32__E                                            
1001c83d  xdc_runtime_Error_init__E                                                 
1001c849  xdc_runtime_Memory_calloc__E                                              
1001c855  xdc_runtime_Memory_getMaxDefaultTypeAlign__E                              
1001c875  xdc_runtime_Gate_leaveSystem__E                                           
1001c87b  xdc_runtime_System_Module_startup__E                                      
1001c881  xdc_runtime_Gate_enterSystem__E                                           
1001c885  xdc_runtime_Memory_HeapProxy_alloc__E                                     
1001c889  xdc_runtime_Memory_HeapProxy_free__E                                      
1001c88d  xdc_runtime_System_Module_GateProxy_enter__E                              
1001c891  xdc_runtime_System_Module_GateProxy_leave__E                              
1001c895  xdc_runtime_System_abortSpin__E                                           
1001c897  xdc_runtime_System_exitSpin__E                                            
1001c899  ti_sysbios_family_arm_m3_Hwi_dispatch__I                                  
1001c969  ti_sysbios_family_arm_m3_TaskSupport_buildTaskStack                       
1001c9b5  ti_sysbios_family_arm_m3_Hwi_initStacks__E                                
1001c9fd  ti_sysbios_family_arm_m3_Hwi_excHandlerAsm__I                             
1001ca1d  ti_sysbios_family_xxx_Hwi_switchAndRunFunc                                
1001ca3b  ti_sysbios_family_arm_m3_Hwi_pendSV__I                                    
1001ca53  ti_sysbios_family_arm_m3_Hwi_return                                       
1001ca55  ti_sysbios_family_arm_m3_TaskSupport_glue                                 
1001ca65  ti_sysbios_family_arm_m3_TaskSupport_swap__E                              
1001ca65  ti_sysbios_knl_Task_SupportProxy_swap__E__mangled__                       
1001ca6d  ti_sysbios_knl_Task_swapReturn                                            
1001ca97  ti_sysbios_rom_cortexm_cc13xx_CC13xx_getRevision__E                       
20000000  ti_sysbios_family_arm_m3_Hwi_ramVectors                                   
20000100  ti_sysbios_knl_Task_Module__state__V                                      
20000144  ti_sysbios_family_arm_m3_Hwi_Module__state__V                             
20000178  ti_sysbios_knl_Clock_Module__state__V                                     
200001a4  ti_sysbios_BIOS_Module__state__V                                          
200001c8  ti_sysbios_knl_Swi_Module__state__V                                       
200001e4  ti_sysbios_family_arm_cc26xx_Timer_Module__state__V                       
200001ec  ti_sysbios_family_arm_cc26xx_TimestampProvider_Module__state__V           
200001f0  xdc_runtime_Startup_Module__state__V                                      
200001f8  xdc_runtime_System_Module__state__V                                       
20000200  xdc_runtime_Memory_Module__state__V                                       
20000208  ti_sysbios_heaps_HeapMem_Instance_State_0_buf__A                          
20002508  task0Stack                                                                
20002808  ti_sysbios_knl_Task_Instance_State_0_stack__A                             
20002bfc  uartCC26XXObjects                                                         
20002d28  __CIOBUF_                                                                 
20002f48  ti_sysbios_family_arm_m3_Hwi_dispatchTable                                
20003010  pdmCC26XXI2SObjects                                                       
2000312c  xdc_runtime_SysMin_Module_State_0_outbuf__A                               
200031ac  PIN_HandleTable                                                           
20003228  pdmCC26XXObjects                                                          
20003358  task0Struct                                                               
20003420  displayUartObject                                                         
20003440  uartCC26XXRingBuffer                                                      
20003498  semStruct                                                                 
200034b4  g_ControlTable                                                            
20003544  parmbuf                                                                   
20003554  PIN_NumPins                                                               
2000355c  g_pControlTable                                                           
20003578  saSem                                                                     
2000357c  driverlib_release_0_47020                                                 
20003580  PowerCC26XX_module                                                        
20003690  ti_sysbios_knl_Swi_Module_State_0_readyQ__A                               
20003710  ti_sysbios_knl_Task_Object__table__V                                      
20003760  ti_sysbios_family_arm_cc26xx_Timer_Object__table__V                       
200037e8  ti_sysbios_gates_GateMutex_Object__table__V                               
20003854  ti_sysbios_knl_Swi_Object__table__V                                       
20003884  pdmParams                                                                 
200038a8  ti_sysbios_knl_Clock_Object__table__V                                     
200038c8  ti_sysbios_knl_Task_Module_State_0_readyQ__A                              
200038e8  ti_sysbios_family_arm_m3_Hwi_Object__table__V                             
20003900  ti_sysbios_heaps_HeapMem_Object__table__V                                 
20003920  streamNotification                                                        
20003938  buttonPinTable                                                            
20003944  ledPinTable                                                               
20003950  xdc_runtime_SysMin_Module__state__V                                       
2000395c  _lock                                                                     
20003960  _unlock                                                                   
2000396c  ti_sysbios_family_arm_m3_Hwi_Module__root__V                              
20003974  ti_sysbios_gates_GateHwi_Module__root__V                                  
2000397c  ti_sysbios_gates_GateMutex_Module__root__V                                
20003984  ti_sysbios_hal_Hwi_Module__root__V                                        
2000398c  ti_sysbios_heaps_HeapMem_Module__root__V                                  
20003994  ti_sysbios_knl_Clock_Module__root__V                                      
2000399c  ti_sysbios_knl_Event_Module__root__V                                      
200039a4  ti_sysbios_knl_Mailbox_Module__root__V                                    
200039ac  ti_sysbios_knl_Queue_Module__root__V                                      
200039b4  ti_sysbios_knl_Semaphore_Module__root__V                                  
200039bc  ti_sysbios_knl_Swi_Module__root__V                                        
200039c4  ti_sysbios_knl_Task_Module__root__V                                       
200039cc  xdc_runtime_Registry_Module__state__V                                     
200039d4  xdc_runtime_System_Module_State_0_atexitHandlers__A                       
200039dc  main_func_sp                                                              
200039e0  ti_sysbios_family_arm_m3_Hwi_Module_State_0_excContext__A                 
200039e4  ti_sysbios_family_arm_m3_Hwi_Module_State_0_excStack__A                   
200039e8  ti_sysbios_knl_Task_Module_State_0_idleTask__A                            
200039ec  ti_sysbios_family_arm_m3_Hwi_Module_State_0_excActive__A                  
20004d00  __stack                                                                   
20005000  __STACK_END                                                               
20005000  __STACK_TOP                                                               
e000e000  ti_sysbios_family_arm_m3_Hwi_nvic                                         
ffffffff  __TI_pprof_out_hndl                                                       
ffffffff  __TI_prof_data_size                                                       
ffffffff  __TI_prof_data_start                                                      
ffffffff  __binit__                                                                 
ffffffff  __c_args__                                                                
ffffffff  binit                                                                     
UNDEFED   SHT$$INIT_ARRAY$$Base                                                     
UNDEFED   SHT$$INIT_ARRAY$$Limit                                                    

[830 symbols]
